:020000040800F2
:100000000020001091D70208F9D702088550000897
:10001000F9D70208F9D70208F9D702080000000052
:10002000000000000000000000000000F9D70208F6
:10003000F9D7020800000000F9D70208B91100083A
:10004000F9D70208F9D70208F9D70208F9D7020848
:10005000F9D70208F9D70208C5240008F1250008DD
:10006000B5250008792500083D2500084539000818
:100070003539000825390008153900080539000808
:10008000F1380008DD380008F9D70208F9D702086E
:10009000F9D70208F9D70208F9D7020801250008A4
:1000A000D956000819570008C956000841570008DA
:1000B00009570008F9560008E9560008F9D7020860
:1000C000F9D70208F9D70208F9D70208F9D70208C8
:1000D000F9D70208E512000869120008ED110008BE
:1000E00089240008F9D70208F9D70208F9D70208CD
:1000F000F9D70208F9D70208F9D70208F9D7020898
:10010000000000000000000000000000F9D7020815
:10011000F9D70208F9D70208CDB20208B1B2020835
:10012000C9380008B5380008A13800088D38000823
:1001300079380008F9D7020800000000000000002C
:10014000F9D70208F9D70208F9D702080000000021
:10015000000000000000000000000000000000009F
:100160000000000000000000F9D70208F9D70208DB
:10017000F9D70208000000000000000000000000A5
:0801800000000000F9D702089D
:1001880070B4EFF31186502383F31288436B1A6817
:10019800D20720D45D686DB9446A826A944217D048
:1001A80081691144D9600ED9A21A5A60846200226A
:1001B80080F850201A6842F00102F1B21A6081F307
:1001C800118870BC704701698A1A5A608562EEE727
:1001D800012380F85030F1B281F3118870BC704768
:1001E800436A8269D154436A0169426B01338B4285
:1001F80028BF00234362002A2FD0EFF31181502338
:1002080083F31288436B1A68D2072CD470B45E68E3
:100218006EB9456A826A954217D084691444DC60D5
:100228000ED9AA1A5A608562002280F850201A68EE
:1002380042F00102C9B21A6081F3118870BC70479C
:100248000469A21A5A608662EEE7012380F85030EA
:10025800C9B281F3118870BC7047C26C136843F04F
:10026800800313607047C9B281F31188704700BFDB
:10027800026B10B462B1036CC2684469D11A013BC5
:10028800615C5DF8044B08BF13460364C8B270474D
:10029800016A4369C4685B5C0131A14228BF114609
:1002A80001625DF8044BD8B2704700BF436B13B1CD
:1002B80090F850007047836A406A181AB0FA80F0C4
:1002C80040097047416A836A99420AD3CB1A416B45
:1002D800026961B14968501E0B4483420AD2C01AB0
:1002E800704702691144CB1A416B0029F2D1501EA4
:1002F800C01A704700207047036B43B1026C5B68FB
:1003080093422FBF981AC0689B1AC0187047C269D9
:10031800036A9A422FBFD01AC0688018C01A704763
:100328000A4B30B503F1140493F900205D78072ACD
:10033800C8BF143A811804330D7313F8025C85544E
:1003480013F8012C0A76A342EED130BD0CFF020847
:1003580003682DE9F041DF691FB13B46BDE8F04174
:100368001847002A164611DD04460D460E4400E0E3
:1003780023689B68204698470028F9D0236815F819
:10038800011B1B6820469847AE42F1D1BDE8F081B9
:1003980000232322027043708370C37070472D239B
:1003A80043702E2303712F23C3717047002870B543
:1003B8001EDB0928044620DD012303EB83035B00D1
:1003C800B0FBF3F2092AF8D87BB10E4EB4FBF3F078
:1003D8000928CCBF57223022A6FB03E5024403FBC1
:1003E8001044EB0801F8012BF0D100230B7070BD0D
:1003F8002D230B7040420131DBE7303001F8010B4F
:10040800F3E700BFCDCCCCCC884230B44FF0010428
:100418002ED301FB04F4B0FBF4F58D42F9D284B17C
:10042800AAB901E0B0FBF4F5092DCCBF5722302260
:100438002A4404FB150003F8012BB4FBF1F4002C4B
:10044800F0D100221A7030BC7047B0FBF4F5092DCA
:10045800CCBF372230222A4404FB150003F8012BB5
:10046800B4FBF1F4002CF0D100221A7030BC7047B4
:100478000546002AEBD1D7E703685A1C02601970B9
:10048800704700BF2DE9F047089C2578002B80466F
:1004980089460CBF4FF0200A4FF0300A661C35B36E
:1004A800002A29DD334601E0024698B113F8011B02
:1004B800501E0029F8D1971E60B13D46013D5146B6
:1004C8004046C8476B1C002BF8DC257827EAE77004
:1004D800013055B1041B29464046C847301916F863
:1004E800015B002DF7D1BDE8F087BDE8F087002A51
:1004F80004DC2846BDE8F0870020EBE7571EDCE760
:1005080083684268D0ED037A00EB8301013393429C
:1005180081ED040A836004BF0023836000EB83033A
:1005280093ED047A036870EE277A9A42C0ED037A55
:1005380077EEC77AC0ED037A0CDA013307EE103A8A
:10054800F8EEC76AB7EE007A87EEA60A036030EEC7
:10055800070A704707EE102AB8EEC77A87EE870AAF
:10056800704700BF90ED057A90ED004AD0ED066A1D
:10057800D0ED014AD0ED047A90ED035AD0ED025A3D
:10058800A4EE007AB0EE406AB0EE470AB0EE667AA2
:10059800A6EE247A67EEC07AA0EE457AE6EE257AD2
:1005A80080ED057AC0ED067A704700BFD0ED057A78
:1005B80090ED013AD0ED003AD0ED064A90ED024AAE
:1005C80090ED077A90ED035A90ED086AD0ED045A41
:1005D800C0ED067AF0EE406A27EE830AC0ED056AA0
:1005E800A3EEA60A80ED087AA4EE240AA5EE470A2F
:1005F800A5EEC60A80ED070A704700BFD0ED007A65
:1006080090ED017A30EE670AE7EE007AB0EE670AFD
:10061800C0ED007A704700BF704700BF0A4491429E
:1006280014D030B40139551E41F2210211F8014F9E
:10063800082380EA042004044CBF82EA40004000FA
:10064800013B80B2F7D18D42F0D130BC704700BF7A
:10065800704700BF704700BF2DE9F04FDFF81CB2AC
:10066800DFF81CE2BBF80020DEF80060BBF90430BC
:10067800BBF90250BBF90A80C2EB261404FB04F450
:1006880024135200C2EBE60203FB04F305FB02F25B
:100698009B1303EBE223B3F5FA364FEAE37589B00F
:1006A80045F1FF373246A6FB0645CDE9024502FB78
:1006B80007F205EB4202CDE90467029EBBF9084048
:1006C800039208FB02FC4FEAE87906FB09CC3A469C
:1006D800A8FB0689049ECBF81830E51704FB02F244
:1006E80006FB0522A4FB0667E14417444FEA1822DB
:1006F80042EA096200924FEA292201923D03DDE9AC
:100708000078340345EA16553F19BBF80660069091
:1007180048EB05083C1C48F5004503EB8302A4FBA5
:10072800068906FB0599803213124FEA69064FEADB
:10073800E977079356EA07038A4600F09280DDE9D5
:100748000489BBF90E20DEF80440BBF910004946C5
:10075800C4F5801ED317DDE9024502FB01F108FB51
:100768000311A2FB08230B444FEA43492B46C11748
:1007780000FB03F304FB0133A0FB0401BBF90C40AD
:100788001944E30001937346DC170023009349EAF8
:10079800D2394FEA4248DDE9002310EB080041EB6B
:1007A8000901E50712184FEACE744B4145EA5E0588
:1007B800A41A65EB0305221945EB050312196B41D1
:1007C80099019001801841EA926159418B00820099
:1007D80043EA9073101943EB05018B00820043EA4A
:1007E800907310460019194632463B4669412CF071
:1007F800F7FDBBF916204C13450B45EAC14502FB32
:1008080004F6D31705FB0366A2FB05233344BBF9A3
:10081800146002FB04F405FB034406FB01FEA2FB83
:100828000523F717234400FB07EE540EA6FB0067C9
:10083800774444EAC3144FEAD64800194FEA63657F
:1008480048EA473869414FEAE74918EB0008BBF91D
:10085800124049EB01094FEA182646EA09662001C9
:100868003618069B0BB1360A1E60BAF1000F02D08B
:10087800079BCAF8003009B0BDE8F08FEC340020BF
:10088800241E0020704700BF2DE9F041364F374D38
:10089800B7F80AC02A893B89B7F91240B7F914E0BA
:1008A800EE68B7F90250B7F90E80A2EB0C0203FB11
:1008B80002F3DA139644E30293FBFEF31344A3F521
:1008C8007A6E0EFB0EF4B7F90CC0FB6122130EFB17
:1008D80005F5B7F9044002FB08F8ED1202FB0CF22B
:1008E800B7F900C00EFB04F405EBE825B7F920E0E2
:1008F800FF88121402EB643205EB8C0505FA0EF53D
:100908000232023592104CF25034A6EBA50502F5DE
:10091800004244FA0EF404FB05F407FB02F2D20B82
:10092800002CB9BFB4FBF2F252006400B4FBF2F23F
:10093800141204FB04F50E4E40F6DE3404FB05F4F5
:1009480003EB830306FB02F524145B0004EB254448
:10095800083304F6CF641B1102EB241200B10260C5
:1009680001B10B60BDE8F081B8340020241E0020DE
:1009780043E3FFFF2DE9F04FDFF8F8C1DFF8F8E1B6
:10098800BCF80A70DEF81060BCF80C30BCF808A09F
:100998003C028BB0361B4FF00004CDE90034009CBC
:1009A800BCF806304FEA17654FF0000767EB0507FC
:1009B800B946B046A4FB06670024CDE90634009C7E
:1009C800002304FB09770024CDE90034AAFB08239F
:1009D800CDE90223039AF30D00930AFB092303933D
:1009E800009B43EA47230093029B4FEAD31AFB1567
:1009F8000193039B4AEA436ADDE9002344464D46D6
:100A0800CDE90845069C12F5FA62A4FB086743F194
:100A1800000304FB0977CDE90623BCF80440039BD7
:100A2800BCF802204FEAE31B230C0593230404932C
:100A3800340A44EA07643D12DDE904674FEAC23824
:100A480016EB0A0647EB0B0718EB0408DDE906343A
:100A58004FEA524949EB0509B3F5FA6F74F10004FE
:100A6800B246BB463CDADDE90067BC00B20044EAA6
:100A78009673B41847EB030522463C462B4602FB07
:100A880004F406FB0344A2FB06232344940844EA27
:100A980083749D105B104FEA3202B8EB040869EBCF
:100AA8000509BAEB020A6BEB030BDDE90623304CB0
:100AB8004FF0FF35A242AB412CDBDDE90856A5FB20
:100AC800052305FB06F403EB4403D40F44EA43046F
:100AD800DD17DDE90623121B63EB0503CDE90623C9
:100AE800DEF81440A4FB082304FB0933540D44EA40
:100AF800C3245D15B4EB0A0A65EB0B0B4FEADA3336
:100B080043EA4B4300B1036009B1069B0B600BB08D
:100B1800BDE8F08F40F6AC52B4184FF0000347EB35
:100B280003052246A2FB022304FB05F403EB44035E
:100B3800941843EB0305A4185D414FEA850CA60001
:100B48004CEA947CB41A6CEB0305DF00D6006D10F8
:100B58004FEA340447EA5277921B63EB0703B8EB7A
:100B6800040869EB05091AEB020A4BEB030BA4E72F
:100B780024FAFFFFDC340020241E002050F8043C37
:100B8800012280F84520103803B11847704700BF8C
:100B980090F8203033B1012B03D14FF400638382E6
:100BA800704770474FF480638382704770B504467E
:100BB80082B01430E56D06236A464321A847B0B1D8
:100BC8009DF804009DF800609DF801109DF8025002
:100BD8009DF803209DF8053041EA062143EA0023E9
:100BE80042EA0522A187E287A4F84030012002B03A
:100BF80070BD00BF70B5044682B00830656A062330
:100C08006A463B21A847A8B19DF804009DF80060FA
:100C18009DF801109DF802509DF803209DF80530BD
:100C280041EA062143EA002342EA0522E1822283BF
:100C38006383012002B070BD10B490E80600047B05
:100C480040690223A3404B6013685DF8044B4FF6DC
:100C5800FE710B401360FFF793BA00BF70B40468CD
:100C6800037B2268022101FA03F31A4213D0426976
:100C78000A49582000FB02124FF6FE765068528946
:100C8800C5680068296831402960C168D24392B2BA
:100C98000A40C260636070BC704700BF70470020A4
:100CA80030B4094B1C7864B1084B002503EBC4042D
:100CB8001A6899885562D06808330143A342D16005
:100CC800F6D130BC704700BF304A0020344A0020BB
:100CD80010B40268047B11680223A340194209D0AA
:100CE8000649406800240C7001684FF6FE742140E4
:100CF800016053605DF8044B704700BFFD38002069
:100D0800F0B4334C00EB800004EB80046468002CE2
:100D18005BD0304E49004FF42040CDB2B061A1699C
:100D2800090444D460682C4F45F08071384041F480
:100D3800903101434FF420406160B06103E0411EEF
:100D4800002838D00846A1698F07F8D54FF420400D
:100D5800A262B06102E0421E68B31046A2691106A1
:100D6800F9D562681C4945F0007545F480350A409C
:100D780015434FF420406560B06102E0421ED0B1D7
:100D88001046A2699207F9D5A362A3694FF42040DF
:100D98009B06B06105D4431E68B11846A3699B063B
:100DA800F9D52023B061E3610120F0BC7047411EF2
:100DB80008B10846B3E7094A138801339BB24FF0DC
:100DC800FF31B1611380F0BC70472046F0BC70471A
:100DD80028620020241E0020009800FCCC3000204F
:100DE800134600200A4668218AE700BF30B504464A
:100DF800C06C61710368A26823F00103036087B0C7
:100E0800A379009213F004023DD04FF4805213F0FE
:100E18000203019244D102934FF4806300220393AA
:100E280011F00103059237D1049308238D07694611
:100E380048BF049329F058F96079E36CA17900F070
:100E48000202002A15BF4FF440324FF480324FF4AB
:100E58000034002410F0010F586808BF2246CC0760
:100E68004CBF024320EA02025A609A6809074CBF45
:100E780042F0080222F008029A601A6842F0010261
:100E88001A6007B030BD13F0020301920BD04FF483
:100E9800005513460295C1E7042304930C23C5E7C4
:100EA8004FF40053B7E70293B8E700BF10B5044604
:100EB800C06CA160036823F001030360A37986B0C6
:100EC80013F00402009141D04FF4805213F0020352
:100ED800019244D102934FF4806362790393D1075E
:100EE8004FF000030493059345BF0423049308239C
:100EF8000C236946920748BF049329F0F5F86079F6
:100F0800E36CA17900F00202002A15BF4FF44032C9
:100F18004FF480324FF40034002410F0010F586869
:100F280008BF2246CC074CBF024320EA02025A609F
:100F38009A6809074CBF42F0080222F008029A603A
:100F48001A6842F001021A6006B010BD13F00203DD
:100F5800019207D04FF4005113460291BDE74FF4B8
:100F68000053B7E70293B8E7002326220360027014
:100F780027228270012243600271837170472DE934
:100F8800F341056906460F467DBBD0F80080C8F3DB
:100F98000A0323B30023D6F80080019321F00CFA4A
:100FA800042819D1214C236943F001032361BBB202
:100FB800A8F8003021F000FA04282ED108F1020325
:100FC8000193019B3F0C1F8021F0F6F92369042847
:100FD80023F00103236125D06FF0010505E021F01E
:100FE800EBF9042805D04FF0FF35284602B0BDE8DC
:100FF800F0810E4C236943F002032361C4F8148086
:10100800236943F04003236121F0D6F923690428BA
:1010180023F002032361BDD0E5E7236923F0010330
:101028002361D9E7336804333360DEE700200240E8
:10103800F8B504460D468E180027B54201D120693F
:10104800F8BDE368591CE160234415F8012B1A72B6
:101058000429F2D1A1682046FFF791FFE7602061DB
:10106800EBE700BF204B5B68C3F3080330B4BBB9A0
:10107800EFF31183A3B91D4B1D4C1868A16800BF7D
:101088001A689042F9D11B4B1C684FF47A7202FB24
:1010980004F3591AB1FBF4F130BC02FB001070479D
:1010A800EFF31182102383F3128811498C680B68BF
:1010B80013F4803F104B02D0012018608C680B4954
:1010C800D2B20D68186882F311880A4B19684FF478
:1010D8007A72284402FB01F31B1B30BCB3FBF1F30B
:1010E80002FB0030704700BF00ED00E0886200207E
:1010F80010E000E08C620020846200202DE9F84FA7
:101108008046FFF7AFFF254E2549DFF8A0E0254AC6
:10111800254D844610274FF47A740120DEF80430F8
:10112800C3F30803D3B9EFF31183BBB90B68D2F843
:1011380008A000BFD1F800904B45F7D1D6F800B011
:1011480004FB0BF9A9EB0A09B9FBFBF904FB0393B0
:10115800A3EB0C034345E1D3BDE8F88FEFF3118A05
:1011680087F31288D2F808B01368DB0344BF2860FD
:10117800D2F808B00B68D5F800905FFA8AFA8AF3BB
:101188001188D6F800A0994404FB0AF3A3EB0B03DB
:10119800B3FBFAF304FB0933DAE700BF8C620020E3
:1011A8008862002010E000E08462002000ED00E08A
:1011B80030B4EFF31183102282F312880649074CEA
:1011C8000A680748013200250A602560DBB2026818
:1011D80083F3118830BC7047886200208462002045
:1011E80010E000E01D4B70B59C68E36C226BDD6974
:1011F800C2B1636B2BB12B0702D5E36C08221A62CC
:1012080070BD2A06F7D5A26A616A8A421FD0511CAE
:10121800A069A162825C2069E66C81423285EAD3CA
:10122800A362E8E7A906E4D5E26A1AB1988C80B20D
:101238009047DEE7E1699B8C6069DBB24E1CE66192
:101248004354E169E368994228BFE261D1E7E26C5F
:10125800136823F080031360CDE700BF742C0020CF
:101268001D4B70B55C68E36C226BDD69C2B1636BC2
:101278002BB12B0702D5E36C08221A6270BD2A062F
:10128800F7D5A26A616A8A421FD0511CA069A1627F
:10129800825C2069E66C81423285EAD3A362E8E782
:1012A800A906E4D5E26A1AB1988C80B29047DEE7C5
:1012B800E1699B8C6069DBB24E1CE6614354E169CD
:1012C800E368994228BFE261D1E7E26C136823F032
:1012D80080031360CDE700BF742C00201D4B70B550
:1012E8001C68E36C226BDD69C2B1636B2BB12B0701
:1012F80002D5E36C08221A6270BD2A06F7D5A26AE5
:10130800616A8A421FD0511CA069A162825C20696F
:10131800E66C81423285EAD3A362E8E7A906E4D500
:10132800E26A1AB1988C80B29047DEE7E1699B8C3B
:101338006069DBB24E1CE6614354E169E368994297
:1013480028BFE261D1E7E26C136823F080031360E1
:10135800CDE700BF742C002003685B6A03B118470F
:10136800704700BF03681B6A03B11847704700BF86
:1013780003682DE9F041DF691FB13B46BDE8F04144
:101388001847002A164611DD04460D460E4400E0B3
:1013980023689B68204698470028F9D0236815F8E9
:1013A800011B1B6820469847AE42F1D1BDE8F08189
:1013B80003689B69184700BF03685B69184700BF4B
:1013C8000368DB68184700BF03689B68184700BFBD
:1013D80003685B68184700BF03681B68184700BFAD
:1013E800014B1868F8E700BFC45C0020054B53F8B0
:1013F800203033B11A689B88918A0B4218BF1B04AE
:10140800936170475462002003682DE9F04F03F19F
:101418003845644EAD0A0124755D05F01F066D0957
:10142800022D04FA06F400F0A280032D00F0A48037
:10143800012D52D08088B0FA80F4C4F11F04A4B200
:10144800E50803EB850504F007042E6AA4000F27BE
:10145800A74026EA07062E622E6A01F0030702FA61
:1014680004F47A1E3443012AC1F3810CC1F3001835
:101478002C62C1F3411135D9C60700F19780850761
:1014880000F1A380440700F1B180020700F1BF809A
:10149800C60600F1CD80850600F1DB80440600F128
:1014A800E980020600F1F780C60500F1058185058F
:1014B80000F11381440500F12181020500F12F811B
:1014C800C60400F13D81850400F14B81440400F11C
:1014D8005981020455D4BDE8F08F334D6E69344309
:1014E8006C61A7E7002422464FF0010E4FF0030974
:1014F80004E00132102A04F10204ECD00EFA02F6DC
:1015080036EA0005F5D1D3F808A009FA04F5ED4349
:101518000AEA050AC3F808A0D3F808B00CFA04FAD6
:101528004AEA0B0AC3F808A0B3F804A01FFA8AFA1B
:101538002AEA06069E80B3F804A008FA02F646EAEC
:101548000A06B6B29E801E682E401E60D3F800A020
:1015580007FA04F646EA0A061E60D3F80CA001FA58
:1015680004F605EA0A0A46EA0A05DD60C1E70E4DF7
:10157800AE693443AC615DE70B4DEE693443EC6111
:1015880058E71A6822F040421A601A6842EA8777D8
:101598001F60DA6822F0404242EA8171D960BDE8F2
:1015A800F08F00BF08230308001002401A6822F0D9
:1015B80003021A601A683A431A60DA6822F00302D2
:1015C8000A438507DA607FF55DAF1A6822F00C02DE
:1015D8001A601A6842EA87021A60DA6822F00C0276
:1015E80042EA81024407DA607FF54FAF1A6822F0B9
:1015F80030021A601A6842EA07121A60DA6822F0A2
:10160800300242EA0112DA6002077FF541AF1A6838
:1016180022F0C0021A601A6842EA87121A60DA6871
:1016280022F0C00242EA8112C606DA607FF533AFC3
:101638001A6822F440721A601A6842EA07221A608D
:10164800DA6822F4407242EA01228506DA607FF500
:1016580025AF1A6822F440621A601A6842EA8722A3
:101668001A60DA6822F4406242EA81224406DA60AB
:101678007FF517AF1A6822F440521A601A6842EAD6
:1016880007321A60DA6822F4405242EA0132DA601C
:1016980002067FF509AF1A6822F440421A601A68F8
:1016A80042EA87321A60DA6822F4404242EA81321A
:1016B800C605DA607FF5FBAE1A6822F440321A607C
:1016C8001A6842EA07421A60DA6822F4403242EAAB
:1016D80001428505DA607FF5EDAE1A6822F44022F2
:1016E8001A601A6842EA87421A60DA6822F44022CD
:1016F80042EA81424405DA607FF5DFAE1A6822F4D7
:1017080040121A601A6842EA07521A60DA6822F42C
:10171800401242EA0152DA6002057FF5D1AE1A683A
:1017280022F440021A601A6842EA87521A60DA689C
:1017380022F4400242EA8152C604DA607FF5C3AE61
:101748001A6822F040721A601A6842EA07621A6040
:10175800DA6822F0407242EA01628504DA607FF5B5
:10176800B5AE1A6822F040621A601A6842EA8762C7
:101778001A60DA6822F0406242EA81624404DA6060
:101788007FF5A7AE1A6822F040521A601A6842EA3A
:1017980007721A60DA6822F0405242EA0172DA608F
:1017A80097E600BF036803F138422DE9F04F920A2B
:1017B800584DAA5C02F01F0552090124022A04FAB6
:1017C80005F400F08C80032A00F08E80012A3CD0BA
:1017D80001F003077A1E012AC1F3810CC1F3001836
:1017E8008088C1F3411135D9C60700F19780850774
:1017F80000F1A380440700F1B180020700F1BF8027
:10180800C60600F1CD80850600F1DB80440600F1B4
:10181800E980020600F1F780C60500F1058185051B
:1018280000F11381440500F12181020500F12F81A7
:10183800C60400F13D81850400F14B81440400F1A8
:101848005981020455D4BDE8F08F334A55692C43B9
:101858005461BDE7002422464FF0010E4FF0030902
:1018680004E00132102A04F10204ECD00EFA02F668
:1018780036EA0005F5D1D3F808A009FA04F5ED43D6
:101888000AEA050AC3F808A0D3F808B00CFA04FA63
:101898004AEA0B0AC3F808A0B3F804A01FFA8AFAA8
:1018A8002AEA06069E80B3F804A008FA02F646EA79
:1018B8000A06B6B29E801E682E401E60D3F800A0AD
:1018C80007FA04F646EA0A061E60D3F80CA001FAE5
:1018D80004F605EA0A0A46EA0A05DD60C1E70E4A87
:1018E80095692C43946173E70B4AD5692C43D461FD
:1018F8006EE71A6822F040421A601A6842EA87774F
:101908001F60DA6822F0404242EA8171D960BDE87E
:10191800F08F00BF08230308001002401A6822F065
:1019280003021A601A683A431A60DA6822F003025E
:101938000A438507DA607FF55DAF1A6822F00C026A
:101948001A601A6842EA87021A60DA6822F00C0202
:1019580042EA81024407DA607FF54FAF1A6822F045
:1019680030021A601A6842EA07121A60DA6822F02E
:10197800300242EA0112DA6002077FF541AF1A68C5
:1019880022F0C0021A601A6842EA87121A60DA68FE
:1019980022F0C00242EA8112C606DA607FF533AF50
:1019A8001A6822F440721A601A6842EA07221A601A
:1019B800DA6822F4407242EA01228506DA607FF58D
:1019C80025AF1A6822F440621A601A6842EA872230
:1019D8001A60DA6822F4406242EA81224406DA6038
:1019E8007FF517AF1A6822F440521A601A6842EA63
:1019F80007321A60DA6822F4405242EA0132DA60A9
:101A080002067FF509AF1A6822F440421A601A6884
:101A180042EA87321A60DA6822F4404242EA8132A6
:101A2800C605DA607FF5FBAE1A6822F440321A6008
:101A38001A6842EA07421A60DA6822F4403242EA37
:101A480001428505DA607FF5EDAE1A6822F440227E
:101A58001A601A6842EA87421A60DA6822F4402259
:101A680042EA81424405DA607FF5DFAE1A6822F463
:101A780040121A601A6842EA07521A60DA6822F4B9
:101A8800401242EA0152DA6002057FF5D1AE1A68C7
:101A980022F440021A601A6842EA87521A60DA6829
:101AA80022F4400242EA8152C604DA607FF5C3AEEE
:101AB8001A6822F040721A601A6842EA07621A60CD
:101AC800DA6822F0407242EA01628504DA607FF542
:101AD800B5AE1A6822F040621A601A6842EA876254
:101AE8001A60DA6822F0406242EA81624404DA60ED
:101AF8007FF5A7AE1A6822F040521A601A6842EAC7
:101B080007721A60DA6822F0405242EA0172DA601B
:101B180097E600BF10B50409013C052C17D80D4BFA
:101B280033F8142000F00F0042FA00F313F0010319
:101B38000DD0012303FA00F0013810402BF0A0FC6F
:101B4800054A064B125D104403EBC00010BD00208F
:101B580010BD00BFE01B0308EC1B03085045002024
:101B68002DE9F04F4A484B4B4B4C4FF090414FF00A
:101B7800010A4FF002094FF004084FF0080C4FF02B
:101B8800100E20274026802530F8022B12F0010F76
:101B980003D01960A3F804A0083312F0020F03D091
:101BA8001960A3F80490083312F0040F03D01960E9
:101BB800A3F80480083312F0080F03D01960A3F8C3
:101BC80004C0083312F0100F03D01960A3F804E022
:101BD800083312F0200F02D019609F80083312F0EA
:101BE800400F02D019609E80083312F0800F02D097
:101BF80019609D80083312F4807F05D04FF4807BF4
:101C08001960A3F804B0083312F4007F05D04FF42C
:101C1800007B1960A3F804B0083312F4806F05D074
:101C28004FF4806B1960A3F804B0083312F4006F06
:101C380005D04FF4006B1960A3F804B0083312F410
:101C4800805F05D04FF4805B1960A3F804B00833B7
:101C580012F4005F05D04FF4005B1960A3F804B0DC
:101C6800083312F4804F05D04FF4804B1960A3F865
:101C780004B00833D20B04D04FF4004219609A80A4
:101C8800083301F58061A1427FF47EAFBDE8F08F93
:101C9800E01B03085045002000180048002867D0C2
:101CA80003682DE9F04F03F138445C4EA40A01257E
:101CB800345D04F01F066409022C05FA06F558D0B5
:101CC800032C00F0A580012C58D08088B0FA80F44D
:101CD800C4F11F04A4B2E50803EB850504F007046A
:101CE8002E6AA4000F27A74026EA07062E622E6A4E
:101CF80001F00307A2407C1E3243012CC1F3810C82
:101D0800C1F300182A62C1F341113CD9C60700F19A
:101D18008980850700F19580440700F1A3800207B8
:101D280000F1B180C60600F1BF80850600F1CD80C4
:101D3800440600F1DB80020600F1E980C60500F1E7
:101D4800F780850500F10581440500F1138102053E
:101D580000F12181C60400F12F81850400F13D8145
:101D6800440400F14B81020400F15981BDE8F08F71
:101D780070472B4CA6693543A561A6E7284C6669D0
:101D880035436561A1E7002422464FF0010E4FF06C
:101D9800030904E00132102A04F10204E6D00EFA25
:101DA80002F636EA0005F5D1D3F808A009FA04F5D9
:101DB800ED430AEA050AC3F808A0D3F808B00CFAFC
:101DC80004FA4AEA0B0AC3F808A0B3F804A01FFAF9
:101DD8008AFA2AEA06069E80B3F804A008FA02F6F0
:101DE80046EA0A06B6B29E801E682E401E60D3F8E8
:101DF80000A007FA04F646EA0A061E60D3F80CA00B
:101E080001FA04F605EA0A0A46EA0A05DD60C1E7AE
:101E1800034CE6693543E56157E700BF082303082B
:101E2800001002401A6822F003021A601A683A4346
:101E38001A60DA6822F003020A438507DA607FF540
:101E48006BAF1A6822F00C021A601A6842EA87021D
:101E58001A60DA6822F00C0242EA81024407DA606A
:101E68007FF55DAF1A6822F030021A601A6842EAFC
:101E780007121A60DA6822F0300242EA0112DA60C8
:101E880002077FF54FAF1A6822F0C0021A601A687D
:101E980042EA87121A60DA6822F0C00242EA811226
:101EA800C606DA607FF541AF1A6822F440721A60FC
:101EB8001A6842EA07221A60DA6822F4407242EA93
:101EC80001228506DA607FF533AF1A6822F4406292
:101ED8001A601A6842EA87221A60DA6822F44062B5
:101EE80042EA81224406DA607FF525AF1A6822F4B7
:101EF80040521A601A6842EA07321A60DA6822F415
:101F0800405242EA0132DA6002067FF517AF1A68DA
:101F180022F440421A601A6842EA87321A60DA6884
:101F280022F4404242EA8132C605DA607FF509AF01
:101F38001A6822F440321A601A6842EA07421A60A4
:101F4800DA6822F4403242EA01428505DA607FF518
:101F5800FBAE1A6822F440221A601A6842EA8742E5
:101F68001A60DA6822F4402242EA81424405DA60C3
:101F78007FF5EDAE1A6822F440121A601A6842EA38
:101F880007521A60DA6822F4401242EA0152DA6013
:101F980002057FF5DFAE1A6822F440021A601A685B
:101FA80042EA87521A60DA6822F4400242EA815211
:101FB800C604DA607FF5D1AE1A6822F040721A6062
:101FC8001A6842EA07621A60DA6822F0407242EA46
:101FD80001628504DA607FF5C3AE1A6822F04062B8
:101FE8001A601A6842EA87621A60DA6822F0406268
:101FF80042EA81624404DA607FF5B5AE1A6822F0DD
:1020080040521A601A6842EA07721A60DA6822F0C7
:10201800405242EA0172DA6002047FF5A7AE1A68FC
:1020280022F040421A601A6842EA87771F60DA682D
:1020380022F0404242EA8171D960BDE8F08F00BFCA
:10204800002852D0036803F138422DE9F04F920A74
:10205800504DAA5C02F01F0552090124022A04FA15
:1020680005F443D0032A00F09080012A43D001F000
:1020780003077A1E012AC1F3810CC1F30018808876
:10208800C1F341113CD9C60700F18880850700F1EA
:102098009480440700F1A280020700F1B080C606D0
:1020A80000F1BE80850600F1CC80440600F1DA809C
:1020B800020600F1E880C60500F1F680850500F10A
:1020C8000481440500F11281020500F12081C60453
:1020D80000F12E81850400F13C81440400F14A811D
:1020E800020400F15881BDE8F08F70472A4A9569CB
:1020F8002C439461BBE7284A55692C435461B6E7E1
:10210800002422464FF0010E4FF0030904E001328B
:10211800102A04F10204E6D00EFA02F636EA0005A7
:10212800F5D1D3F808A009FA04F5ED430AEA050A3F
:10213800C3F808A0D3F808B00CFA04FA4AEA0B0A64
:10214800C3F808A0B3F804A01FFA8AFA2AEA060618
:102158009E80B3F804A008FA02F646EA0A06B6B268
:102168009E801E682E401E60D3F800A007FA04F671
:1021780046EA0A061E60D3F80CA001FA04F605EA3E
:102188000A0A46EA0A05DD60C1E7034AD5692C4315
:10219800D4616CE708230308001002401A6822F093
:1021A80003021A601A683A431A60DA6822F00302D6
:1021B8000A438507DA607FF56CAF1A6822F00C02D3
:1021C8001A601A6842EA87021A60DA6822F00C027A
:1021D80042EA81024407DA607FF55EAF1A6822F0AE
:1021E80030021A601A6842EA07121A60DA6822F0A6
:1021F800300242EA0112DA6002077FF550AF1A682E
:1022080022F0C0021A601A6842EA87121A60DA6875
:1022180022F0C00242EA8112C606DA607FF542AFB8
:102228001A6822F440721A601A6842EA07221A6091
:10223800DA6822F4407242EA01228506DA607FF504
:1022480034AF1A6822F440621A601A6842EA872298
:102258001A60DA6822F4406242EA81224406DA60AF
:102268007FF526AF1A6822F440521A601A6842EACB
:1022780007321A60DA6822F4405242EA0132DA6020
:1022880002067FF518AF1A6822F440421A601A68ED
:1022980042EA87321A60DA6822F4404242EA81321E
:1022A800C605DA607FF50AAF1A6822F440321A6070
:1022B8001A6842EA07421A60DA6822F4403242EAAF
:1022C80001428505DA607FF5FCAE1A6822F44022E7
:1022D8001A601A6842EA87421A60DA6822F44022D1
:1022E80042EA81424405DA607FF5EEAE1A6822F4CC
:1022F80040121A601A6842EA07521A60DA6822F431
:10230800401242EA0152DA6002057FF5E0AE1A682F
:1023180022F440021A601A6842EA87521A60DA68A0
:1023280022F4400242EA8152C604DA607FF5D2AE56
:102338001A6822F040721A601A6842EA07621A6044
:10234800DA6822F0407242EA01628504DA607FF5B9
:10235800C4AE1A6822F040621A601A6842EA8762BC
:102368001A60DA6822F0406242EA81624404DA6064
:102378007FF5B6AE1A6822F040521A601A6842EA2F
:1023880007721A60DA6822F0405242EA0172DA6093
:1023980002047FF5A8AE1A6822F040421A601A6853
:1023A80042EA87771F60DA6822F0404242EA817188
:1023B800D960BDE8F08F00BF10B1036882881A8524
:1023C800704700BF10B1036882889A61704700BFE8
:1023D80038B100298388026814BF002110218B407E
:1023E800936170470E4B1B8801463BB90D4B0E4A53
:1023F8001B7810680BB981F00101E9E70B4B5A69AA
:102408001AB118B91A68106058747047084A1868E1
:102418001188084A92FBF1F2012102605974704751
:10242800606200206262002064620020686200200E
:102438008062002020A1070010B40A4B0A4A1C78C9
:1024480001238340234052F8200029B9B3FA83F1CD
:1024580049095DF8044BBBE7191C18BF01215DF859
:10246800044BB5E7506200205462002030B1036885
:1024780082881B8A1A4214BF01200020704700BFBF
:102488002DE9F0410B4E356873691D4010D0DFF817
:1024980028800127B5FA85F4C4F11F0408EB8403EA
:1024A80007FA04F4D86903689847A5437461F1D121
:1024B800BDE8F08100040140241E00202DE9F04110
:1024C8000B4E356873691D4010D0DFF8288001274E
:1024D800B5FA85F4C4F11F0408EB840307FA04F481
:1024E800D86903689847A5437461F1D1BDE8F081C4
:1024F80000040140241E00202DE9F0410B4E3568F0
:1025080073691D4010D0DFF828800127B5FA85F4DB
:10251800C4F11F0408EB840307FA04F4D8690368BC
:102528009847A5437461F1D1BDE8F08100040140EA
:10253800241E00202DE9F0410B4E356873691D40BB
:1025480010D0DFF828800127B5FA85F4C4F11F04FC
:1025580008EB840307FA04F4D86903689847A5438D
:102568007461F1D1BDE8F08100040140241E00200F
:102578002DE9F0410B4E356873691D4010D0DFF826
:1025880028800127B5FA85F4C4F11F0408EB8403F9
:1025980007FA04F4D86903689847A5437461F1D130
:1025A800BDE8F08100040140241E00202DE9F0411F
:1025B8000B4E356873691D4010D0DFF8288001275D
:1025C800B5FA85F4C4F11F0408EB840307FA04F490
:1025D800D86903689847A5437461F1D1BDE8F081D3
:1025E80000040140241E00202DE9F0410B4E3568FF
:1025F80073691D4010D0DFF828800127B5FA85F4EB
:10260800C4F11F0408EB840307FA04F4D8690368CB
:102618009847A5437461F1D1BDE8F08100040140F9
:10262800241E0020002800F084802DE9F0418488D1
:10263800B4FA84F4C4F11F04651C82B06BD0E5B20F
:1026480005F0FC0606F1804606F5803605F0030520
:10265800D6F808E0374F0068AD004FF00F0C0CFAC1
:1026680005FC2EEA0C0E07EB840CC0F38720CCF88F
:102678001C10C6F808E0D6F80880DFF8C4C0DFF8F8
:10268800C4E000FA05F10120A04041EA0801B16068
:10269800CCF80000DEF80050274EDFF8AC80C143CC
:1026A8000D40CEF8005035680D403560DEF800501A
:1026B800224E0543CEF80050D8F800500D40C8F817
:1026C80000505CF8085C34442940102B4CF8081C76
:1026D800247DACF1080C21D003F1804303F582334B
:1026E800196801431960274497F85C30934212DD5A
:1026F8002644002196F824308DF8043094110123E3
:1027080001A887F85C208DF805408DF806108DF833
:10271800073027F045FD02B0BDE8F081D8F8003059
:102728000343C8F80030DCF800100143CCF800106F
:10273800D9E77047241E0020040401400CFF02085A
:1027480014040140000401400804014070B5044627
:1027580090F85900002833D104F11405236E802223
:102768006B2128469847642003F0C0FD236E284655
:1027780003226B219847236E94F854201921284688
:1027880098470F2003F0B2FD236E94F85220284694
:102798001A219847236E284618221B219847236E32
:1027A800284618221C219847236E284602223721E2
:1027B80098472846236E01223821BDE87040184703
:1027C800FFF7A8F90546FFF751FE0028C4D115B157
:1027D8002023E871AB7128460021FFF731FC214620
:1027E800054B41F8103F28460823F022FFF71AFF4F
:1027F80028461DF033FEAFE7850B00080B490C4A4D
:102808008B6943F0010310B58B611368094C43F4DD
:102818008053136004F11C00402200212DF0BDFA02
:102828004FF0FF33E365C4F85F3010BD001002407D
:1028380000000140241E00202DE9F04104461846FE
:102848000D46164698462AF021F92768E67228446C
:10285800A07229467D69434632462046AC46BDE80B
:10286800F0416047036810B504461B689847236821
:1028780020469B689847A37B0133A37310BD00BF14
:10288800427A02B9704710B504460368406804F1FB
:102898000A0198470023637210BD00BF437A5A1C8F
:1028A8000344D2B242729972037A934200D802B9B1
:1028B800704710B504460368406804F10A01984758
:1028C8000023637210BD00BF30B40B4D002305F127
:1028D8002C0101E0272B0CD011F8132082424FEA7B
:1028E800430403F10103F5D12C4494F82D0030BCC6
:1028F8007047002030BC70470CFF020870B5448850
:1029080006460D46C4F30B042246002128462DF046
:1029180044FA3369094A934209D3094A934206D2D1
:10292800224628461946BDE870402AF0B7BF23B1B1
:1029380021462846BDE87040184770BD1860030856
:102948000D610308064B07498B4202D30023184642
:1029580070471A88C2F30B029042F8D01433F3E799
:10296800B85B030818600308024A136823EA0000EA
:1029780010607047B43C0020F8B5174D2B78A32B96
:1029880028D16B78BE2B25D1022229464FF6FF703D
:10299800FDF744FE114FAC1C22884AB1A618BE426E
:1029A80018D2052A16D92146FDF738FE3446F3E732
:1029B80021460222FDF732FE0222A118FDF72EFE63
:1029C8000634074B641B1C8041F60F53C31A584248
:1029D8005841F8BD0020F8BD00F0030800000408C5
:1029E800CE3000202DE9F04FDFF848914C4F8BB0E6
:1029F8000326A7EB09071822002104A82DF0CDF91A
:102A0800484BCDF8109005971A69120604D5464A26
:102A18005A6002F188325A6001228DF8242034224B
:102A2800DA60424B424C1B88ADF8003002226946FE
:102A380004A8FEF7FDFA022269464FF6FF70FDF77B
:102A4800EDFDDFF8F4A080464FF0000B544536D377
:102A58000AAC002524F8245D0222214604A8FEF7CA
:102A6800E7FA022221464046FDF7D8FD40BAC043A6
:102A7800ADF80800022202A904A8FEF7D9FA0798BF
:102A880060B106ABC0F10402294618442DF085F95F
:102A9800069904A8FEF773FA079508909DF8243064
:102AA800089A23B11F490B6943F080030B61013E6B
:102AB8002DD0002A9FD1FFF75FFF50B32CE0658827
:102AC8008DF80DB0C5F30B05AB1DADF808302388A4
:102AD800C3F30B02ADF80A201B0B062202A904A8B7
:102AE8008DF80C30FEF7A4FA062202A94046FDF73D
:102AF80095FD616880462A4604A8FEF799FA616840
:102B080040462A46FDF78AFD143480469EE7002A8F
:102B1800D1D0052002F0D4FF0BB0BDE8F08F00BF84
:102B280000000408002002402301674586FF0208D0
:102B3800B85B030800F00308186003080378202B2B
:102B4800024600F10100F9D0092BF7D02D2B2CD02B
:102B58002B2B03BF5378B7EE000A0246B7EE000AE4
:102B6800A3F13001C8B209289FED467A10D8F2EED9
:102B7800046A07EE901AF8EEE77A12F8013FE7EEDA
:102B8800267AA3F13001C8B20928B0EE677AF0D9E5
:102B98002E2B4CD003F0DF03452B0BD0F7EE007A39
:102BA80067EE276A20EE260A70475378BFEE000AC0
:102BB8000246D5E710B451782D2959D02B290ABFE0
:102BC8009178501C901C0024A1F13003092B53D894
:102BD800002303EB830301EB430310F8011FA1F16A
:102BE8003002092AA3F13003F3D9B3F59A7F28BF3D
:102BF8004FF49A73072B42D9DFED236A1A46F7EE92
:102C0800007A083A072A67EEA67AFAD803F007038B
:102C18002BB1F2EE046A013B67EEA67AFBD124B32E
:102C2800C7EE276A5DF8044B20EE260A70475378F2
:102C3800A3F13001C8B2092802F10102AAD8F2EEC4
:102C4800046AF0EE665A07EE901AF8EEE77A12F880
:102C5800013F87EEA66AA3F13001C8B2092866EEE3
:102C6800A56A37EE067AEED994E767EE276AD9E7C0
:102C7800901C91780124A7E7F7EE007ACFE7F7EEEA
:102C8800007AC5E70000000020BCBE4CB5EEC00AC3
:102C9800DFED317AF1EE10FACCBF30EE270A30EED4
:102CA800670ADFED2E7A20EE270A30B5FDEEC07AEE
:102CB80087B017EE904A054684EAE470002303A91A
:102CC800A0EBE47001930093029326F0C5FB002C5F
:102CD800ACBF20232D2303A88DF8003029F0D6FEA1
:102CE800012803A924D002282DD0032805BF3023AA
:102CF800684668468DF801302DF075F8684629F069
:102D0800C5FE0338C4B22246694628462DF0C9F8E4
:102D180000232B55284629F0B9FE2E22431C2A549D
:102D28000DEB0401E8182DF07BF8284607B030BDFC
:102D3800302368468DF801308DF802308DF8033065
:102D48002DF051F8DAE7302368468DF801308DF818
:102D580002302DF048F8D1E76F12033A00007A44A8
:102D68002DE9F041064615460846B6FBF2F43CB993
:102D780005FB1464124B1B5D00F8013BBDE8F081B4
:102D8800B4FBF2F767B90E4B05FB174705FB146454
:102D9800DA5D00F8012B1B5D00F8013BBDE8F0810E
:102DA800B7FBF2F8B8F1000F02D04046FFF7D8FFA2
:102DB80005FB1878024B13F8082000F8012BE3E70D
:102DC800E427030830B402681146531C036011F865
:102DD800024B0160D31C517803609378151D056080
:102DE8001B0443EA0123D078234343EA006030BC44
:102DF800704700BF0368591C1A46016012F8021B8D
:102E08000260587841EA0020704700BF03685A1CE6
:102E180002601878704700BF38B504460068154648
:102E28002AF03CFD22682A44226038BD036810B4A9
:102E38000A0A5C1C04601A7003685A1C0260197044
:102E48005DF8044B704700BF03685A1C026010B459
:102E5800197003680A0A5C1C04601A7003680A0C7B
:102E68005C1C04601A700368090E5A1C0260197011
:102E78005DF8044B704700BF03685A1C0260197064
:102E88000368090A5A1C0260197070472DE9F04757
:102E9800002488B080460F461E46A14605AD531C47
:102EA8000393117839B3252933D1931CCDF81090A9
:102EB8000393507830284ED04FF0000AA0F1300329
:102EC800DBB2092B42D96C2819D0642800F0938012
:102ED80024D825281CD063D9582876D063281BD13C
:102EE80031784046B847039A531C03931178043647
:102EF80001340029D7D1204608B0BDE8F087039BEC
:102F08005A1C03921B78642B7CD02AD8252B54D1C9
:102F1800252140460134B847039AC0E7732833D0C7
:102F280044D975284FD106F1040E30682B4600228B
:102F38000A217646FDF768FA049A00955346394601
:102F48004046FDF79FFA039A0444A8E704AA03A998
:102F58001FF064FCB7E7D31C039390784FF0010A85
:102F6800ACE7732B10D05BD9752B3AD0782B96D160
:102F7800A3F15802B2FA82F2306852092B461021A6
:102F88000436FDF741FAD7E73368049A00933946C7
:102F980000234046FDF776FA04360444039A7EE798
:102FA8000028B9D1204608B0BDE8F0876E28B3D113
:102FB800039A336804361C6071E72AD9582BD7D096
:102FC800632B8DD06BE77828A6D1A0F15802B2FA0E
:102FD80082F2306852092B461021FDF715FA0436A3
:102FE800AAE706F1040E30682B4600220A2176462D
:102FF800FDF70AFAA0E7331D306829461E46FDF79B
:10300800D5F999E7331D306829461E46FDF7CEF9F4
:1030180092E7002B7FF443AF204608B0BDE8F08765
:103028006E2BC6D03BE700BF0EB400B584B005AB2D
:10303800019053F8042B0649039301A8FFF726FFD4
:10304800019B00221A7004B05DF804EB03B07047CE
:10305800810400080FB430B583B006AB0A490B48A9
:1030680053F8042B096800680193FFF70FFF084C19
:1030780005462068FEF7A0F90028FAD0284603B0D4
:10308800BDE8304004B07047682C00206C2C00204C
:10309800C45C0020DFED2B7AB4EEE70AF1EE10FAFB
:1030A8004ADDDFED296A9FED297A01E0B0EE670A73
:1030B800B4EEC70AF1EE10FA70EE667AF6DC9FED10
:1030C800247AF4EEC77AF1EE10FA38D5DFED1E6AED
:1030D8009FED207A01E0F0EE407AF4EEC77AF1EE47
:1030E80010FA37EEA60AF6D4DFED1B7AB4EEE70A3B
:1030F800F1EE10FA14DDDFED137A37EEC00A60EE58
:10310800006A9FED166A9FED167ADFED167AA6EE35
:10311800867A20EE266AE6EE877AA6EE270A7047B8
:10312800DFED117AB4EEE70AF1EE10FA44BFDFEDF5
:10313800087A37EEC00AE2E7F0EE407ABFE7B0EE71
:10314800670AD1E7DB0F4940DB0FC940E4CB1641E2
:10315800DB0F49C0E4CB16C1DB0FC93F92E741B989
:103168009730083C15A82ABEDB0FC9BF80EAE07378
:10317800A3EBE0738B4205DB002801DD401A7047A2
:1031880002D17047002070470844704709B909E028
:10319800194690FBF1F301FB13030846002BF7D106
:1031A800084670470146FBE79FED317A70EE077AD3
:1031B800FDEEE76A16EE903A2033402B02D99FEDD8
:1031C8002D0A7047B4EEC70AF1EE10FA0FDDB0EE23
:1031D800677A9FED296ADFED296A01E0B0EE677A28
:1031E800B4EEE67AF1EE10FA77EEC67AF6DC9FEDE9
:1031F800247AF4EEC77AF1EE10FA0FD5B0EE677ABA
:103208009FED1D6ADFED1F6A01E0B0EE677AB4EE4C
:10321800E67AF1EE10FA77EE867AF6D49FED147A14
:10322800F4EEC77AF1EE10FA1DDC9FED177AF4EE92
:10323800C77AF1EE10FA44BF9FED117A77EE677AFC
:1032480027EEA76ADFED115ADFED116A9FED117ABB
:10325800E6EE256A67EE865AA6EE267AE5EE877AC6
:10326800B0EE670A70479FED0C7A77EE677AE7E76A
:10327800DB0FC93F00000000DB0FC940E4CB16415B
:10328800DB0F49C0E4CB16C1DB0FC9BF92E741B9D8
:103298009730083C15A82ABEDB0F494010B507EE49
:1032A800901A2DED028BB8EE678ADFED217A28EEB1
:1032B800008A044628EE278AB0EE480A2AF0AEFCB7
:1032C800F0EE408AB0EE480A2AF00AFCF7EE007ADF
:1032D8009FED187AF0EE675AE8EE875A0023A3614B
:1032E800B0EE676AC7EEA56A63612362E361A8EE80
:1032F800C76ABDEC028B77EEC07AB6EE007AF8EEBC
:10330800005A27EE877A20EE250A27EE267A26EE3F
:10331800266A67EEA67A20EE260A84ED046AC4EDD2
:10332800017A84ED007A84ED027A84ED030A10BDF7
:1033380027D4D236F304353F10B44C09012250F893
:10334800243001F01F0102FA01F10B4340F8243048
:103358005DF8044B704700BF4B0901F01F0150F89E
:103368002320012303FA01F1114214BF184600205B
:10337800704700BFF0B5254F254B2649DFF8B4C08C
:10338800254E264D264CDFF8B0E0264801223A703B
:1033980005270A75CF741A7015218CF803201B2293
:1033A80014279971DA7100210222DF70597099701F
:1033B80059711A71717132716A7064262A700F21FD
:1033C8000422194F194B267061702025A270212103
:1033D8002C268EF8022044F268224570817006700F
:1033E8003A8003F1EA0546223E20132128241A7068
:1033F80058709970DA70187159719C754E33AB42D8
:10340800F5D10B4B1A701A731A76F0BD9C57002031
:1034180038340020304F002050300020102D00207C
:10342800633B0020E036002048470020783B00201E
:103438004C360020A4340020CC4A0020B0F1FF3FD5
:103448000AD0022810B403DC5DF8044BFDF758BC21
:1034580000205DF8044B70470020704710B4044604
:10346800134690F904000A4661795DF8044BE5E7D4
:103478000378012B00D070473122F421EEE700BF1A
:10348800044B93F820209201343202F0FC02F4211C
:10349800E4E700BFB83400202E22F421DEE700BFA5
:1034A8000278012A00D070474821D7E70278012A1C
:1034B80000D070475821D1E7F0B55B4B5B4A97B015
:1034C8001968914200AF00F0A3805949594A002376
:1034D8004FF47000C1F888003B607B60136843F4C8
:1034E8008033136003E03B68B3F5A04F09D013683D
:1034F80003F400337B603B6801333B607B68002B3F
:10350800F1D04C4B1B6813F4003318BF01237B60C8
:103518007B68012B52D0464C464B474AE260474AEB
:10352800596A11605A6A42F080725A625A6942F4C2
:10353800FC025A610025032207F10801012341F624
:10354800FF764FF09040FD60BE603A73BB7316F093
:103558007FFA4FF6FF7307F108013948BB6016F090
:1035680077FA07F108013748374E16F071FA07F174
:103578000801364816F06CFA07F10801344816F0CD
:1035880067FA07F10801334816F062FA07F10800F4
:1035980016F06EF8BB683049304AA1FB0313304976
:1035A8009B0CF0204FF0070E5C370B60566084F8D8
:1035B80023009560C2F800E0BD46F0BD294A1D4BC6
:1035C800122111605A685A605A685A605A6842F45F
:1035D80080625A605A6822F47C125A605A6842F42F
:1035E800E8125A601A6842F080721A601A689201EA
:1035F800FCD559680F4A21F003015960596841F018
:1036080002015960536803F00C03082BFAD182E7D2
:1036180000221A6062B6144B1B6883F30888134BA8
:103628001B689847FEE700BFFC9F0020EFBEADDE99
:1036380000ED00E0001002400005FA055C4F002094
:1036480000040048000800483F190100000C004829
:10365800001000480014004883DE1B4310E000E01F
:103668008C6200200020024000D8FF1F04D8FF1FF2
:1036780070B50F4C0F4DC0EBC00004EB80046869B7
:1036880026693043686182B09209667BA160002593
:10369800012101A863618DF804608DF805208DF87B
:1036A80006508DF8071026F07BFD02B070BD00BFF4
:1036B800F81A002000100240074BC0EBC00030B4DD
:1036C80003EB8000054C056963692B436361017650
:1036D800427630BC704700BFF81A00200010024044
:1036E8002DE9F04F5E4C54F8204083B0002C71D087
:1036F800666D984691465B4B7268E264A1602360F0
:1037080004F15A014FF4807304F5AD726161A2614E
:10371800E36023610746307E25F08AF9F068A8B196
:10372800514B00215A68904203F11C0300F092802B
:1037380001310C29F6D100207A1CD2B20C21FFF7F6
:10374800BBFFE36CF26822632433A364B068D8B18A
:10375800454B00215A68904203F11C0378D001318F
:103768000C29F7D100257A1CD2B20B212846FFF785
:10377800A3FF2346F27E3D492846FFF779FFE36C15
:10378800B26862632833636494F85900FEF7C2F99B
:10379800054694F85800FEF7BDF918F0080F824660
:1037A80096F819B01AD0CDB118F0110F4FF00B03DD
:1037B80007F1010714BF4E213E21EF715A46AB7144
:1037C8002846FEF76BFA18F0010F45D0236B5BB360
:1037D800636B4BB3204603B0BDE8F08F18F0010FC0
:1037E8000CBF4FF02E084FF04E0819F0020F09D009
:1037F80045B10B227B1CAA71EB7128465A464146FB
:10380800FEF74CFA19F0010FE0D0BAF1000FDDD045
:1038180001370C238AF807705A4641468AF8063061
:103828005046FEF73BFAD1E7337FB27E8DF804208D
:103838009B090021012201A88DF805308DF806109A
:103848008DF8072026F0ACFC204603B0BDE8F08FC9
:10385800CDB288E7C8B26FE72846FEF7ADFDB5E7F9
:10386800742C002088FF0208F81A0020410C000878
:103878000348D0F83C3113B100F59A7018477047E7
:10388800F81A00200348D0F8203113B100F58C70E5
:1038980018477047F81A00200348D0F804310BB1D4
:1038A800FC301847704700BFF81A00200348D0F8CA
:1038B800E8300BB1E0301847704700BFF81A002015
:1038C8000348D0F8CC300BB1C4301847704700BF5C
:1038D800F81A00200348D0F8B0300BB1A8301847C8
:1038E800704700BFF81A00200348D0F894300BB195
:1038F8008C301847704700BFF81A00200248836FC1
:103908000BB1703018477047F81A00200248C36D91
:103918000BB1543018477047F81A00200248036C5E
:103928000BB1383018477047F81A00200248436A2C
:103938000BB11C3018477047F81A002002488368FA
:1039480003B11847704700BFF81A0020F0B53E4C85
:10395800059D00EB800004EB80046468002C71D0A6
:103968003A4E49004FF42040CFB2B061A169090432
:1039780054D46068DFF8E0E047F4903100EA0E00C4
:1039880001434FF420406160B06103E0411E00280C
:1039980048D00846A1698907F8D54FF42040A262AB
:1039A800B06103E0421E00283CD01046A2695206CE
:1039B800F8D5274A6168DFF8A0E0B06142EA03421F
:1039C800174301EA0E0217436760C3B1013BDBB23C
:1039D80001332B44A0694FF4204210F0040002F197
:1039E800FF3207D1511C26D0A06910F0040002F163
:1039F800FF32F7D0626A05F8012B9D42EAD14FF4F5
:103A08002040B06102E0431E60B11846A3699B06DE
:103A1800F9D52023B061E3610120F0BD411E08B152
:103A28000846A3E70B4A138801339BB24FF0FF31D6
:103A38001380B161F0BD0749B2610B8801339BB2B5
:103A48000B80F0BD2046F0BD28620020241E002017
:103A580000240002CC300020009800FC70B590F9DA
:103A680004506C1C82B00AD0022D08DC16460A46A7
:103A7800417900962846FFF769FF02B070BD002023
:103A880002B070BD70B50378012B82B004D1062353
:103A98006A46F721FFF7E2FF9DF801209DF8043000
:103AA8009DF800609DF803509DF802409DF80500C0
:103AB800074912011B0142EA063243EA053342EA8A
:103AC800141243EA10134A600B6002B070BD00BFC5
:103AD800241E002010B582B001AA0323F621FFF7A7
:103AE800BDFF9DF80530094A9DF804409DF8060081
:103AF800B2F9202006491B0243EA04430343C2F1FA
:103B08000802D340CB6002B010BD00BFB83400201B
:103B1800241E002000B583B001AA0223F621FFF776
:103B28009DFF9DF804109DF80530034A43EA0123E0
:103B3800138103B05DF804FB241E002000B5037850
:103B4800012B83B004D1032301AA0021FFF786FFCC
:103B58009DF805309DF804209DF806001B0243EAF5
:103B68000243184303B05DF804FB00BF08B5FFF734
:103B7800E5FF014B586108BD241E002008B5FFF77A
:103B8800DDFF014B186108BD241E0020F0B585B08B
:103B980002AB04460093032206231E210020FFF7F0
:103BA800D5FE00283CD09DF808509DF809109DF8D6
:103BB8000A709DF80B209DF80C609DF80D3041EAC5
:103BC800052142EA072243EA062309B212B21BB2D0
:103BD800144D06EE901A07EE102A07EE903AF8EE0A
:103BE800E66A95ED005AD5ED025A95ED016AB8EEF0
:103BF800C77AF8EEE77A66EE856A27EE257A67EEE9
:103C0800867AFDEEE66ABDEEC77AFDEEE77A16EE35
:103C1800901A17EE102A17EE903A2180A28063803E
:103C280005B0F0BD000000202DE9F043322083B03C
:103C380002F05CFB0022104611231E21FFF7FEFB59
:103C4800602301221E210020FFF7F8FB642002F008
:103C58004DFB6846FFF79AFF0024DFF89081254660
:103C680026460A27012302221E210020FFF7E6FB31
:103C7800322002F03BFB6846FFF788FFBDF902E0FF
:103C8800BDF90410BDF900208E457346A8BF0B4648
:103C98009342A8BF134643454FF0010075440C44B6
:103CA8001644C0F29380FDF7A1FB013FDAD14FF033
:103CB80001090022104612231E21FFF7BFFBDFF87F
:103CC8002C810A27012302221E210020FFF7B6FBC0
:103CD800322002F00BFB6846FFF758FFBDF902E0FF
:103CE800BDF90410BDF900208E457346A8BF0B46E8
:103CF8009342A8BF134643454FF00100A5EB0E05BC
:103D0800A4EB0104A6EB02065DDBFDF76FFB013FA8
:103D1800D8D107EE906AF8EEE76A07EE905AB8EE47
:103D2800E77A07EE904ADFED2B5A9FED2B5A2B4E80
:103D3800F8EEE77A85EEA66A0022104670231E2167
:103D4800C5EE876A85EE277AB0EEC66AF0EEE66AB7
:103D5800F0EEC77A86ED006AC6ED016AC6ED027A12
:103D6800FFF76CFB202301221E210020FFF766FBD2
:103D78000023184602221E21FFF760FB642002F090
:103D8800B5FAB9F1000F04D14FF07E533360736078
:103D9800B360134C206810B1FEF768FB18B9012016
:103DA80003B0BDE8F0830F490F4B41F8643FF022A0
:103DB80008232068FEF736FC20681CF04FFB012022
:103DC80003B0BDE8F0834FF00009A2E74FF0000907
:103DD8006FE700BF00406F4601C05E46000000204C
:103DE800B0340020241E00205D06000801F0FFFF0B
:103DF800F0B587B00DF10F030546009302220123A9
:103E08000C210020FFF7A2FD18B19DF80F30DB0749
:103E180003D40024204607B0F0BD04AB009303226E
:103E280006230C210020FFF791FD0DF10F030093ED
:103E3800092201230C210020FFF788FD04460028F1
:103E4800E7D09DF80F0010F00C00E2D19DF811E0CA
:103E58009DF810109DF813709DF812209DF81560BC
:103E68009DF8143041EA0E2142EA072243EA06236C
:103E7800C1EB8131C2EB8232C3EB833389009200FC
:103E88009B0029806A80AB800A2201230C21FFF75E
:103E9800D5FABFE710B5002384B018460A220C21D2
:103EA800FFF7CCFA142002F021FA0F230A220C2182
:103EB8000020FFF7C3FA0A2002F018FA03AB0093B8
:103EC800102203230C210020FFF740FD0A2002F0F6
:103ED8000DFA002318460A220C21FFF7AFFA0DF15C
:103EE8000B040A2002F002FA0094012302220C219A
:103EF8000020FFF72BFD0094012309220C2100204C
:103F0800FFF724FD01230A220C210020FFF796FA6F
:103F1800012004B010BD00BF00B583B0002000929E
:103F28000A466821FFF712FD03B05DF804FB00BFE5
:103F38001749184B184A194810B4D1F8884044F466
:103F48007004C1F888401C6844F001041C605C6877
:103F580022405A601A6822F0847222F480321A6071
:103F68001A6822F480221A605A6822F4FE025A6003
:103F7800DA6A22F00F02DA621A6B002410404FF05E
:103F8800006218639C608A605DF8044B704700BF4C
:103F980000ED00E0001002400CC07FF8CCFC00FFF0
:103FA80038B50B4C23688BB15A68821A002A05462B
:103FB80004DA0CE05A68AA1A002A07DB9A68226019
:103FC80018461A6890472368002BF3D138BD38BDCE
:103FD800FC3F00200B4B002210B4027203F5A074C2
:103FE800032102E0072A09DC9979890702D51979A2
:103FF800815401329C4203F11403F3D15DF8044B60
:10400800704700BF1023030810230370704700BFD8
:10401800012310B415211424222244704171C27066
:104028000370037183705DF8044B704708B510F096
:1040380025FC024B024ADA60FEE700BF00ED00E013
:104048000400FA05024A034B1278197816F0BEBD2F
:1040580078210020792100202DE9F0470569C368FF
:104068001D4028D00F4606464FF000484FF0000983
:10407800B5FA85F328FA03F2D2431B3B32611540A7
:10408800042B16D8DFE803F03129211903007B6AD5
:10409800002B32D003F1FF3A1FFA8AFAC7F82490AE
:1040A8003C6A34B123682046514698476468002C1E
:1040B800F8D1002DDCD1BDE8F0873868716B036852
:1040C80089B29847002DD3D1F5E77868B16B0368BA
:1040D80089B29847002DCBD1EDE7B868F16B03683A
:1040E80089B29847002DC3D1E5E7F868316C0368B9
:1040F80089B29847002DBBD1DDE7F36A1FFA83FA2E
:10410800CEE700BF2DE9F04F2DED028BA0F10A0399
:1041180089B00C46E72B00F24686DFE813F01C0155
:104128004406440644064406440644064406440637
:104138004406440644064406440644064406440627
:1041480044064406440644064406440644062D0133
:1041580044064406440659054406440644064B01F1
:104168004406580144062D024406220244061A0257
:104178004406C9034406F201440644064406EB011A
:10418800E4014406DD0144064406D6014406AE01B6
:104198004406440644069C01440644064406440674
:1041A800CF054406FC0044064304EF0544064406D4
:1041B8004406440644064406440617054406DA0441
:1041C8004406A6044406520444060602440644066D
:1041D80044064406A4056905C7051306E800440615
:1041E8004406900310034406D902BD02440644065F
:1041F80044064406B20244064406910244064406B4
:10420800440682026B027C033A03440644064406D1
:104218002B0344061C0323044406440644064406B0
:104228004406440644064406440644064406440636
:10423800440644064406A4054406440644064406C7
:104248004406440644064406440644064406440616
:104258004406440644064406440644064406440606
:1042680044064406440644064406440644064406F6
:1042780044064406440644064406440644064406E6
:1042880044064406440644064406440644064406D6
:1042980044064406440644064406440644064406C6
:1042A80044064406440644064406440644064406B6
:1042B80044064406440644064406440644064406A6
:1042C8004406440644064406440644064406440696
:1042D8004406440644064406440644064406440686
:1042E800440644064406440644061804EE03AE4E4B
:1042F800337853B1AD4F002537F8021F2046FEF73B
:10430800BBFD33780135AB42F6DC012009B0BDECCA
:10431800028BBDE8F08FA44E3378002BF5D0A44F64
:104328000025B846236817F81520591C21601A7013
:1043380098F8011001EB810101EB810101F2EE21F6
:1043480089B22046FEF798FD33780135AB4208F173
:104358000208E7DCD9E7974D284628F097FB0028A4
:10436800D3DD2B460544226813F8011B501C9D42DF
:1043780020601170F7D1C8E78F4D05F150062878F5
:1043880023F080FC2368027A591C21601A70236884
:104398006A78591C21601A702368AA78591C216010
:1043A8001A702368EA780435591CAE4221601A70E5
:1043B800E5D1AAE70B68814A581C1178206019706A
:1043C80023685278591C216001201A709EE77C4DA1
:1043D8000B682A7A591C21601A70A98B2046FEF7AF
:1043E8004BFD298B2046FEF747FD698B2046FEF7DB
:1043F80043FD2368EA7C591C21601A70A98C204669
:10440800FEF73AFDE98C2046FEF736FD2368AA7FC1
:10441800591C21601A70236895F82020591C2160C6
:104428001A70698C2046FEF727FD2368EA7A591C22
:1044380021601A70E9682046FEF706FD23682A7C89
:10444800591C21601A70236895F82120591C216095
:1044580001201A705AE70B6800255A1C0A6020468A
:1044680029461D70FEF7F0FC29462046FEF7ECFCB5
:1044780029462046FEF7E8FC47E70B684F4A514DAE
:104488001178514A581C2060197011682046FEF7AF
:10449800DBFC23684A4A591C127A21601A70298861
:1044A8002046FEF7E9FCA9882046FEF7E5FC2989A5
:1044B8002046FEF7E1FC00212046FEF7DDFC204601
:1044C8000021FEF7D9FC012020E7084608223C49D4
:1044D800FEF7A2FC012019E70B683C4A581C9178AA
:1044E800206019706CE70B6801229918216010464A
:1044F8001A700BE7364B08461968FEF7A5FC012031
:1045080004E7344D344E05F1280795F90210334B72
:1045180093F906208A4203F1080300F047849E427B
:10452800F6D10835BD42F0D1EFE60B682C4A2D498B
:10453800D0782D4A5D1C2560187023684979581C6D
:10454800206019702368D278591C216001201A70E4
:10455800DCE60B681A4A591C527D216001201A704A
:10456800D4E6224D05F1800655F8041F2046FEF7D3
:104578006BFCAE42F8D1C8E61D4D05F14006B5F812
:1045880080102046FEF778FC236895F88220591C95
:1045980021601A70236895F883200435591CAE42AF
:1045A80021601A70EBD1B0E634370020D66E0020B7
:1045B800985400205830002038340020343400202B
:1045C800304F0020A02C0020B43C0020F0700020C8
:1045D8001C350020544400200C4F0020E44E0020DD
:1045E80028440020483B0020A4340020EC37002059
:1045F800F03700200A689D4B9D491878551C2560A6
:10460800107022685878551C2560107022689B78B5
:10461800501C206013702046C988FEF72DFC01202D
:1046280074E6934D08462988FEF726FC69882046DB
:10463800FEF722FC2046A988FEF71EFC012065E64D
:104648008C4D05F16006A9882046FEF715FCE9881F
:104658002046FEF711FC29892046FEF70DFC236849
:10466800AA7A591C21601A702368EA7A591C2160B9
:104678001A7055F80C1B2046FEF7E6FBB542E2D14E
:1046880043E67D4952232268501C2060137011F8BC
:10469800013F002BF7D138E67848002322680568E7
:1046A80003EB4301561C6D5C266015700268256893
:1046B8000A446E1C527826602A70026825680A44EB
:1046C80001339278691C0A2B21602A70E6D11CE616
:1046D8006B4D0B682A68591C127821601A702B6878
:1046E80022689978531C2360002311702A68216876
:1046F8001A4401335279481C032B20600A70F5D103
:1047080023682A68591C127A21601A7023682A685B
:10471800591CD27821601A7023682A68591C1279AA
:1047280021601A702B6820465989FEF7A5FB2A6874
:104738002368527A591C21601A702A6840E6514B46
:1047480008461968FEF780FB4F4B20461988FEF78C
:1047580093FB0120DAE54D4B4D49B3F9003081FB5D
:104768000321DB17C3EBA101204689B2FEF784FBC6
:104778000120CBE5474D0846298AFEF77DFB698A6B
:104788002046FEF779FB2046A98AFEF775FB012033
:10479800BCE5DFF818E10027FEB271460023226865
:1047A800501C206016702268501C2060137022680C
:1047B80011F8010F0133551C062B25601070EED13E
:1047C8000137062F0EF1060EE6D133490023226881
:1047D800501C206017702268501C206013702268DB
:1047E80011F8010F0133551C0B2B25601070EED109
:1047F80023682A4A581C0721206019702368002161
:10480800581C20601970236892F8F020591C216008
:1048180001201A707AE50B68214A224910781B4A50
:104828005D1C2560187023688978581C20601970F1
:1048380023689278591C216001201A7066E51A4D88
:1048480008462988FEF718FB69882046FEF714FBFE
:10485800B5F904300E4AD91782FB0323C1EBA30133
:10486800204689B2FEF708FB01204FE5102D0020F5
:104878003430002084580020B0FF02084836002059
:10488800CC7000203C2D0020BC1F0020A434002048
:104898006766666648470020D3380020F037002056
:1048A800CC4A002028440020CC360020AF38002015
:1048B8009F4B03F15A0522685979501C20601170EA
:1048C80022681978501C2060117022685978501C91
:1048D8002060117022689978501C2060117022683D
:1048E800D978501C20601170226819790633501C41
:1048F8009D4220601170DED107E58E4B03F17005F3
:1049080022681978501C2060117022685978501C50
:104918002060117022689978501C206011702268FC
:10492800D978501C2060117022681979501C2060B9
:10493800117022685979501C206011702268997989
:104948000733501C9D4220601170D9D1DDE47A4DA7
:104958000846E989FEF790FA2046A989FEF78CFAFD
:104968000120D3E40B68754F591C3A7821601A70FE
:104978003B78002B3FF4C9AC0025EEB230461EF060
:1049880083FB23684278591C216030461A701EF058
:104998007BFB01892046FEF76FFA3B780135AB4275
:1049A800EBDCB2E40B6800255A1C0A601D700B682A
:1049B8005A1C0A601D700B685A1C0A6029461D7033
:1049C80053E500212046FEF757FA00212046FEF75E
:1049D80053FA00212046FEF74FFA2368584D002667
:1049E8005A1C22601E7023682A68591C92F82C20D1
:1049F80021601A7023682A68591C92F836202160B1
:104A08001A7023682A68591C92F8372021601A7096
:104A180023685A1C22601E7023685A1C22601E706C
:104A280023685A1C22601E702B682046598FFEF797
:104A380023FA2B682046198FFEF71EFA23682A6886
:104A4800591C92F82E2021601A7023685A1C226083
:104A58001E702B682046598EFEF70EFA2B682046EA
:104A6800998EFEF709FA012050E4364E0B687279E8
:104A7800334D591C21601A702B682046198CFEF79B
:104A8800FBF92B682046D98BFEF7F6F97189204689
:104A9800FEF7F2F9B1892046FEF7EEF92B682046B9
:104AA800598CFEF7E9F92B682046998CFEF7E4F952
:104AB800F1892046FEF7E0F9318A2046FEF7DCF955
:104AC8002A68236892F82620591C216001201A7050
:104AD8001CE41C4EF378002B00F060820B6808225F
:104AE800591C21601A7023680122991821601A70D4
:104AF8002368154D591C2A7921601A702368AA78F1
:104B0800591C21601A7029882046FEF7B5F9E989F1
:104B18002046FEF7B1F92368F279591C21601A7012
:104B28002368EA78591C216001201A70FFF7EEBB50
:104B3800682E0020EC550020284400201D5000203D
:104B480048360020CC4A00204847002016F022F8BA
:104B5800FF28064600F02E8208A9002501F8125DFC
:104B68000DF10D008DF80D5015F0F4FF08A800F8B0
:104B7800115D15F0E3FF08A800F8105D15F0D2FFED
:104B880008A820F8085D15F0C1FF23685A1C2260A8
:104B98001E7023689DF80D20591C21601A70236827
:104BA8009DF80E20591C21601A7023689DF80F206B
:104BB800591C21601A7023689DF81020591C216027
:104BC8001A702046BDF81810FEF756F9FFF79DBB7E
:104BD800A54D08462988FEF74FF9A9882046FEF713
:104BE8004BF920462989FEF747F90120FFF78EBBCC
:104BF8009E4B9B8AB3F5006F00F2CE81B3F5806FB0
:104C080000F2EF81B3F5007F34BF01270227984DEA
:104C180005F10C0655F8041B91FBF7F1204689B203
:104C2800FEF72AF9AE42F5D1924D934F05F10C06E5
:104C3800B5EC010AD7ED087A80EE270A28F0A2FF22
:104C480081B22046FEF718F9AE42F1D18B4D05F13D
:104C58000C0655F8041B204689B2FEF70DF9B5423B
:104C6800F7D1FFF752BB00258146DFF84882DFF80D
:104C780048B2059504950695079501214FF6FF7AE8
:104C880005E001350B2D00F0AF8018F9011F4F1C0E
:104C98004AFA05F3F5D0DE07F3D5BBF800302B410F
:104CA800D807EED506A8FEF747FBEAE70846102224
:104CB8007349FEF7B1F80120FFF728BB0B68714D67
:104CC800591C2A7921601A7023686A79591C216055
:104CD8001A7029882046FEF7CFF82368AA79591C4C
:104CE80021601A7069882046FEF7C6F82368EA79B9
:104CF800591C216001201A70FFF708BB0B68624E2F
:104D080001255A1C0A601D700B68B2785919216078
:104D18001A7027F045FE23685C4A5D495F192760D1
:104D28001870B1F90010B2F90000FEF72FFA2368E5
:104D38005A192260187031882046FEF79DF82846D7
:104D4800FFF7E4BA534D544E9FED548ADFF86C8157
:104D5800DFED538A05F120070EE0FCEEE77ACDED92
:104D6800017ABDF8041020460435FEF785F8AF42F5
:104D780006F118063FF4C9AA717C0029F3D0494B03
:104D8800D5ED007A1B78012BE7D1474B1B68DB0474
:104D980040F1FA80F5EE407AF1EE10FA40F0238106
:104DA80040F2DC51DFE70020FFF7B0BA23685A1C55
:104DB8002260197029882046FEF75EF82368EA7891
:104DC800591C21601A7023682A79591C21601A70AD
:104DD8002368AA79591C21601A7023686A79591CBA
:104DE80021601A70FFF79DBBDFF8D4A000254FF0B3
:104DF80008080135C5F1200208FA02F2A5F12003DE
:104E08002AFA05F6164328FA03F31E43252D06F061
:104E180001024FF000030BD01343EAD0E8B226F0AA
:104E2800C9FB0028E5D0294606A8FEF785FAE0E781
:104E38001E4B1B78DA0700F1C48000251C4E2F4654
:104E480002E00135252D3DD029463046FEF784FA8B
:104E58000028F6D0294606A8FEF77EFA002840F07A
:104E68008E800137EDE700BFA02C002074360020AB
:104E7800AC360020684D0020E04A0020BC360020F7
:104E88005032002050300020943C002088720020CE
:104E98008A720020603200208846002000004042CC
:104EA80000E082446C470020744D0020D235002079
:104EB8003C5D0020E0FF020826390020DB9B914181
:104EC80090E33FF4664B674DB3F850102046FDF76A
:104ED800D3FF654B1988204689B2FDF7CDFF634B98
:104EE80019684B0103F02002C1F340031343C1F3D7
:104EF800800243EA4203C1F3C00243EA8203C1F3DA
:104F0800401243EAC20301F0100119432046FDF79D
:104F1800B3FF04A904222046FDF77EFF2368297801
:104F2800534A581C2060197011886429A8BF64214D
:104F38002046FDF7A1FFB9F1960F47D00021204682
:104F4800FDF79AFF2168B7F1190348BFA7F11203CB
:104F5800A3F3C4034A1C226020461A460B7005A915
:104F6800FDF75AFF2368434A581C10212060197026
:104F780020461188FDF768FF0120FFF7C7B93946B9
:104F880004A8FEF7D9F96CE7F4EEC87AF1EE10FA46
:104F980045DA4FF47A71E6E6082738E60B68B17807
:104FA800354A581C2060197023681278591C2160F2
:104FB8001A709DE523685A1C226001201E70FFF7B5
:104FC800A5B9069B43F00103069336E7236803223D
:104FD800591C21601A7023686A78591C21601A705C
:104FE800B0E7042713E6F4EEC87AF1EE10FA3FF5BD
:104FF800D7AEF4EEE87AFDEEE77AF1EE10FA17EEA6
:10500800901A1ED86FF4F973303903FB01F140F29E
:10501800E73391FBF3F101F2DB5189B2A3E6FDEE30
:10502800E77A40F2E73217EE903A303B02FB03F39F
:1050380088FB0312D917C1EB622101F2E93189B269
:1050480091E640F2F313A1F5836103FB01F140F20D
:10505800E73391FBF3F101F2DD5189B283E600BF3A
:105068003C0100203C360020CC3000207036002067
:10507800D0300020143700209C57002008B50121AB
:105088000220FDF7D9F9094B1B7803F00503052B1E
:1050980008D000210120FDF7CFF900210846FDF7CF
:1050A800CBF9FEE70FF07CFCF3E700BF702C002083
:1050B800022828BF022010B4084C094B207000EBCE
:1050C8008002C0EBC20207495DF8044B013003EBD4
:1050D8004203C0B20B6023F079BB00BF3C3600200E
:1050E800783B00204836002008B51BF00BF8FDF788
:1050F80079FCBDE808401AF0EDBF00BF38B5434B56
:105108005A899989914224BF00225A81198ADA89D9
:10511800914224BF0022DA81DA788AB3072A2FD095
:105128003B493C4D91F85700012400210A282C7076
:105138009C70D9713DD00C2865D0DFED377A8ABBD9
:10514800364C9FED370AA278002918BFF0EE407A56
:10515800062A04D8334901EB820191ED0F0A21791F
:1051680059B3013A032A4DD8F7EE007A87EE800A40
:1051780028F008FD2388984228BF1846208038BDAB
:10518800D97921B198780428B8BF042098702048AC
:1051980090F857000A280CD00C28CED1DFED227ADF
:1051A800002ACDD0072ACBD00A282CD1DFED1F7AD0
:1051B800C6E70A20DFED1E7AC1E79B78154A07EE9D
:1051C800103A1178B8EEC77A27EE277A07EE901AC8
:1051D800F8EEE77A67EE877AB4EEE70AF1EE10FAAE
:1051E80010DDC0EE077AFDEEE77A17EE903A102B45
:1051F800A8BF1023012BB8BF0123DBB28B4238BFF5
:105208000B46137038BDDFED0B7A99E7CC4A0020C6
:10521800E04A00209C5700206F12033948470020BD
:105228006F120338B0FF02080AD7A3390F506E3A3D
:105238005304E9386F12833A38B50D4C0D4DAC4222
:1052480006D2616820461434FDF758FBAC42F8D307
:10525800FEF790F8084A094B094C146000220949E6
:105268001A705A7008480860BDE8384015F01ABA34
:10527800B85B030818600308483600203C36002055
:10528800783B0020CC7000204C36002008B5FFF792
:10529800D3FF1AF037FFFDF7A5FBBDE808401AF069
:1052A80019BF00BFF0B50C292BD8DFE801F06F2A31
:1052B8002A2A4C2A2A2A2B2A2A2A0700046AB2F800
:1052C8000CE097881668674D24F480540462036ADA
:1052D8004468C16923F4005343EA0E3321F4E641DC
:1052E800A84243EA073341EA062100F0B58005F5F4
:1052F8000065A84200F0B08092684460C161026411
:105308000362F0BD046A96899588D2F800E0554F8B
:1053180024F480740462036A4468C16923F4007346
:1053280043EA062321F07301B84243EA052341EA20
:105338000E017ED04C4DA8427BD092684460C1617A
:10534800C2630362F0BD046A96899588D2F800E0CA
:10535800444F24F010040462036A4468816923F00E
:10536800200321F0807143EA061321F4E641B84294
:1053780043EA051341EA0E2148D03B4DA84245D0E7
:1053880092684460816182630362F0BD046A938914
:10539800B2F804E01768334E24F001040462056A89
:1053A8004468816943EA0E0321F4803125F002053F
:1053B8009BB221F07301B04243EA050341EA0701B9
:1053C80014D0294DA84211D005F54065A8420DD04A
:1053D80005F58065A84209D005F58065A84205D085
:1053E80092684460816142630362F0BDD689158A80
:1053F800578A23F0080333433D43D68824F4407486
:1054080023F00403ADB233432C43E9E7D589178A67
:10541800D68823F0800343EA051324F44064558AB0
:1054280023F0400344EA870443EA061344EA850468
:10543800A6E7D589178AD68823F4006343EA0523AB
:1054480024F44054558A23F4806344EA071443EA59
:10545800062344EA051470E7158A24F4804444EAD4
:10546800851449E7002C0140003401402DE9F84F2C
:105478004FF48C7200218248824C834D834E844FB6
:10548800DFF82882DFF828922AF087FC81488249D1
:10549800DFF820E2DFF820C200221359834200F02F
:1054A800C380B3F1804F00F0D580AB4200F0D980C3
:1054B800B34200F0D880BB4200F0D780734500F0BB
:1054C800D680634500F0A680434500F0D2804B4566
:1054D80000F0D280DFF8E4A1534508BF4FF48023E1
:1054E80000F09A801432B2F5AA7FD6D1654D6B4F81
:1054F8006B4E05F5AA784FF0030A4FF0020903E056
:105508001435454500F08E80AB79002BF8D02B7907
:105518001C09013C052C03F00F03F1D837F81400DF
:1055280040FA03F2D207EBD54FF0010B0BFA03F365
:10553800013B184027F0A4FF5A4B1B5D184416EB9B
:10554800C004DDD056F830305748297A03F1384284
:10555800920A825C02F01F005209022A0BFA00FB31
:1055680071D0032A68D0012A05D14B4A4A485269AA
:105578004BEA02024261B4F804E0BEFA8EF2C2F1CC
:105588001F0292B2D00803EB800002F00702046AFF
:1055980092004FF00F0C0CFA02FC24EA0C0404628F
:1055A800046A01FA02F22243002402624FF0010C5D
:1055B800224603E0102A04F10204A1D00CFA02F0FA
:1055C80030EA0E0102F10102F4D1D3F808B00AFA68
:1055D80004F1C9430BEA010BC3F808B0D3F808B0CB
:1055E800C3F808B0B3F804B01FFA8BFB2BEA00002D
:1055F8009880988880B29880186808401860D3F816
:1056080000B009FA04F040EA0B001860D8680140BD
:10561800D960CFE74FF40053D1F818A043EA0A0342
:105628008B615FE7BDE8F88FD1F818A04FF40063ED
:1056380043EA0A038B6155E7174A1748D2694BEAD0
:105648000202C26197E7144A134892694BEA0202C0
:10565800826190E70123D1F81CA043EA0A03CB61D9
:1056680040E70223F7E70423F5E71023F3E72023B5
:10567800F1E74FF48033CFE74FF40033CCE700BFB6
:10568800846F002010230308000400400008004035
:1056980000100040002C014000100240E01B0308ED
:1056A80050450020EC1B0308082303080040014074
:1056B800004401400014004000340140004801400B
:1056C80001490248FEF7C8BC747000200048014038
:1056D80001490248FEF7C0BC247000200040014088
:1056E80001490248FEF7B8BCFC6F002000080040E2
:1056F80001490248FEF7B0BCD46F00200004004006
:1057080002494FF08040FEF7A7BC00BFAC6F0020F5
:1057180010B5064C06482146FEF79EFC04F1C80168
:105728000448BDE81040FEF797BC00BF846F002016
:10573800002C01400044014001490248FEF78CBC9E
:10574800846F0020002C01402DE9F0410468514D80
:10575800A30AAB4200F084800AD94F4DAB4277D000
:105768000135AB425FD0023DAB426DD0BDE8F08160
:105778004A3DAB4270D00135AB4258D0B3F5801FDB
:10578800F4D14FF0480E012647794FEA970C0029CB
:105798006AD0B000634685190227D4F80C809F4070
:1057A8000CEB4503BFB23D4D03F1040C47EA080773
:1057B80045F8231045F82C20E760EFF311815022BB
:1057C80082F31288821905EBC2021369002B32D0CA
:1057D80013620433821905EBC202576917B11F60BF
:1057E80053690433821905EBC202976917B11F6028
:1057F80093690433821905EBC202D76917B11F6098
:10580800D36904330027CAB21F6082F31188304479
:1058180005EBC000036A8BB9E3684FF6FE721340CC
:10582800E360BDE8F0814FF4887E0626ACE74FF0D0
:10583800980E0326A8E705EB0E03CBE7E36843F0D1
:105848000103E360BDE8F0814FF0C00E04269BE73A
:105858004FF0E80E052697E74FF0700E022693E703
:105868004FF0200E00268FE7BF08022306FA03F048
:10587800BB40DB43E768094D9BB23B4087190CEB03
:10588800470CE3600CF1040345F82C1045F823207D
:1058980093E700BF4B00100051001000846F0020F8
:1058A80030B503685C4D18885C4CB4FBF2F20139E2
:1058B800013AAB4294B283B089B282B266D05848FA
:1058C800834263D0B3F1804F60D0A0F59830834213
:1058D8005CD000F58060834258D0524883425BD048
:1058E80000F5806083427DD022F4407200F58C3050
:1058F80092B283421A80D9621C850ED0484A9342DC
:105908000BD002F54062934207D002F580629342C1
:1059180003D002F58062934201D100221A86012247
:105928005A611A883C4992B242F001028B421A80AD
:1059380062D0B3F1804F61D03B4A934260D002F508
:10594800806293425ED002F5006293425CD002F519
:10595800806293425AD002F59032934258D002F5B1
:105968004062934256D002F5806293421ED002F5FF
:105978008062934208BF092219D002A84FF0012380
:1059880040F8043D24F00CFC03B030BD254822F05B
:105998007002834292B2A3D101201A80D9621C8579
:1059A80058611A8892B202431A80C5E708221F4B31
:1059B80003EBC20301A893F85D408DF8044001236E
:1059C80000228DF805308DF807308DF8062024F078
:1059D800E7FB1B2CD8D1164B019301A824F0E0FB60
:1059E80003B030BD01201A80D9621C8558611A881D
:1059F80092B202431A809CE70022D8E70122D6E738
:105A08000222D4E70322D2E70422D0E70522CEE718
:105A18000622CCE70722CAE7002C014000A24A046C
:105A2800003401400010004000040040B0FF0208AC
:105A380019010001204B98422DD0B0F1804F2CD095
:105A4800A3F5943398422AD003F58063984228D06E
:105A580003F50063984226D003F58063984224D06A
:105A680003F59033984222D003F54063984220D042
:105A780003F58063984207D003F58063984208BF16
:105A8800092202D00020704708220C4B03EBC20306
:105A980093F85C0070470022F7E70122F5E702223D
:105AA800F3E70322F1E70422EFE70522EDE70622F8
:105AB800EBE70722E9E700BF002C0140B0FF02082E
:105AC8002DE9F04F013085B0C3B203938E4D8F4F4F
:105AD8008F4C904E0A230293DFF840921AF02AFB6B
:105AE8004FF4FA7A4FF0100C4FF47A70D9F804306A
:105AF800C3F30803002B40F0C880EFF31183002B99
:105B080040F0C3802968A26800BF2B689942F9D188
:105B1800D7F800E000FB0EF39B1AB3FBFEF300FB83
:105B280001314FF0010E0191D9F80430C3F3080395
:105B3800002B40F08E80EFF31183002B40F089801A
:105B48002B68A16800BF2A689342F9D1D7F800B042
:105B580000FB0BF2521AB2FBFBF200FB0323019A83
:105B68009B1AB3F57A7FDFD3BAF1010ABED1039B42
:105B7800002B40F0C4804FF47A7ADFF8A0915046A9
:105B88004FF0100CD9F80430C3F30803002B40F091
:105B98009980EFF31183002B40F094802968A26864
:105BA80000BF2B689942F9D1D7F800E000FB0EF34B
:105BB8009B1AB3FBFEF300FB01314FF0010E01917C
:105BC800D9F80430C3F308033BBBEFF3118323BBBD
:105BD8002B68A16800BF2A689342F9D1D7F800B0B2
:105BE80000FB0BF2521AB2FBFBF200FB0323019AF3
:105BF8009B1AB3F57A7FE3D3BAF1010AC2D1029BAB
:105C0800013B02937FF468AF4349444B4448454AFB
:105C18000860DA6005B0BDE8F08FEFF311888CF307
:105C28001288A1682368DB0344BFC6F800E0A168B6
:105C38002B6832685FFA88F888F31188D7F80080F3
:105C48001A4400FB08F35B1AB3FBF8F300FB0233BA
:105C5800CDE7EFF311888CF31288A1682368DB0382
:105C680044BFC6F800E0A1682B6832685FFA88F87C
:105C780088F31188D7F800801A4400FB08F35B1AF0
:105C8800B3FBF8F300FB023369E7EFF311828CF3FF
:105C98001288D4F808E02368D90303D501233360B8
:105CA800D4F808E02B683168D2B282F311883A68D8
:105CB800194400FB02F3A3EB0E03B3FBF2F300FB62
:105CC80001312EE7EFF311828CF31288D4F808E043
:105CD8002368D90303D501233360D4F808E02B687F
:105CE8003168D2B282F311883A68194400FB02F392
:105CF800A3EB0E03B3FBF2F300FB01315DE718469B
:105D080023F01AFA37E700BF886200208C6200206F
:105D180010E000E084620020FC9F002000ED00E01D
:105D2800EFBEADDE0400FA052DE9F047AD4FAE4EEB
:105D38001AF0E8F9BE421ED2DFF83483DFF8349354
:105D48004446258862197DB14A450DD2052D0BD9E7
:105D580033886188C3F30B03994200F0F28014463C
:105D680025886219002DEFD1716830461436FCF78A
:105D7800C5FDBE42E4D39D4A1378A3F11701022959
:105D88000FD99B4911F83300002840F0FC80D80057
:105D98000144497829B1974911F83330002B00F0B4
:105DA8001A81954C6378022B84BF00236370237893
:105DB800022B84BF00232370904B9A78042A00F0AA
:105DC800018132B91A88B2F5F07F84BF4FF4F072BE
:105DD8001A808B4D8B4A2B681A40002A00F0FE80EF
:105DE800D80700F1EA80590400F1E2801A0700F1AF
:105DF800DA809B0400F1D080834D2B685A8C998CF3
:105E0800914224BF00225A84FFF778F91CF0AEF8BB
:105E180010B97E4821F084FF8020FCF7A5FD4FF4DF
:105E28008020FCF7A1FD4FF40010FCF79DFD4FF01A
:105E38000070FCF799FD4FF08060FCF795FD6378E2
:105E4800022B06D8724A734903EB430302EB830320
:105E58000B602378022B07D803EB83016E4AC3EB50
:105E6800C10302EB43032B6025F01CFC0021302208
:105E78006A4829F092FF28681FF01CFE684B2E68BC
:105E880003F1500102E0043399427AD01A78002ACB
:105E9800F9D19C78D8788442F5D26249624B91F85E
:105EA80004E06248624D5C6B624B2860C82764213D
:105EB80011FB0E71DFF8C0E159605F4F30F8061C26
:105EC8005E4DAEF8001000219960D96019615961E2
:105ED8009961D96183F8201083F821103A702E60F7
:105EE8000CB119F06BFF564B9FED565A1B88564A5A
:105EF8009FED566A5579564C56495748086006EE44
:105F0800903AF8EEE66A1388C5EE265A07EE103A7C
:105F180053881279C4ED005A07EE903AB8EEC77A62
:105F28004E4BF8EEE77A1D725A7227EE067A67EE44
:105F3800867ABDE8F04783ED017AC3ED007A1AF05E
:105F4800C9B863799B077FF40AAF716894F804A015
:105F58003046FCF7D3FC3388BAEB133F04D0143631
:105F6800BE42FFF4EDAE06E773887068AA1FC3F35C
:105F78000B039A4204F10601A8BF1A4627F08EFCCB
:105F8800EDE7012289E7D8000C186468002C7FF43B
:105F9800FFAE17241470FBE63148FCF7E5FC4020FF
:105FA800FCF7E2FC28E72F48FCF7DEFC2B6820E72B
:105FB8002D48FCF7D9FC2B6818E72C48FCF7D4FCD3
:105FC8002B6810E79A8AB2F57A7FBFF402AF4FF4D4
:105FD8007A729A82FDE618231370E2E643F008030A
:105FE8002B60FDE618600308B85B03083434002012
:105FF80064240308581C03083C3600204847002046
:10600800B43C0020096000024836002054440020B7
:106018004C360020CC700020783B0020F423002070
:106028003834002050300020743600202E440020E0
:10603800145D0020F0360020481C00202824002091
:10604800482D0020C0C9FB48941E002017B7D1383E
:106058004C2D0020242E00203661023D002E002009
:1060680009400002016000020920000208600002E5
:1060780002F0030800000408B843002008B51AF02D
:1060880041F8FCF7AFFC1AF025F8FFF74DFE0120A8
:10609800BDE8084022F09ABB2DE9F04F013085B0E9
:1060A800C3B203930B4602918B4C8C4E002B00F02D
:1060B80099808B4D8B4FDFF830921AF03BF84FF4F4
:1060C800FA7A4FF0100C4FF47A70D9F80430C3F311
:1060D8000803002B40F0DE80EFF31183002B40F023
:1060E800D9802968A26800BF2B689942F9D1D7F8EE
:1060F80000E000FB0EF39B1AB3FBFEF300FB01313B
:106108004FF0010E0191D9F80430C3F30803002BB6
:1061180040F08780EFF31183002B40F082802B68DA
:10612800A16800BF2A689342F9D1D7F800B000FBF4
:106138000BF2521AB2FBFBF200FB0323019A9B1AE3
:10614800B3F57A7FDFD3BAF1010ABED1039B002BE6
:1061580040F0BD804FF47A7ADFF88C9150464FF0CA
:10616800100CD9F80430C3F30803002B75D1EFF3F2
:106178001183002B71D12968A26800BF2B6899424E
:10618800F9D1D7F800E000FB0EF39B1AB3FBFEF33E
:1061980000FB01314FF0010E0191D9F80430C3F32F
:1061A800080313BBEFF31183FBB92B68A16800BF89
:1061B8002A689342F9D1D7F800B000FB0BF2521AC3
:1061C800B2FBFBF200FB0323019A9B1AB3F57A7F1B
:1061D800E3D3BAF1010AC4D1029B013B0293002B1D
:1061E8007FF467AF05B0BDE8F08FEFF311888CF34B
:1061F8001288A1682368DB0344BFC6F800E0A168E1
:106208002B6832685FFA88F888F31188D7F800801D
:106218001A4400FB08F35B1AB3FBF8F300FB0233E4
:10622800D2E7EFF311888CF31288A1682368DB03A7
:1062380044BFC6F800E0A1682B6832685FFA88F8A6
:1062480088F31188D7F800801A4400FB08F35B1A1A
:10625800B3FBF8F300FB023370E7EFF311828CF322
:106268001288D4F808E02368D90303D501233360E2
:10627800D4F808E02B683168D2B282F311883A6802
:10628800194400FB02F3A3EB0E03B3FBF2F300FB8C
:1062980001317FE7EFF311828CF31288D4F808E01C
:1062A8002368D90303D501233360D4F808E02B68A9
:1062B8003168D2B282F311883A68194400FB02F3BC
:1062C800A3EB0E03B3FBF2F300FB013118E718460A
:1062D80022F032FF3EE700BF10E000E084620020B9
:1062E800886200208C62002000ED00E02DE9F04F6C
:1062F800DFF830C1474A4849484E494D8046102783
:1063080018F1FF38C0F08480DCF80430C3F30803C8
:10631800002B5CD1EFF31183002B58D10B689468E4
:1063280000BF08688342F9D1D6F800904FF47A701C
:1063380000FB09FEAEEB040EBEFBF9FE00FB03EE0C
:10634800DCF80430C3F308034FF47A740120FBB976
:10635800EFF31183E3B90B68D2F808A000BFD1F8B6
:1063680000904B45F7D1D6F800B004FB0BF9A9EB28
:106378000A09B9FBFBF904FB0393A3EB0E03B3F57E
:106388007A7FBDD2DCF80430C3F30803002BDFD0DA
:10639800EFF3118A87F31288D2F808B01368DB0389
:1063A80044BF2860D2F808B00B68D5F800905FFAAF
:1063B8008AFA8AF31188D6F800A0994404FB0AF3F4
:1063C800A3EB0B03B3FBFAF304FB0933D5E7EFF3B5
:1063D800118487F31288D2F808901368D80303D57C
:1063E80001232B60D2F808900B682868E4B284F384
:1063F8001188D6F800A04FF47A7400EB030E04FB62
:106408000AF3A3EB0903B3FBFAF304FB0E3E97E789
:10641800BDE8F08F10E000E0886200208C62002068
:106428008462002000ED00E02DE9F04F2DED028B95
:1064380093B0834615F060FCB84B1D7825B113B0B6
:10644800BDEC028BBDE8F08FB54B1B685B05F6D53C
:10645800B44FB54E3B68002B5BD0B44C3168D4F8D0
:1064680010218A1A7C2A54D994F81421DFF8088359
:106478009FEDAF8AC4F81011013284F814214FF04F
:10648800240A5E20984750463B689847A94BF8EC89
:10649800016A9B8A07EE103AF8EEE66AB8EEC77A08
:1064A8000AF1010AC6EE877A5FFA8AFA67EE887AF5
:1064B800FDEEE77ACDED027ABDF908905FFA89F032
:1064C8001DF07AF9C9F307201DF076F9BAF1270F04
:1064D8003B68D6D15E2098473B6830209847D4F86F
:1064E80018815FFA88F01DF067F9C8F307201DF0DE
:1064F80063F93B685E20984794F8143113F0030859
:1065080000F0868113F0070801F07082282B01F053
:106518004383894B1B78002B72D0844C874AD4F86C
:106528002031ABEB0303934200F2868794F828915D
:10653800B9F1000F35D1DFF84482D8F80000FAF736
:1065480047FFC0B201280FD902287D4F41F0BD8313
:106558003B78002B41F00986D4F82C31ABEB0303D0
:10656800B3F57A6F81F0B087D4F83031002B47D07B
:1065780094F82831C3B9734B1B689B7801211E3BE3
:1065880000228B4284F8281184F83C2141F25F876D
:10659800D8F80000022104301DF084F894F8343152
:1065A80011E0D4F830315BB3D4F8383140F6B73263
:1065B800ABEB0303934223D994F83431002B01F059
:1065C800D482DFF8B881013BDBB284F83431002B88
:1065D80000F0A487D4F8307194F83C2117F8011B17
:1065E80094F83D31D8F80000C4F830710A440133FA
:1065F80084F83C2184F83D31FAF7EEFEC4F838B14E
:10660800514BD6F800801B7843B1504F386828B1F9
:106618004F4B1B78013B012B40F290874D4B1B7869
:1066280063B14D4F3B684BB1404CD6F80090D4F85D
:106638005431A9EB0303632B00F21D81DFF840817D
:1066480098F80030022B01F06F823D4F97F87430B4
:10665800032B00F04D87414B1B7873B1404D2B68DD
:106668005BB1324CFAF7FEFCD4F86031029044F684
:106678001F62C31A934200F259813A4B1B78002BD0
:1066880040F08080384B1B7843B1284CD4F8B032A6
:1066980003F5C333A0339B4580F07C86334B1B78CE
:1066A800002B3FF4CCAE214E314C324D06F2D127AF
:1066B8002068FAF78DFE00283FF4C1AE2068FAF78B
:1066C8007FFE2B7880465A1E33B120682A70FAF76D
:1066D8007FFE0028F2D1B2E603223946781E29F05F
:1066E80042FB96F8D03296F8D12286F8D38283F40A
:1066F8007F4383F0FF039B1A1FFA88F89BB2B8EB1D
:10670800132FD5D196F8D222DBB29A42D0D1781E77
:106718001CF034FD2B7818442870C9E73736002060
:10672800744D0020B852002088620020A41E00206A
:1067380000007A4474360020C63900203F0D03005B
:106748001C000020B4520020C8390020B850002096
:10675800D0390020D8390020246B0020E0390020EF
:10676800E4390020243A0020353A0020EA39002094
:10677800F0390020F4390020AC360020B052002057
:10678800C25300205B4C2278A2B15B4B9B7A53B179
:10679800FAF768FC594B1B68C31AA3F57A73B3F56B
:1067A800FA6F07D82278564B56491868FAF7E0FD71
:1067B80000232370544CD4F8A83203F5C333A03314
:1067C8009B45FFF45FAF514DC4F8A8B22B78002B5E
:1067D80041F045834E4D2B78002B41F02D824D49D9
:1067E80094F8AC228D5CE90701F10285AA0701F152
:1067F800C2846B0701F1AE83474A94F8AC32117832
:10680800013393FBF1F201FB123384F8AC3239E720
:10681800D4F8102141F288339A4201F222823B686F
:106828005E2098473B68142098473C4B3C4AB3F994
:10683800043082FB03124FEAE378C8EBA2080FFA90
:1068480088F85FFA88F01CF0B7FFC8F307201CF03F
:10685800B3FF3B685E2098473B681C2098470020A0
:106868001CF0AAFF00201CF0A7FF3B685E20984799
:1068780094F8143146E6DFF8A4A0DFF8A48041209C
:106888001CF0C0FEBAF9023088FB0320DB17C3EB0B
:10689800A00080B21CF09CFEBAF9003088FB0320EF
:1068A800DB17C3EBA00080B21CF092FEBAF90430EB
:1068B80088FB0320DB17C3EBA00080B21CF088FE26
:1068C800184B38681978FAF787FD94F8583113F09F
:1068D800010801F01B82144AC4F854910133DBB259
:1068E800A2FB0312D20802EB8202A3EB420384F854
:1068F8005831A3E6B8390020304F0020344000203A
:10690800283A002078390020A41E00202C3A0020C4
:106918002D3A0020303A0020343A0020CC360020AE
:10692800676666667C6F0020CDCCCCCC94F8663167
:10693800002B41F07C81DB4B1A6802F00803002B26
:1069480048F603414AF60B404BF60F4349F6074712
:1069580004BF03460F4612F0040F4FF0190118BF89
:106968001F46920684F8661103D547F4804747F01E
:106978002007CD4B5A79C7F30909002A41F0D18580
:106988009B79002B41F0D386984664204FF0FF3A5C
:106998004FF0000C0A970B97ADF834C0CDF83AC009
:1069A800CDF83EC0CDF842C0CDF83090ADF8368075
:1069B800ADF838A08DF846000AAF0FCFDFF800E336
:1069C80084F805C0AEE80F0097E80F00AEE80700AE
:1069D8002EF8023B71464FF0010C1B0CFE271F20BE
:1069E800C82201F81E39A770A27184F807C0E070A8
:1069F80094F87601207180F0F10383EA0313DAB288
:106A0800130983F0E70343EA022383EAC2031BB2B4
:106A180083EA0312D2B2C3F3072383EA121343EAC9
:106A2800022383EAC2031BB283F0C80282EA02127D
:106A3800D2B2C3F3072383EA121343EA022383EA99
:106A4800C2031BB283EA0C0787EA0717FFB2C3F336
:106A5800072282EA171242EA072200EB0C0382EAB5
:106A6800C7070EEB0C0084F87631278011F8013B3C
:106A78007B4083EA0313DBB21A0982EA172242EA4F
:106A8800032282EAC3031BB29FB281422780EDD161
:106A980083F07C0383EA0313DBB24FEA131E8EEA0A
:106AA800172E8EEA032E8EEAC30E0FFA8EFE1FFAF9
:106AB8008EFADFF810C2A4F800A05FFA8EFE4FEA43
:106AC8001A2A84F828A084F827E00CF5CF7804F176
:106AD8002209DCF80000DCF80410DCF80820DCF8F7
:106AE8000C3047460FC70CF1100CCC45B846F0D116
:106AF800DCF8000038606D4F9CF8043088F80430EA
:106B080007F1270884F8C5E184F8C6A117F8011F22
:106B18002868FAF761FCB845F8D194F86731002B7A
:106B280041F080806249326809780A2084F8670158
:106B3800002901F005825F4F01293888069041F24B
:106B48000B860229B7F802E001F00685B88805909F
:106B5800032901F0FA85F8880490042901F01186C8
:106B68000529388901F008860629B7F80A9001F046
:106B7800FF850729B7F80C8001F0F785FB89039397
:106B880094F876110A920B4683F0300282EA0212D8
:106B9800D2B217094849079387F07A0747EA0227CC
:106BA8000988237187EAC202444FC1EB012187FBA0
:106BB800013A069B4FF0000C63F30F0C059B6EF334
:106BC8001F4C4FF0000E63F30F0E049BCDF82CC042
:106BD80012B28A440027C91763F31F4EC1EB6A2A11
:106BE800039BCDF830E082EA021160F30F07002022
:106BF800C9B268F30F00C2F3072269F31F4782EA9C
:106C0800111263F31F404FF000090D978DF83DA056
:106C18000E908DF83C9042EA01220DF1280C82EA90
:106C2800C107BCE80F003FB287F0C80888EA081817
:106C3800DFF88CE084F805905FFA88F8C7F3072737
:106C4800AEE80F0087EA181747EA08239CE8030014
:106C580083EAC8031BB283F023024EF8040B82EACE
:106C68000212D2B2C3F30723079F83EA12137046B6
:106C780043EA022383EAC20207F1010C20F814193F
:106C88004FF023081621FE27C82384F876C12280F6
:106C980084F807800EF1020EA770E170A371114607
:106CA80012E000BF70360020E036002043200020AC
:106CB80034370020D86E00202439002003082080B3
:106CC800AC1E0020A61E002010F8013B4B4083EAB2
:106CD8000313DBB21A0982EA112242EA032282EA8A
:106CE800C3031BB299B270452180EDD183F0F40340
:106CF80083EA0313DBB24FEA131E8EEA112E8EEAE3
:106D0800032E8EEAC30E0FFA8EFE1FFA8EF8E44F9A
:106D1800A4F800804FEA182C5FFA8EFE84F81EE073
:106D280084F81FC07968BA683868FB6807F5CF78B7
:106D3800A8E80F0038697969BA6904F29F17A8E8CA
:106D4800070004F2BD1884F8BDC184F8BCE117F847
:106D5800011F2868FAF740FBB845F8D194F86EC1CE
:106D6800BCF1000F40F05887CE4B94F87671B3F918
:106D78000010B3F90220B3F904309FEDCB6ADFF8B5
:106D880044E384F805C007EE103A33680A9387F0A5
:106D98006A0383EA031306EE901AD9B20B0983F04B
:106DA800D50343EA012383EAC1031BB283EA031133
:106DB8005242C9B207EE902AC3F3072383EA11139C
:106DC80043EA0123F8EEE77AF8EEE66AB8EEC77A06
:106DD80083EAC1031BB267EE867A66EE866A27EEFF
:106DE800067A002083F0C808CDED0C7ACDED0B6A49
:106DF8008DED0D7A0E900F90109088EA08160DF11F
:106E08002809F6B2C3F30728B9E80F0088EA16186C
:106E180048EA062888EAC6080FFA88F8AEE80F009C
:106E280088F01E0699E8070086EA0616F6B2C8F347
:106E3800072383EA161343EA06238EE8070083EA4A
:106E4800C6061C20C8214FF005084FF01E0CFE2373
:106E58007A1CE070A17184F86E8184F807C0A37071
:106E6800AEF1100127710EF10C00268084F876210E
:106E780011F8013B734083EA0313DBB21A0982EA73
:106E8800162242EA032282EAC3031BB29EB281425F
:106E98002680EDD183F0270383EA0313DBB24FEAA0
:106EA800131E8EEA162E8EEA032E8EEAC30E0FFAF2
:106EB8008EFE1FFA8EFC7A4FA4F800C05FFA8EFE91
:106EC8004FEA1C2C84F825C084F824E007F5CF7815
:106ED80004F1220938687968BA68FB6846460FC623
:106EE80010374F45B046F5D1704E3B88A8F80030B2
:106EF80006F1240784F8C2E184F8C3C116F8011F1B
:106F08002868FAF769FAB742F8D194F86FA1BAF18C
:106F1800000F40F07B86664B1B68052213F0140FA8
:106F280084F86F2140F08587DFED627A94F876C1A6
:106F38005C4B614AB3F90410B2F906205F4E604811
:106F4800CDED0C7A8CF0220383EA0313DFB23B0900
:106F580083F0590343EA072383EAC703B2F5FA6FBC
:106F68001BB2A8BF4FF4FA6283EA0317FFB2B2F567
:106F78007A7FC3F3072383EA1713B8BF4FF47A72F3
:106F88004FF0640E43EA0723A2F57A720EFB02F271
:106F980083EAC70386FB02E680FB01E01FB2D21733
:106FA800C9174FF00008C2EBA612C1EBA00187F089
:106FB800C806ADF83A20ADF83810CDF82880CDF8DD
:106FC8002C80CDF834800DF1280E86EA0616BEE82E
:106FD8000F00F6B2C7F3072787EA161747EA06270E
:106FE80087EAC606374FDEF800E084F804C00FC70A
:106FF80036B286F04A0383EA0313DBB2C6F30721ED
:1070080081EA13113A4641EA03210CF1010C81EAA5
:10701800C303142042F810E9FE264FF04A0E00215F
:1070280084F876C14FF0C80CE0702380043784F8E8
:1070380007E0A670617184F806C0184612F8011BB3
:10704800414081EA0111C9B20B0983EA102343EADE
:10705800012383EAC10109B288B2BA422080EDD186
:1070680081F0140181EA0111C9B24FEA111E8EEABA
:10707800102E8EEA012E8EEAC10E0FFA8EFE1FFA2E
:107088008EF6074F26804FEA16295FFA8EFE84F89F
:107098001D9084F81CE079683868BA68FB6813E0CA
:1070A800A61E0020CC36002088C3E43A43200020E6
:1070B8007036002000000000D86E0020D34D62100A
:1070C80067666666AC1E0020B7F8188007F5CF7CA7
:1070D800ACE80F0038697969ACE8030004F29F1640
:1070E800ACF8008084F8BB91B04684F8BAE104F2A9
:1070F800BB1918F8011F2868FAF76EF9C145F8D1CD
:10710800C44BC54A1B781278013B12F00100DBB270
:1071180014BFC0214021172B03D8C04A134493F849
:1071280030A0BF4B1A8893071ABF002341F0100103
:10713800012312F4027F18BF022312F0100F18BFA8
:10714800062312F0200F18BF1023002841F0AE814B
:107158004FF0030C94F876910A9389F0460383EA7A
:107168000313DAB2130983F0920343EA022383EA92
:10717800C2031BB283EA0310C0B2C3F3072282EA38
:10718800101242EA002282EAC00212B282F0C80E4D
:107198008EEA0E1E5FFA8EFEC2F30722002382EAF1
:1071A8001E1203208DF82CA08DF82FC08DF82D30DD
:1071B80042EA0E2C8DF82E108DF830000AAA07CA64
:1071C8008CEACE0E0FFA8EFEDFF868A2E3718EEA23
:1071D8000E1CAAE803005FFA8CFCCEF3072E8EEA99
:1071E8001C1E4EEA0C2181EACC0C94F808E08AF8BF
:1071F80000200FFA8CFC8EEA0C0E8EEA0E1E5FFA47
:107208008EFECCF3072282EA1E1242EA0E22607A30
:10721800A17A94F80BC0637182EACE0212B2504090
:1072280080EA001E5FFA8EFEC2F3072080EA1E1075
:1072380040EA0E2080EACE0000B2414081EA011106
:10724800C9B2C0F3072282EA111242EA012282EA95
:10725800C10212B28CEA020C8CEA0C1C5FFA8CFC9C
:10726800C2F3072282EA1C1242EA0C2294F80CE0CC
:10727800607BA17B94F8108084F8049082EACC02A9
:1072880012B28EEA020E8EEA0E1E5FFA8EFEC2F36C
:10729800072282EA1E1242EA0E2282EACE0212B2C5
:1072A800504080EA0010C0B2C2F3072282EA1012EE
:1072B80042EA002282EAC00212B2514081EA011178
:1072C800C9B2C2F3072282EA111242EA012282EA13
:1072D800C102E17B13B281EA030282EA0212D2B24E
:1072E800C3F3072383EA121343EA022383EAC203A0
:1072F8001BB288EA030282EA0212D2B2C3F307235E
:1073080083EA121343EA022383EAC2031BB283F01F
:10731800320282EA0212D2B2C3F3072383EA1213BB
:1073280043EA022383EAC2031BB29AB24FF0FE0C6F
:107338004FF0090EC82009F10101DBB284F802C040
:1073480084F803E04FEA122CA07184F876112280A9
:1073580084F812C0637438687968BA68B7F80C9012
:107368000AF5C87EAEE807000AF5D07A8EF80280E2
:10737800AEF8009084F8B0C184F8AF3116F8011F58
:107388002868FAF729F8B245F8D1029BC4F86031A9
:10739800FFF773B994F8B432204AC4F8B0B202EBDC
:1073A8008302926C42B312AD04F2BB231D4E45F822
:1073B800203D002104F2CD2331800B938021152339
:1073C800A52784F8BA32284684F8B91284F8B87226
:1073D800904728463188FBF74FFD0A9D124804F56F
:1073E8002E716D1A152DA8BF15252A4626F056FAB6
:1073F8000E4A94F8B43215700D4A013382FB031219
:10740800A2EBE37202EB42029B1A84F8B432FFF754
:1074180045B900BF34340020D23500205800030895
:107428002639002034390020C83E0020DD3E0020E7
:1074380056555555AC1E0020D14AD24B92F80BE058
:107448003068D4F824211B88CF49801A4FF47A7207
:10745800DFB202FB0EF21B0A8F770F7590424FF0D6
:107468000007CB774B758F700F7180F0EC83C74B9B
:10747800C74F1B68C74ADFF838E310689268C4F83A
:1074880020B187FB038CDB17C3EB6C13D4F818C14E
:1074980087FB0C878EFB00988EFB029ED217C2EBEF
:1074A800AE0203F5FA734FEAEC7E9BB2CEEB671E91
:1074B800C0170CF5EA47C0EBA80030378B761B0ADB
:1074C8000EF1780E3F120CF1300CCB764FEA2028E3
:1074D8001312087781F81D8081F8202081F8213067
:1074E80081F824E081F8237081F822C0FFF71EB8E4
:1074F800DFF8C092D9F80000F9F75EFF00283FF4E2
:10750800AAA8D9F800000121F9F752FF02220023A6
:1075180087F8742088F80030FFF79DB894F83C117C
:1075280094F83D31D8F800004A1C013384F83C2116
:1075380084F83D31F9F750FFFFF760B8964CDFF853
:1075480078924FF0000A0AE01B2B00F003830D2B02
:1075580000F016824FF0010389F801303868F9F716
:1075680037FF002838D03868F9F72AFF83B27E2B16
:1075780032682AD099F801100029EFD194F83E21F9
:10758800002AE1D07D2B00F0108294F84CE1BEF186
:10759800000F04D080F02003DBB284F84C11511C9A
:1075A800C9B22244092984F83E1182F8403100F01A
:1075B800F0810829D2D8B4F84A21134403EB1323E5
:1075C80003F0FF03A4F84A31C8E784F83EA184F821
:1075D8003FA189F801A0C1E794F84D3133B194F87F
:1075E800413184F84D01302B00F0588794F83F2141
:1075F8006A4BDFF8C8C1DFF8C8E1DFF8C8A1012786
:10760800104600283FF40AA83268A2EB0802012AB3
:1076180000F2B18194F84E91B9F1000F40F0B182B7
:1076280094F84F1133F8112012B984F84F71E8E734
:107638000131B2F5826F84F84F1100F01F811FD914
:10764800B2F5E26F00F0C08035D9B2F5046F00F0F2
:10765800CA80B2F5116F00F0D380B2F5E46FD0D1D3
:1076680010464F4A176C918A642303FB07F393FB78
:10767800F1F11BF0FDFF002384F83F31FEF7CEBF88
:10768800B2F5007F00F0D6802DD8B2F5807F00F0EB
:107698004881B2F5887FB4D1DCF800205207B0D514
:1076A800D4F818114FF488701BF0E2FF002384F817
:1076B8003F31FEF7B3BFB2F5C06F00F0CF80B2F52F
:1076C800E06F9ED1364A906B918A642303FB00F3E6
:1076D8004FF4E06093FBF1F11BF0CAFF002384F83C
:1076E8003F31FEF79BBFB2F5047F00F02A81B2F567
:1076F800806F86D194F850310133DBB2032B00F24E
:107708005B8142F2107184F8503101FB03F1254B83
:107718001B88002B40F04E810131234B1B78DF077B
:10772800224B1B8848BF0431D80748BF0A319A0743
:1077380048BF14311F0648BF2831D80548BF283133
:107748005A0748BF64311F0748BFC831980548BF6A
:1077580001F5C8719A0648BF01F57A71DF0648BF7E
:1077680001F5FA61580648BF01F57A614FF4806067
:107778001BF07EFF002384F83F31FEF74FBF00BFA8
:10778800E4500020CC500020F83900203C2D002087
:107798001F85EB51C0500020A41E0020580003088C
:1077A8007436002014370020D235002026390020F6
:1077B80067666666485400201C000020703600206A
:1077C800E0360020F250002010467E4AD76B918A9E
:1077D800642303FB07F393FBF1F11BF049FF84F8E3
:1077E8003F91FEF71BBF784BB3F9041001EB810101
:1077F800104649001BF03CFF84F83F91FEF70EBF8E
:107808009EF80520002A3FF4FCAE9AF800100029E3
:107818003FF4F7AE6D4B1B8803EB83035B004FF41B
:10782800116093FBF1F11BF023FF002384F83F3133
:10783800FEF7F4BE9EF8061000293FF4E2AE644B52
:1078480064491B68104681FB0321DB17C3EBA101C8
:107858001BF00EFF84F83F91FEF7E0BE9EF806206D
:10786800002A3FF4CEAE5A4B4FF4C06099681BF023
:10787800FFFE002384F83F31FEF7D0BEDCF800207D
:1078880012F020097FF4BDAE534A1168090600F1D1
:10789800EF85524A127B002A3FF4B3AE94F8511197
:1078A800032900F26886DFE801F0322819024C4B00
:1078B8001B6859799A79DB7901F1407101EB022152
:1078C80001EB0341002384F851314FF482601BF02F
:1078D800CFFE002384F83F31FEF7A0BE414B1A6863
:1078E800137A507992781B0403EB002313444A1C43
:1078F80084F8512103EB0161E7E73A4B1A68D37921
:10790800107952781B0403EB00231344EFE7354B3F
:107918001A689379D07812781B0403EB0023134478
:10792800E5E7DCF8002051077FF56BAE2E4B4FF4EE
:10793800807019681BF09CFE002384F83F31FEF725
:107948006DBE9EF80520002A3FF45BAE9AF8001041
:1079580000293FF456AE214B5B7B002B00F0B0852D
:107968001A4B1B8893FBF1F101EB810149004FF49D
:1079780004701BF07DFE002384F83F31FEF74EBEF5
:107988004FF0010184F83E1184F84031A4F84A21EF
:10799800E4E5B4F84A21C2F1FF0293427FF4DAAD7C
:1079A8004FF0010384F84D31D4E54FF0010384F81A
:1079B8004C31D3E50231B0E6012384F8503142F26C
:1079C8001071A4E674360020CC360020CC5000207C
:1079D800C050002067666666744D0020E4500020A1
:1079E800CC700020483600203C2D00203B685E20EB
:1079F80098473B6802209847FF201BF045FB037817
:107A0800FF2B00F0328590F901304FEAE3785FFAF6
:107A180088F8D8B21BF0D0FE40461BF0CDFE3B687C
:107A28005E2098473B6803209847FF201BF02CFBFB
:107A38000378FF2B00F01485B0F90830D8B2C3F3EF
:107A48000729DFF8B8821BF0B7FE48461BF0B4FEE2
:107A580098F80530002B40F0D7820AA99E481BF001
:107A68006FFE3B685E2098473B6813209847BDF936
:107A780028805FFA88F01BF09FFEC8F307201BF0F0
:107A88009BFE3B685E2098473B681B209847BDF9E2
:107A98002A805FFA88F01BF08FFEC8F307201BF0DE
:107AA8008BFE3B685E2098473B68232098474E2012
:107AB8001BF082FE00201BF07FFE0AA986481BF0FF
:107AC8003FFE3B685E2098473B6812209847BDF907
:107AD80028805FFA88F01BF06FFEC8F307201BF0C0
:107AE8006BFE3B685E2098473B681A209847BDF9B3
:107AF8002A805FFA88F01BF05FFEC8F307201BF0AE
:107B08005BFE3B685E2098473B68222098474520EB
:107B18001BF052FE00201BF04FFE3B685E2098478A
:107B280094F81431FEF7F2BCF9F79CFA6B4B1B681A
:107B3800C01A40F6B833984200F28681DFF8C0A137
:107B48009AF804303A2B00F0B183002388F800300B
:107B5800FEF781BD3868F9F73BFC00287FF4FAACE2
:107B68004FF0010384F83F31F8E4C4F8303184F869
:107B78002831DFF890811BF0C9FD94F83431FEF705
:107B880022BD574906201BF07FFB002384F84E01D5
:107B980084F83F31FEF742BD4FF000083B68D6F845
:107BA800009084F814815E2098473B684D4C17205C
:107BB800984740461BF000FE4B4BA3FB09239B0B49
:107BC800A4FB03125209C2EB0212A3EB8203D8B240
:107BD8001BF0F2FD3B685E2098473B6818209847E9
:107BE800424BA3FB09239B09A4FB03125209C2EBD6
:107BF8000212A3EB8203D8B21BF0DEFD40461BF055
:107C0800DBFD3B685E209847FEF783BC0AF1FF3A2C
:107C180084F86FA1FFF7B9BB0CF1FF3C84F86EC183
:107C2800FFF773B9013B84F86731FFF797B8013B59
:107C380084F86631FEF771BF2D493A201BF024FB0A
:107C48002870FEF71FBD2B4B32681B78C4F824211F
:107C5800013B012B3FF60BAC102202238A700B71FB
:107C680005E43B68DFF8A0905E2098473B68102049
:107C78009847214AD9F8003082FB032ADB17C3EB67
:107C88006A1A5FFA8AF01BF097FDCAF307201BF007
:107C980093FD3B685E2098473B6821209847D9F8B8
:107CA8000030154AD81782FB0329C0EB69106422FB
:107CB80002FB10300028B8BF4042C0B21BF07CFD68
:107CC80040461BF079FDFEF7AABD1BF00FFD01230E
:107CD8003B70FEF749BC00BF80969800C85300204F
:107CE800733602088988888873B2E745D34D6210D5
:107CF80081BC01082A3900201F85EB51E03600209D
:107D0800B0530020B05200203C2D0020AA4B1B8805
:107D1800DA0515D4D80600F11B84990600F12784EA
:107D28005A0600F13384180700F13D84D90700F1A1
:107D3800FA8413F0020F0CBF4FF004084FF00C0840
:107D48009E4B9F4A1B78D27803F001030AB143F097
:107D58000203532002931BF055FC9A4A128802EB47
:107D6800820202EB8202900080B21BF031FC0020FC
:107D78001BF02EFC944A954912883868C2EBC2124F
:107D8800520081FB023111444FEAE27ACAEB612AC0
:107D98005FFA8AFA5146F9F71FFB8D4B38681A7853
:107DA800029B48EA03088A4B8AEA020A002183F800
:107DB80000A0F9F711FB41463868F9F70DFB844B31
:107DC800834A1B78386888EA0303DBB219461370C4
:107DD800F9F702FB94F85831002B7EF47CAD4F2064
:107DE8001BF010FC21F0F0FE21F0EEFE21F0ECFE7D
:107DF80001213868F9F7F0FA764A754B92F8008055
:107E08001B78734A386808F0010883F0010341467B
:107E18001370F9F7E1FA6E4B6D4A1B78386888EAF7
:107E2800030319461370F9F7D7FA94F85831FEF797
:107E380052BD694B9FED697AD3ED007AF8EEE77A87
:107E480067EE877AFFF772B8654AB2F85A310021AF
:107E58000133A2F85A3188F80010FEF7FCBB614ED6
:107E6800614B00930024A6F13F01604B604A0891E2
:107E780006F8404C5F4909960AA8FBF7D5F8089E12
:107E8800731C08933470089B2922591C08911A7096
:107E9800089BEA22591C08911A70089BC822591C91
:107EA80008910AA81A7024F0F1FD471C0AA93A465D
:107EB800089825F0F3FC089AD31901330893D45590
:107EC800089B5A1C08921C70089B5A1C08921C702C
:107ED800089B5A1C08921C70089B5A1C08921C701C
:107EE800089B5A1C08921C70089B5A1C08921C700C
:107EF800089B5A1C08921C70089B5A1C08921C70FC
:107F0800089B5A1C08921C70089B5A1C08921C70EB
:107F1800089B5A1C08921C70089BFF22591C089148
:107F28001A70089B0122991812A808911A7050F823
:107F3800283D9B1B337013F06FFE2C70FEF7A2BB1D
:107F4800884689460846049105918E460691039114
:107F5800FEF716BE284A234B12680B93A3F140057F
:107F680000202121D70003F8400CA97040F1CD82F0
:107F780022490326104B1B88580500F1C382DA07F3
:107F880000F1F28203F002031D4A002B1CBF0326F6
:107F980011461C4F3246384625F080FCF31912A8CA
:107FA8000133B91E40F8203D00225B1AF2556B7070
:107FB80013F032FEFEF720BC26390020D23500200F
:107FC800F0360020CC5000202439002003082080FF
:107FD8007C6F0020FC3100203C2D00200AD7233C78
:107FE800A41E0020783900204136002028280308E4
:107FF800302803083C280308F4310020142803081B
:10800800242803083B3900209E4B93F800A0BAF1BE
:10801800000F3FF422AD9C4AB4F81CE111883B687C
:1080280002924FEA0E1E64201FFA8EFE00FB01A189
:108038004FEA4A00B1FBF0F14EEA012E1FFA8EFE1C
:10804800C1F303215E204EEA010998473B680620E8
:1080580098475FFA89F01BF0AFFB4FEA19201BF035
:10806800ABFBB4F81C31029A8849B2F800904A7AFE
:1080780001339BB2012A93FBFAF00AFB1033A4F8F0
:108088001C3100F041836E2381484A7B03FB09F3CE
:1080980080FB03014FEAE379C9EBA1092AB1794BC7
:1080A8001FFA89F91B7899FBF3F93B68DFF8F8A107
:1080B8005E2098471FFA89F93B683A209847AAFB3F
:1080C800093A4FEA5A1A1FFA8AF3D8B202931BF0F8
:1080D80073FB029B180A1BF06FFB3B685E209847F6
:1080E8003B683B209847642303FB1A939BB269487B
:1080F800053380FB0320DB17C3EBA000C0B21BF0E5
:108108005BFB00201BF058FB3B68DFF890A1DFF811
:1081180084915E2098473B6828209847DAF8003019
:1081280089FB0329DB17C3EBA9095FFA89F01BF068
:1081380043FBC9F307201BF03FFB3B685E209847D1
:108148003B6804209847B8F80830002B40F022829A
:10815800DAF8083083F310085FFA88F01BF02CFB7C
:10816800C8F307201BF028FB77E4C4F82CB187F884
:108178000090FEF7F9B9484A434B0B9212AEA2F1B0
:108188003D0046F8200D1988444FA2F14003002015
:108198004FF00A0E02F8400C082283F801E030463E
:1081A8009A70FAF743FE3B683A49DA1781FB0313E2
:1081B800C2EBA30399B23046FAF738FE08F0EAFAA0
:1081C800BF680A9B3A0C591C0A911A700A9B3A0A12
:1081D800591C0A911A700A9B5A1C0A921F700A9B12
:1081E8005A1C0A921870304613F016FDFEF701BBB0
:1081F8002B4F9FED2C8AB7F9022027480B9007EEEA
:10820800902AF8EEE77A12AE67EE887AA0F13D017F
:10821800FDEEE77A46F8201D00F8403C0823CDED36
:10822800027A00F83F3C1E23BDF8081000F83E3CD7
:108238003046FAF7FBFDB7F9003007EE903AF8EE52
:10824800E77A304667EE887AFDEEE77ACDED027A76
:10825800BDF80810FAF7EAFDB7F9043007EE903ACE
:10826800F8EEE77A304667EE887AFDEEE77ACDEDEC
:10827800027ABDF80810FAF7D9FD304613F0CCFCA5
:10828800FEF7B4BAF2500020CC500020E450002091
:10829800310CC3306766666678390020C05000200C
:1082A800CC36002058A08B411F85EB519AF802402C
:1082B800C4B1013CE4B2013454445146002211F8DF
:1082C800013B534083EA0313DBB2120ADF0042EAA0
:1082D80003228C4287EA131382EA0302EFD1002AB1
:1082E8007FF433ACB24AB34FB34B1288B349B44CA2
:1082F800FA61DFF8F8921A6809689B68FA62B4F8BC
:108308005A21F866FB64D9F80000F963FA65F7F7B3
:10831800F3FF029000287EF499A90221D9F8000001
:10832800F9F746F894F85C319AF803200392642B25
:108338004FF0040287F8742040F05C8194F85D31B6
:10834800072B04BF9DF8083084F85D3194F85D313F
:10835800069307EB031ADAF804100291084624F092
:1083680095FBDAF8081005915FFA80FA084624F0C0
:108378008DFBC0B204900AEB0002069B914802995B
:1083880002900832C27123F00F0286468272049866
:1083980003F00F0300EBCA008EF80D3052468EF83A
:1083A8000E000EF10F0025F079FA874B049A059913
:1083B8000AF10900184425F071FA0298C37903F10B
:1083C800010ACBB1013B5FFA83FC0CF1080CDFF822
:1083D80020E284440023073010F8011B59408B0029
:1083E800CA0883EA410302F018024B404EFA02F22F
:1083F80053408445DBB2EFD1734A03980AF8023040
:1084080021F0B0FB94F85D310022013384F85D312E
:1084180084F85C21029BDDF808A09B785BB11AF810
:108428000510D9F80000F8F7D7FF01359AF802309F
:10843800EDB2AB42F3D894F85C310322013384F8EF
:108448005C3187F8742088F80020FFF753B80221C0
:10845800D8F80000F8F7ACFF94F83431FEF7B3B859
:108468004FF000094846FFF7ECBA4046FFF7D2BA8A
:108478001023042218460AA98DF82A908DF82B900B
:108488008DF82C908DF82D908DF828308DF82920B6
:108498001BF0D0F884F83F91FEF7C0B84B49881F0D
:1084A8001AF096FF84F84E01FFF7A0B8484AD27830
:1084B800002A0CBF4FF0040C4FF0050CFEF74ABE23
:1084C8003B4B1988FFF750BA0123D8F800003B70DE
:1084D800F8F776FF0746D8F80000F8F771FF7F062F
:1084E8007EF442A88E287EF43FA894F82831002B09
:1084F8007EF457A8374BC4F830312D2384F8343133
:10850800FEF739B80326344943E5344B344A1B682F
:10851800344903F48003834216BF11460426032618
:1085280028E523499A790B8803EB830303EB83033C
:108538004FEA83081FFA88F8002A00F003811E4BCF
:108548001B680FFA83FA08F025F940B2FEF720BA43
:108558004FF03408FFF7F4BB984699461846049341
:1085680005930393FEF70CBB1F49042611E54FF052
:108578002408FFF7E5BB4B1CDBB2042B84F8513110
:108588004FEA01617FF4A1A9FFF79CB94FF01008E9
:10859800FFF7D6BB08F0FEF81BF00EF900201BF021
:1085A8000BF9FFF75ABA4FF02008FFF7C9BB00BF15
:1085B800CC5000201C000020C05000203C2D002082
:1085C800A41E0020FC6A0020026B0020EC1F002083
:1085D800F0360020F839002018280308744D0020D0
:1085E800142803080C2803081C28030848540020F2
:1085F8000007090E97F875A0654904951AF00F0F42
:1086080004BF0AF1010A5FFA8AFABAF1070F28BF14
:108618004FF0010A4FEA0A1C07EB0C03187C5D4B6C
:1086280002930A18002392F824105A4A93725FFAA8
:108638008CF31A46584B964607EB0C024EEA00009C
:1086480001291870D26803F101000CD90239C9B2A6
:108658008D1C1D44034603F8012BAB424FEA12223E
:10866800F9D101310844BC4422F060030AF1010A3F
:108678009CF811205FFA8AFA1343BAF1080F0370C5
:1086880000F101035AD04FEA0A1C07EB0C01424AD9
:10869800087C3F4901449A1A91F8241055180EF1A4
:1086A800100E132D5FFA8EFEC6DD049D0298DFF8CA
:1086B800F4E0D1B28B1DDBB243F04002C27103F18A
:1086C800010CCBB14B1DDBB20833C31804930EF178
:1086D8000100002310F8011B59408B0083EA410375
:1086E800CA084B402D4902F0180241FA02F25340E1
:1086F800049A8242DBB2EDD103980CF80E3087F869
:1087080075A021F02FFA85E63B685E2098473B6804
:10871800392098475FFA89F01BF04EF84FEA192084
:108728001BF04AF8F0E44FF00808FFF709BB1C4BB0
:108738009046B3F900A06420FEF72AB9164A049DB2
:108748009A1AB3E74FF0FF33FBE698469946184666
:1087580004930393FEF714BA98469946184604936F
:1087680005939E460393FEF70BBA0393FEF708BAE8
:1087780098460393FEF704BA984699460393FEF782
:10878800FFB99846994618460393FEF7F9B900BF12
:1087980058000308FC6A0020096B00200007090E36
:1087A800C0500020026B00202DE9F047B0F90840C6
:1087B8000C81E4B2442C8AB00D46164600F033848E
:1087C800074642D9812C00F06F8300F29480542C24
:1087D80000F0C78040F2D1806E2C00F0F283802C2C
:1087E80040F0CE80724B93F8009009F1020919F01D
:1087F800FF0900F093806F4B6F4F704EDFF8E4A1D4
:10880800994403F101080A2416E0322C01F0398258
:10881800A4F13C00C0B2132841F23D8200232A682B
:10882800511C296014702A68C84502F101012960A9
:10883800137073D018F8014B0A2CE6D1BAF800303F
:10884800FF2BA8BFFF23DBB2E9E7052C00F0D98393
:108858001ED8022C7DD040F20783032C00F0A7839A
:10886800042C40F08D80564928462246FAF7D4FA5F
:1088780000212846FAF700FB2A680021531C01242E
:108888002B602046234611706B810AB0BDE8F08743
:10889800242C5CD040F29E82282C00F04D83382C8A
:1088A8006ED10A68474B0124511C296014702A684C
:1088B80005211019286011702A680A2110192860EA
:1088C80011702A6800211019286011702A68197817
:1088D8001019286011702A685978101928601170C9
:1088E8002A68997813192B602346117020466B81EA
:1088F8000AB0BDE8F087A02C17D040F28A82B82CC5
:1089080000F05383FE2C3BD12F4C04F1080634F8B9
:10891800021B2846FAF7B0FAA642F8D101242346EA
:1089280020466B810AB0BDE8F087284B08461968D5
:10893800FAF78AFA264B28461968FAF785FA254B7A
:10894800196828460124FAF77FFA2346E8E7224BFC
:10895800F6E70422214928460124FAF75DFA23465E
:10896800C4E70B6800215A1C2A6019702A68012480
:1089780013192B6023461170B8E7522C3FF47CAFD3
:1089880029462046FBF7BEFB0028C7D1742C00F00F
:108998007E82772C28D13B687A689A421BBF5A1C82
:1089A8003A60014619780E4A28461FF017F9B5E7CC
:1089B8001D500020AC00030867666666842400200A
:1089C80041360020633B002040500020ACF7FF1FD9
:1089D800B0F7FF1FB4F7FF1FB43C0020A828030816
:1089E800A56E0208AC240020F52C00F04983292C40
:1089F8003E6801F0CE81392C01F0B981212C01F0BB
:108A080096817A680B3C931BEF2C00F2058401A138
:108A180051F824F0AB9A000821920008219200082E
:108A28002192000821920008219200082192000852
:108A38002192000821920008219200082192000842
:108A48002192000821920008219200082192000832
:108A58002192000821920008219200082192000822
:108A68002192000821920008219200082192000812
:108A7800219200085B9A000821920008419A000898
:108A8800219200081F9A00082192000821920008EC
:108A980021920008AF9B000821920008399B00082A
:108AA80021920008079B000821920008E19A00081B
:108AB800219200080D9A000821920008B99900082F
:108AC800219200084199000821920008219200088B
:108AD80021920008219200082589000821920008A7
:108AE800259900082192000821920008319C00086D
:108AF80021920008D79B00082192000821920008C3
:108B08002192000821920008219200082192000871
:108B180021920008219200084B9C0008219200082D
:108B2800D798000821920008219200089998000817
:108B38002192000821920008219200082192000841
:108B4800219200082192000821920008CD97000880
:108B5800219200084B97000821920008A19600086E
:108B680021920008CD95000821920008A5950008DB
:108B78008795000821920008219200082192000898
:108B880021920008219200082192000821920008F1
:108B980021920008219200082192000821920008E1
:108BA80021920008219200082192000821920008D1
:108BB80021920008219200082192000821920008C1
:108BC80021920008219200082192000821920008B1
:108BD80021920008219200082192000821920008A1
:108BE8002192000821920008219200082192000891
:108BF8002192000821920008219200082192000881
:108C08002192000821920008219200082192000870
:108C18002192000821920008219200082192000860
:108C28002192000821920008219200082192000850
:108C38002192000821920008219200082192000840
:108C48002192000821920008219200082192000830
:108C58002192000821920008219200082192000820
:108C68002192000821920008219200082192000810
:108C78002192000821920008219200082192000800
:108C880021920008219200082192000821920008F0
:108C980021920008219200082192000821920008E0
:108CA80021920008219200082192000821920008D0
:108CB80021920008219200082192000821920008C0
:108CC800219200085D950008219200084795000848
:108CD80021920008219200082192000821920008A0
:108CE8002192000821920008219200082192000890
:108CF8002192000821920008219200082192000880
:108D08002192000821920008EB94000821920008A3
:108D1800B39400082192000817940008FD930008F6
:108D2800E193000821920008799300082192000835
:108D3800519300083F930008E5920008219200082B
:108D4800B792000821920008219200089592000825
:108D580067920008539200082B92000803920008BB
:108D6800E191000821920008C991000821920008A9
:108D780021920008219200082192000821920008FF
:108D880021920008219200082192000821920008EF
:108D980021920008219200082192000821920008DF
:108DA80021920008AF910008219200082192000842
:108DB800579100082192000821920008219200088A
:108DC80021920008219200082192000821920008AF
:108DD8003F910008202C7FF4D3AD0B68964C591CAA
:108DE800627829601A702B682278591C29601A70D9
:108DF8002B68A278591C29601A7021892846FAF72D
:108E08003BF82B686279591C29601A702A68A17985
:108E180034E5822C7FF4B4AD0B68884A884C11780D
:108E2800854A581C2860197011892846FAF724F8D1
:108E3800844B2A681B88FF2B02F10101A8BFFF237E
:108E480029601370A16881F3100189B22846FAF7E6
:108E580013F8216801F30F0189B22846FAF70CF8D4
:108E6800794B2A68197809E5012C7FF489AD0B68DC
:108E78000022591C29601A702B685A1C2A601C7021
:108E88002A682421531C2B60234611702EE53B6869
:108E98007A689A421BBF5A1C3A60014619786B4A95
:108EA80028461EF09BFE39E5694B1E78033616F0FE
:108EB800FF063FF433AD674B674F1E4403F10109CA
:108EC8004FF00A0820E0B8F1500F00F0E186B8F141
:108ED800320F00F0F686A8F13C00C0B2132840F229
:108EE8000D87002421462B685A1C2A60284683F8DF
:108EF8000080F9F7C1FF21462846F9F7BDFF4E4526
:108F08003FF40CAD19F8018BB8F10A0FDBD1534BC4
:108F18009C68196804EB84044FF6FF7364009C4254
:108F2800A8BF1C469942A8BF194624EAE47421EA5E
:108F3800E171A4B289B2D6E70B68DFF84081484EE8
:108F4800591C022229601A702B6806275A1C2A60AD
:108F58001F702B680A22591C29601A702B6801247B
:108F68001A192A601C70B8F800102846F9F784FF0F
:108F7800B8F802102846F9F77FFF2B681A192A60FB
:108F88001F702B685022191929601A702B6800224B
:108F9800191929601A7031882846F9F76DFF718808
:108FA8002846F9F769FF2346A0E42E4BC8E40B686E
:108FB8005A1C0A601C700B680222591C29601A701E
:108FC8005AE4204B0A681B881D4CFF2BA8BFFF23BF
:108FD800511C29601370A16881F3100189B22846D9
:108FE800F9F74AFF204B28461988F9F745FF216809
:108FF80001F30F0189B228460124F9F73DFF234602
:1090080074E40B2219492846F9F706FF0822184983
:109018002846F9F701FF0124072216492846F9F7DF
:10902800FBFE234662E4002A3FF478AC124B13603F
:10903800012423465AE400BFE0360020F250002005
:10904800C0500020CC5000202A390020857A020820
:109058001D500020BC0003087C2400203824002078
:109068006C2400205C2E002024390020B02803083E
:10907800BC280308C828030835400008AC2D002088
:109088003B687A689A4240F09E86C04BFF221A706D
:109098004FF00009BE4C21F097FE49462022BD48FA
:1090A80084F8009026F079FE8DF804909DF804303D
:1090B800072B00F2E486DFF81483B64F4A469DF882
:1090C800043003EB430308EBC3035B7CE3B19DF877
:1090D800043003EB430308EBC30320215B699BB116
:1090E8009DF8043003EB430308EBC303586947F8C2
:1090F8002200F8F7A5FF237857F82300F9F762F95B
:1091080022780132D2B222709DF804300133DBB2EA
:109118008DF804309DF80430072BD0D92B68591CE2
:1091280029601A70002E3FF4F9AB9B4B3360012481
:109138002346FFF7DBBB994B1B78DB076CD4012474
:10914800FBF7D2FFFCF7F0FD2346FFF7CFBB731CFC
:109158003B6033780F2B5FD8B21C3A60C3EBC30374
:109168008F4A7178D154F11C39601344B2785A701F
:10917800321D3A60F2789A70721D3A603279DA706C
:10918800B21D3A6072791A71F21D3A60B2795A7159
:1091980006F108023A60F2799A7101241CF044FA47
:1091A8002346FFF7A3BB3846F9F724FE7D4EF0812E
:1091B8003846F9F71FFE0124B0812346FFF796BB16
:1091C8003846F9F717FE784A00EB8000430001247F
:1091D80013802346FFF78ABB3846F9F70BFE734E18
:1091E80030823846F9F706FE70823846F9F702FEF3
:1091F8000124B0822346FFF779BB3346721C3A60DC
:1092080013F8020B3B60F31C71783B60B27813F0E3
:1092180001F900287FF482AB4FF0FF342346FFF7B3
:1092280065BB3346721C3A60614A13F8021B117021
:109238003B605C4A73789370F31C3B605A4BB2787E
:109248009A7001242346FFF751BB5A4B5A491868B4
:109258004E22012424F022FB2346FFF747BB324667
:10926800731C3B60554B12F8021B19703A607278F8
:109278005A70F21C3A60B2789A703846F9F7BAFD1B
:109288004F4B0124D8802346FFF730BB3846F9F707
:10929800B1FD4B4E30803846F9F7ACFD708038464A
:1092A800F9F7A8FD0124B0802346FFF71FBBDFF8BC
:1092B800208198F80030002B3FF430AB414E002459
:1092C8003846F9F797FD0BF057FA98F80030A6ECF6
:1092D800010A01349C42F3DBFFF720BB0D2B9BD125
:1092E800731C3B603478072C96D8DFF8E880384642
:1092F8000C26F9F77FFD06FB04F608EB0604A080B0
:109308003846F9F777FDE0803846F9F773FD3B6892
:1093180020811A46591C396012F8021BA1723A6062
:109328005B78E3723846F9F74DFD012448F80600EA
:109338002346FFF7DBBA3846F9F75CFD224B0124D8
:1093480018802346FFF7D2BA731C3B6030780606B4
:1093580000F1D985114B1B78DC073FF5DFAA0328FC
:1093680028BF00200124FBF7A3FE2346FFF7BEBA5F
:109378000A4B1B78D8073FF5D1AA0124FBF786FFD3
:10938800FCF7D2FC2346FFF7B1BA00BF78210020D2
:10939800CB540020CC530020714F0208D235002056
:1093A800EC55002028440020A43400204847002021
:1093B800CC4A00204836002000050308102D002064
:1093C80034300020882F00200C2D002088460020F3
:1093D8001D50002084580020A34B1B78DA073FF566
:1093E8009DAAA24A1378012443F00403137023466C
:1093F800FFF77CBA9C4B1B78D9073FF58FAA9C4B8B
:109408004FF4C87201241A802346FFF76FBA092B5C
:109418007FF702AFDFF87C823346721CD8F8004031
:109428003A6013F8022B22703B607378A370F31C28
:109438003B60B378642BA8BF6423321D63713A6024
:10944800F378642BA8BF6423721DA3713A60337943
:10945800E371B31D3B607379642BA8BF6423F21DCD
:1094680023723A60B379E37006F108033B60F3793D
:1094780023713846F9F7BEFC7A683B686081D11AD7
:1094880000290CDD591CD8F800003960521A002A4E
:109498001978417203DD9A1C3A605B7843700124A5
:1094A80022F000F92346FFF721BA724B1868F31C23
:1094B80002462136991E396013F8031C1170591E93
:1094C800396013F8021C51703B6013F8011C91704D
:1094D80003339E4202F10302ECD11CF057FCFFF764
:1094E8001DBAC3F34704122C3FF696AEBCB10AABC3
:1094F8000DF1020803EB44094646A9F1260938464E
:10950800F9F778FC26F8020FB145F8D15A4B38F82C
:10951800022F23F8022F4645F9D1112C09D8574AB2
:109528006300023B13440021223223F8021F9A42AF
:10953800FBD1534A01231C461370FFF7D7B9514E8C
:10954800002338463360F9F73DFC01243060234698
:10955800FFF7CCB93346721C3A6013F8024B3B60F4
:10956800F31C70783B60B178002C00F0D784012C94
:109578007FF4D4A921F0B4FE2346FFF7B7B93A4BDC
:109588001B7813F001017FF447AE731C3B60307801
:10959800012421F0E7FD2346FFF7A8B93346721CE2
:1095A8003A60394A13F8021BD1703B60374A737826
:1095B8005371F31C3B60364BB278DA7001242346B2
:1095C800FFF794B93846F9F715FC3846F9F712FC55
:1095D8003846F9F70FFC3846F9F718FC3B68254C74
:1095E8001946581C2268386011F8020B82F82C00C2
:1095F8003960597882F83610D91C39609B7882F81E
:1096080037303846F9F702FC3846F9F7FFFB384699
:10961800F9F7FCFB38462668F9F7ECFB7087384603
:109628002668F9F7E7FB3B687A683087D11A012981
:109638000ADD591C226839601B7882F82E303846BA
:10964800F9F7E4FB3B687A68D31A032B09DD38463F
:109658002668F9F7CFFB708638462668F9F7CAFB03
:10966800B086206839E700BFD2350020FC310020E1
:10967800EC70002048360020CE520020D052002046
:10968800F45200205C2E002028440020483B002093
:10969800A4340020CC700020731C3B60B94CDFF868
:1096A8000883337888F8053038462668F9F7A2FB2E
:1096B800308438462668F9F79DFB7A683B68F08362
:1096C800D11A072915DD3846F9F794FBA8F80A00DE
:1096D8003846F9F78FFBA8F80C0038462668F9F7E2
:1096E80089FB708438462668F9F784FB3B687A68FA
:1096F800B084D11A03290BDD3846F9F77BFBA8F8AB
:109708000E003846F9F776FB3B687A68A8F810002F
:10971800D21A002A05DD591C226839601B7882F8A4
:109728002630FBF7EBFC17F025FF974B1B68002B47
:1097380000F0BF83206801241CF00AF82346FFF7D5
:10974800D5B83346721C3A60DFF85C8213F8022BF6
:1097580088F802203B608D4A73781370F31C3B60D5
:109768008B4CB3782371331D3B60F378092BA8BF6A
:1097780009233846A370F9F73DFB3B687A682080D7
:10978800D11A012905DD3846F9F734FB3B687A68B8
:10979800E0819A4207D05A1C3A601B78003318BF00
:1097A800012388F80730FBF7A9FC3B687A689A42DE
:1097B8003FF4B4A85A1C3A601B78E370012423468E
:1097C800FFF794B83846F9F715FB044611F0E2F9AB
:1097D800FF283FF4A3A83F2C00F254830DF128087A
:1097E800002308F8243DE60841460DF103008DF8F2
:1097F8000330013611F0AEF99DF80330F6B204F0EB
:109808000704B34204F1010403D19DF80430A342D4
:1098180003D02146304611F0A9F93B687A68D21A7C
:10982800012A7FF77BA85A1C0AA83A6000221C78F4
:1098380000F8252D11F082F99DF80330A3420AD0D3
:10984800544B1B683BB19A79A24204D31B681B692D
:109858000BB1204698473B685A1C3A6040460022A4
:109868001C788DF8042011F05DF99DF80430A342AE
:109878003FF454A8474B1B68002B3FF44FA81B68C4
:109888005B69002B3FF44AA820469847FFF746B883
:10989800414B1B78012B3FF641A83346711C3960B8
:1098A800DFF8088113F8021B88F80210F11C3B60EE
:1098B800531A012B7078396040F336833846F9F72C
:1098C80099FA0124A8F800002346FFF70FB8731C83
:1098D8003B6096F80080B8F1110F3FF69DACB31CC1
:1098E8003B602E4C737804F818303846F9F782FA42
:1098F80040F6CA039842A8BF184640F2EE239842A1
:1099080004EB4801B8BF18460124A0F2EE22234612
:10991800192092FBF0F24A70FEF7E8BF3346721C3A
:109928003A601F4A13F8021B91703B6073785370BA
:1099380001242346FEF7DABF0722B3FBF2F2C2EB9B
:10994800C2041B1B7FF468ACD2B202F1FF385FFA85
:1099580088F8002A3EF4E2AFDFF8489008F10108E1
:109968001C46731C3B600F4B96F90010002693F9B8
:1099780002208A4203F1080300F05C820136052EBA
:10998800F5D149E4483600201C3400209C570020BB
:109998004847002040370020913C00209854002080
:1099A800F070002054440020CC4A0020943C002051
:1099B800731C3B6033780E2B3FF62EACB21C3A601A
:1099C800707803283FF628ACC049062202FB03F250
:1099D8008B18F41C58713C60B0788854321D3A607A
:1099E800F2785A70721D3A6032799A70B21D3A60F4
:1099F8007279DA70F21D3A60B2791A71012423463D
:109A0800FEF774BF731C3B60B14B32785A75012462
:109A18002346FEF76BBF3846F9F7ECF9AD4E3060D8
:109A28003846F9F7E7F970603846F9F7E3F90124A1
:109A3800B0602346FEF75ABFA74E0023336038466E
:109A4800F9F7C0F933680124034333602346FEF76E
:109A58004DBF731C3B603478132C3FF6DDABB31C51
:109A68003B6070781EF0F4F800283FF4D5AB9B4BB0
:109A7800027803F82420F21C3A6003EB8403B278DE
:109A88005A70321D3A60F2789A70721D3A609449A1
:109A98003279DA700868012421F092FD2346FEF736
:109AA80025BF9049102B4FF0000228BF10230A60F1
:109AB8004A608A60CA600A74002B3EF42FAF3A6885
:109AC8000139134401323A6012F8010C01F8010F10
:109AD8009342F7D1FEF722BF721C3A6034781F2CEC
:109AE8003FF69AAB052B7FF497AB3846F9F76AF93E
:109AF8007D4B43F8240010F0D5FDFEF70FBF7A4CDC
:109B080004F140063846F9F775F93B68A4F8800077
:109B1800591C1A46396012F8021B84F882103A6000
:109B28005B7884F883300434B442EBD1FEF7F6BE98
:109B3800731C674C3B60337823723846F9F75AF93F
:109B4800A0833846F9F756F920833846F9F752F9D1
:109B58003A686083531C3B601278E2747A68D31ABF
:109B6800032B00F3B1813B68D11A05290EDD5A1C7D
:109B78003A601B78E3723846F9F724F93B68E060ED
:109B88005A1C3A601B7823743B687A68D21A002AF8
:109B98007EF7C4AE5A1C3A601B7884F82130012441
:109BA8002346FEF7A3BE731C3B605049307808700B
:109BB800D31A002B7EF7B2AEB31C3B607378003328
:109BC80018BF012301244B702346FEF78FBE731C78
:109BD8003B60464B3278DFF800811A700023C8F8E2
:109BE80000303846F9F7EEF83A68D8F800303849C6
:109BF800384C0343501CC8F80030386013780B7297
:109C08003846F9F7F7F820603846F9F7F3F8606056
:109C18003846F9F7EFF8A0603846F9F7EBF8384618
:109C2800F9F7E8F8FEF77ABE314B06F1080101367C
:109C38003E6016F8012C03F8012F8E42F7D1FEF78B
:109C48006DBE3346721C2B4C3A6013F8022B2271FE
:109C58003B60737863713846F9F7CCF83B6820802D
:109C68005A1C3A601B78A3713846F9F7C3F83B6869
:109C780060805A1C3A601B78E37101242346FEF782
:109C880035BE3388FF2BA8BFFF23DBB2FEF7C7BD65
:109C9800194BFFF73DB919F0F7F900283EF4BEADAE
:109CA80003780A2B41D8B0F9023087FB0312DB177F
:109CB800C3EBA2039BB2FF2BA8BFFF23DBB2FEF7C7
:109CC800AEBD97E81200FFF725B900BF682E002047
:109CD800304F0020A02C0020B43C00203834002055
:109CE8004836002058300020F03700203434002057
:109CF8002F4F0020503000207024002019F0C4F9A4
:109D080000283FF4EEA803780A2B3FF6EAA8B0F93A
:109D18000430B0F9061003EB830383F3500421EAFF
:109D2800E171A4B289B2FFF7DEB80023C6E7334673
:109D3800721C3A60834C13F8022B62703B60737894
:109D48002370F31C3B60B378A3703846F9F752F8D8
:109D58003B682081591C1A46396012F8021B617150
:109D68003A605B78A37101242346FEF7BFBD731CDC
:109D78003B6033780A2B4ED03846F9F747F8384617
:109D8800F9F744F801243846F9F740F82346FEF776
:109D9800ADBD731C3B6033780A2B0FD0502B7FF47A
:109DA8003BAF3846F9F726F8674E30803846F9F762
:109DB80021F8012470802346FEF798BD3846F9F74C
:109DC80019F8624EF1E75A1C19463A60604811F8D2
:109DD800022B027039605B784370042A04D9FF2A89
:109DE8007EF44AADFFF754B95A490978994205D823
:109DF800022A7EF441ADFF2B7EF43EAD2B68012490
:109E08001A192A601C70002E3EF488AD524B33603C
:109E18002346FEF76BBDB31C3B60504B72781A703B
:109E2800F21C3A60B2785A70321D3A60F2789A7031
:109E3800FEF774BD09EBC60A38468AF80210F8F72F
:109E4800D9FF3B6829F836001A46591C396012F8C0
:109E5800021B8AF803103A605A788AF80420DA1C40
:109E68003A609A788AF806201E1D3E600134DB7835
:109E78008AF80530A0457FF474ADFEF74FBD4A4619
:109E8800FFF74CB90DF10408404610F03FFEBDF84D
:109E98000430A3423FF4C1AC314B1B68002B3FF4A4
:109EA800BCAC1B689B69002B3FF4B7AC20469847B5
:109EB800B3E42C482C492D4A2D4B036001240B6038
:109EC80013602346FEF712BD3846F8F793FFA084C7
:109ED8003846F8F78FFF3B687A68E084D11A03297F
:109EE8007FF742AE1A46591C396012F8021BA17757
:109EF8003A605B7884F820303846F8F77BFF3B6897
:109F08007A68608430E600F07F00032828BF0020CC
:109F1800012421F001FA2346FEF7E8BC01241BF0D6
:109F2800ADFD2346FEF7E2BC124BB1781A88012436
:109F380012FB00F2234692FBF1F2A8F80020FEF78C
:109F4800D5BC00BFE03600206C240020AC2D0020DA
:109F5800782100201D5000204D400008633B002060
:109F680040370020DC56002030570020985700204A
:109F780021060008887200202DE9F04F2DED0C8B8A
:109F8800404B1B7893B0012B039001F0BC803E4CF2
:109F980094F80021002A41F0C780072B01F0CE80F9
:109FA8004FF0000ADFF8ECB0DBF804305846984769
:109FB800002800F06F81BBF8B46000228BF85520B0
:109FC800002E40F06687BBF93C50DBF82410BBF943
:109FD8003E00DBF82820BBF94030691ACBF8301076
:109FE8002A490191821ADBF82C00CBF834200D465F
:109FF8001B1A9BF85610CBF838300BF1300015F0CF
:10A008005FFE2B68990040F1E980DBED0D5ADBED2E
:10A018000C7A1F4A94ED416AD4ED426A94ED437A72
:10A02800D4F810311268B8EEE58ADBED0E5AF8EE76
:10A03800E77AF8EEE58A013377EE867A38EE268AF3
:10A0480078EE878A9342C4ED417A84ED428AC4ED62
:10A05800438AC4F8103101F0F1820A4B1E78142E9D
:10A0680002F0A1840023D4F818510293062D00F2BF
:10A07800A880DFE815F0F712E6120B127B12110028
:10A088002114BA133C5000207C210020744D00207C
:10A0980080400020E04A0020D44B1A78D4F81C7184
:10A0A800DFF8B8E39FEDD27AF8000EEB000383EDFA
:10A0B800007A002A7AD0CF49B0EE476AF0EE476AB4
:10A0C8000023F1EC017A013367EEA77A05EE903AA6
:10A0D800B4EEE77AF1EE10FAF8EEE55AB8BFB0EE52
:10A0E800677A9A4276EEA76AA7EEA56AE9D1F5EEF5
:10A0F800C06A0EEB0003F1EE10FA83ED007A55DD2D
:10A10800C6EE265ABC4BBD4A1288F7EE007A75EEA9
:10A11800E75AD3ED007A65EEA77AFDEEE77A17EEF7
:10A12800903A812B43F317839342A8BF134607EE57
:10A13800903AF8EEE77AB24BC11903EB810393ED3D
:10A14800057AD3ED003A93ED066A93ED014AD3ED13
:10A15800046AD3ED034A93ED025AA3EEA77AA4EE5C
:10A16800276A66EEC76AA7EE646ABDEEC77AE5EEAF
:10A17800276A17EE101A812983ED056AC3ED066A6E
:10A1880043F3E6828A42A8BF0A4607EE902AF8EE11
:10A19800E77AFCEEE77ACDED047ABDF810300EEBE5
:10A1A8000002938017B9132E03F0A687152E42F0EC
:10A1B800BF817044DFF8A882838828F81730D4F864
:10A1C8001851904B013583FB05235A19EB17C3EB44
:10A1D800A203C3EBC303ED1AC4F818518A4B1B78CA
:10A1E800002B01F0E380894DCDF808A0DFF87482D8
:10A1F800DFF86C92DDF804A005F5BC770026844BE7
:10A20800DBED087A1B78172B01F0258495ED007A91
:10A21800B8EEC78A082B28EE278A07D1B0EE480A7D
:10A22800019323F0AFFC019B29F81600DAF800200F
:10A2380092000BD5002E04F00981B0EE480ADBF835
:10A24800143207F170009847B0EE408AB0EE480A21
:10A25800DBF83431A7F170009847DBF8A4313846B1
:10A2680098476B4B1B78032BB0EE408A01F0ED83C7
:10A27800D5F8F800DBF8B830B0EE480A9847013650
:10A28800032E07F12407A8EC010A05F10405B6D14D
:10A29800DDF808A05E4B1F78072F00F0BA8694F807
:10A2A80028310493002B40F0C2865A4B5B79002B6F
:10A2B80040F0E9850123564A84F828311278072AA4
:10A2C80001F0748600230593534B94ED4C9A93ED5B
:10A2D800007A524BD4ED4BCAD3F800A0504B0293EE
:10A2E800F7EE007A37EEC9CA00252CEE07CA4D4BA7
:10A2F800DFF87491DFF874B1DFED4B8A9FED4BAA5C
:10A30800DFED3BBADFED4A9A9FED4ABADFED4AAA84
:10A31800DFF85C81494F0193B4EEE7CAF1EE10FA19
:10A3280088BFB0EE67CA2E46454B99ED008A2B448C
:10A33800D3ED007AF5EE407AF1EE10FA17D0414BE2
:10A348002B44D3ED006A38EE667AB0EEC76AF4EEB5
:10A35800C67AF1EE10FA08D5B5EEC07AF1EE10FA29
:10A36800CCBF37EEA68A36EEE78A83ED008A364BF5
:10A378001A8893077ED0022E7CD09AF82E10334B81
:10A3880007EE901A2B4493ED007A4B42F8EEE76AF9
:10A3980007EE903A26EE877AF8EEE77AB4EEE77A97
:10A3A800F1EE10FA0AD407EE901AF8EE677AF4EE96
:10A3B800C77AF1EE10FA88BFF0EE477A244B2549A8
:10A3C80003EB460331F91600B3F90C30C01A07EE57
:10A3D800100AB8EEC77AD007E7EE687A40F12F8600
:10A3E8001D4B93ED008A27EE888A43E086400020C3
:10A3F800000000007C2100208840002084400020CC
:10A40800BC420020932449927D400020104B00203C
:10A418003C500020CC4A0020F0570020483600204D
:10A42800644D002000320020CDCCCC3DAE47813FAA
:10A438000000C84200003443610BB63B0C320020D8
:10A44800E4570020BC22002026390020C822002022
:10A4580028440020CC360020CC570020A4420020FD
:10A4680040500020684D0020B0220020D85600201F
:10A4780018320020029B94F864212B44D3ED01DAB2
:10A4880038EE6DDA002A3DD0D34BD4F86821039911
:10A498001B688A1A9A4235DD9AF84830022B01F077
:10A4A800BC85022E03F05987CC4B1B68990740F1F5
:10A4B8006487CB4BCB49DFF8A0E331F916C09EED9A
:10A4C800008ADFF898E3C7ED00BA03EB460028EEF0
:10A4D800288AB0F90C00A0EB0C0007EE900AF8EE01
:10A4E800E77ADEF8000027EE888A904238EE6DDAC7
:10A4F800C1F27980F7EE007AB4EEE79AF1EE10FA3D
:10A5080001F14880B84B2B4493ED000A019B2CEED7
:10A51800800A022E20EE0D0AA3EC010A019303F033
:10A528004487B24B9BED007AD3ED007AB04BD7ED60
:10A53800006A93ED006AAF4B67EE277A2B4427EE4B
:10A548008C7AD3ED007A67EE277AF0EE665AEDEE54
:10A55800275AB1EE467AF4EEC75AF1EE10FA08D44B
:10A56800F4EEC65AF1EE10FA8CBFB0EE467AB0EEB1
:10A57800657A94ED4C6AF7EE007AB4EEE76AF1EE8C
:10A5880010FAACBF0123002343B1F0EEE66AF0EE07
:10A59800C77AF4EEE67AF1EE10FA01D587ED007A83
:10A5A800022E03F0D386944A944B52F826001B6877
:10A5B800B0EE6D0A9847924A924B52F826001B68F3
:10A5C80098479AF8373023B18F4B1B88002B00F03F
:10A5D800BA85B0EE6B8A8D4B9BED007A38EE400A57
:10A5E8002B4493ED008A83ED000A9AF8483030EE48
:10A5F800480AC0EE077A2BB3854B1B78DB0721D5B9
:10A60800B7EE007AB4EEC79AF1EE10FA04DB94F8CC
:10A618006431002B00F06587D4F86831039AD31AA7
:10A628006D4A12689A420DDD7A4B93ED007AB0EECE
:10A63800CDDAB4EEC7DAF1EE10FA40F1F087002374
:10A6480084F86431744B94F874212B4493ED007AA8
:10A658002CEE877A67EE277AC8ED007A32B9019B2B
:10A66800C7ED00BA43ED01BAC8ED00BA0136032EB2
:10A6780009F1040908F1040807F1040705F10405C4
:10A688007FF452AE654B1B78072B01F01482012B27
:10A6980001F091840023029394F87C31002B40F060
:10A6A80097855F4B5F4A1B68126813F4805C92F8C9
:10A6B8002C2040F0A4865C495C4891ED006A408BF0
:10A6C8005B4984ED636A91ED007A5A4984ED647AB6
:10A6D80007EE900AF8EEE76AD1ED037A564984ED61
:10A6E800616A37EE467A77EEE67AD1ED006A84ED54
:10A6F800607A012184F89411C7EEA65A4F48504950
:10A7080090ED005A4F489FED506A90ED004A4F482F
:10A71800DFED4F6AD0ED004A91ED007A35EE045A2C
:10A72800F7EE007AF4EEE75A35EE245AF1EE10FA15
:10A7380088BFF0EE675A25EE065AF4EEE65AB1EEF7
:10A74800476AF1EE10FAB4EEC65AB8BFF0EE665A90
:10A75800F1EE10FAC4ED665A00F1FD87B4EEC75A5F
:10A76800F1EE10FA88BFB0EE475A3449DFED366A89
:10A77800D1ED017A334991ED014A344977EE847A73
:10A78800D1ED014A77EEA47A67EEA67AB4EEE76ACD
:10A79800F1EE10FA08DCB4EEE77AF1EE10FA8CBFAD
:10A7A800B0EE676AB0EE476A2449DFED276AD1ED5B
:10A7B800027A2449D1ED024A264977EEA47A91ED2E
:10A7C800007A67EEA67AB1EE473AF4EEC37AF1EE74
:10A7D80010FA4ED444E000BFF8570020703600202D
:10A7E80028440020CC360020A057002094000020E8
:10A7F80014580020AC570020E0560020DC560020FA
:10A80800345700203057002026390020E822002045
:10A81800D235002004580020B85700203C500020B2
:10A82800744D00204836002088320020304F002028
:10A8380028300020F45000203C3000200032002056
:10A84800185800200C3200206F12833A183200206A
:10A85800000000001C580020CC570020F4570020AE
:10A86800F4EEC77AF1EE10FA8CBFB0EE473AB0EECC
:10A87800673AED49497809B9B1EE433A002A41F0FF
:10A888003E82F7EE003ADFF8C8B39BF80020002AB2
:10A8980002F03782E549DFEDE67AD1ED024AD1EDE3
:10A8A800016A91ED037A66EE244AE5EE264AE3EE64
:10A8B800074A63EEA44AF4EEE74AF1EE10FAB4BF91
:10A8C800B0EE674AB0EE644A98BFF0EE647A012AA7
:10A8D800CDED0A4A02F0368291ED067AD1ED052ACD
:10A8E800D1ED076A26EE077AA5EE227AA3EE267A3C
:10A8F80023EE877AB4EEE77AF1EE10FAB4EEC47A72
:10A908008CBFF0EE676AF0EE476AF1EE10FA88BF86
:10A91800F0EE676AB4BFF0EE447AF0EE477A022AA6
:10A928008DED0B7A00F0DE8091ED0A7AD1ED092ADF
:10A9380091ED0B4A26EE077AA5EE227AA3EE047A69
:10A9480023EE877AB4EEE67AF1EE10FAB4EEE77AFF
:10A958008CBFB0EE664AB0EE474AF1EE10FA98BFE7
:10A96800F0EE446AA8BFF0EE477A032A8DED0C7A20
:10A9780000F0B88091ED0E7AD1ED0D2A91ED0F4AD5
:10A9880026EE077AA5EE227AA3EE047A23EE877ADA
:10A99800B4EEE67AF1EE10FAB4EEE77A8CBFB0EED8
:10A9A800664AB0EE474AF1EE10FA98BFF0EE446AF4
:10A9B800A8BFF0EE477A042A8DED0D7A00F0928058
:10A9C80091ED124AD1ED112A91ED137A26EE044A3F
:10A9D800A5EE224AA3EE074A23EE844AB4EEE64ADD
:10A9E800F1EE10FAB4EEE74A8CBFB0EE667AB0EE3C
:10A9F800447AF1EE10FA98BFF0EE476AA8BFF0EE7D
:10AA0800447A052A8DED0E4A6CD091ED164AD1EDA7
:10AA1800152A91ED177A26EE044AA5EE224AA3EEEE
:10AA2800074A23EE844AB4EEE64AF1EE10FAB4EE91
:10AA3800E74A8CBFB0EE667AB0EE447AF1EE10FACF
:10AA480098BFF0EE476AA8BFF0EE447A062A8DED6B
:10AA58000F4A47D091ED1A4AD1ED192A91ED1B7A88
:10AA680026EE044AA5EE224AA3EE074A23EE844ABC
:10AA7800B4EEE64AF1EE10FAB4EEE74A8CBFB0EE57
:10AA8800667AB0EE447AF1EE10FA98BFF0EE476AB3
:10AA9800A8BFF0EE447A072A8DED104A22D091ED36
:10AAA8001E7AD1ED1D2A91ED1F4A26EE077AA5EEF2
:10AAB800227AA4EE037A27EE237AB4EEE67AF1EE50
:10AAC80010FAB4EEE77A8CBFB0EE666AB0EE476A69
:10AAD800F1EE10FA8DED117A98BFF0EE466AA8BF34
:10AAE800F0EE477A77EEE67AF7EE006AF4EEE67A69
:10AAF800F1EE10FAC4ED4C7A43F39A8286EEA77A07
:10AB0800022ADDED0B7A67EE244A67EE877ACDEDEF
:10AB18000A4ACDED0B7A2DD0DDED0C7A67EE877AF7
:10AB2800032ACDED0C7A25D0DDED0D7A67EE877A14
:10AB3800042ACDED0D7A1DD0DDED0E7A67EE877A09
:10AB4800052ACDED0E7A15D0DDED0F7A67EE877AFE
:10AB5800062ACDED0F7A0DD0DDED107A67EE877AF3
:10AB6800072ACDED107A05D0DDED117A27EE877A28
:10AB78008DED117A2F49096811F0805800F09687F9
:10AB8800F6EE005AC4ED665A002A02F0B18094F934
:10AB98009401D4ED644A284D284994ED636A284EFF
:10ABA800284FDFF8B0E0B5F81AA0C978B6F90690D2
:10ABB80097ED005A9EF800E0D4ED606AD4ED617A12
:10ABC80007EE100AFDEEE44A1F4814EE905A00788A
:10ABD800FDEEC64A03F0100603F4800300F00107F7
:10ABE800B8EEC77A14EE900A0193002941F0C680A6
:10ABF8000E49002E40F07C8791ED006A9DED0A5ABF
:10AC0800124B25EE866AA5EE076AB0EE675AA6EEE5
:10AC1800265ABDEEC56A16EE10EA16EE106AAE4563
:10AC2800A8BF2E4618E000BF34340020A82F00200B
:10AC380000000000F4310020304F0020F0360020E2
:10AC4800D86E0020842F0020D235002060320020EA
:10AC58001D5000206C4700207045C8BF064606EE10
:10AC6800106AB8EEC66A012A83ED006A00F0DC803B
:10AC780091ED046A9DED0B5A25EE866AA5EE076AEA
:10AC8800B0EE675AA6EE265ABDEEC56A16EE10EA71
:10AC980016EE106AAE45A8BF2E467045C8BF0646D8
:10ACA80006EE106AB8EEC66A022A83ED016A00F061
:10ACB800BB8091ED086A9DED0C5A25EE866AA5EEDB
:10ACC800076AB0EE675AA6EE265ABDEEC56A16EEBA
:10ACD80010EA16EE106AAE45A8BF2E467045C8BFEA
:10ACE800064606EE106AB8EEC66A032A83ED026AC3
:10ACF80000F09A8091ED0C6A9DED0D5A25EE866A5A
:10AD0800A5EE076AB0EE675AA6EE265ABDEEC56AEA
:10AD180016EE10EA16EE106AAE45A8BF2E4670452C
:10AD2800C8BF064606EE106AB8EEC66A042A83ED66
:10AD3800036A79D091ED106A9DED0E5A25EE866A68
:10AD4800A5EE076AB0EE675AA6EE265ABDEEC56AAA
:10AD580016EE10EA16EE106AAE45A8BF2E467045EC
:10AD6800C8BF064606EE106AB8EEC66A052A83ED25
:10AD7800046A59D091ED146A9DED0F5A25EE866A42
:10AD8800A5EE076AB0EE675AA6EE265ABDEEC56A6A
:10AD980016EE10EA16EE106AAE45A8BF2E467045AC
:10ADA800C8BF064606EE106AB8EEC66A062A83EDE4
:10ADB800056A39D091ED186A9DED105A25EE866A1C
:10ADC800A5EE076AB0EE675AA6EE265ABDEEC56A2A
:10ADD80016EE10EA16EE106AAE45A8BF2E4670456C
:10ADE800C8BF064606EE106AB8EEC66A072A83EDA3
:10ADF800066A19D091ED1C6A9DED115A65EE865AC6
:10AE0800E7EE055AE6EEA57AFDEEE77A17EE901A18
:10AE18008D42A8BF0D468842C8BF054607EE905A26
:10AE2800F8EEE77AC3ED077A2FB922B19200D34939
:10AE3800D34822F033FDD34B1B68002B40F0A48489
:10AE4800D14B1B7893B19BF8000060B1CC4ECF4F2B
:10AE58000025E8B23B68B6EC010A98479BF8000069
:10AE680001358542F5DBCA4B1B689847C94B1B78EF
:10AE7800072B00F03586012384F8003113B0BDECB0
:10AE88000C8BBDE8F08FC44B1B78013BDBB2FFF79E
:10AE980012BAC24B02934FF47A751B68B5FBF3F3F1
:10AEA800C3EB4315BE49DFF8248391F80190B949F3
:10AEB800B8F906000F7803EB8503DD00ADB2AE42AA
:10AEC80001F08586DBF88810BBF93CE0DBF86C30D4
:10AED8004A1C07EE90EA7344012ACBF88820CBF885
:10AEE8006C30F8EEE77A01F07F86DBED1E5ADBED79
:10AEF800206A07EE102A37EEE56AB8EEC75A012E27
:10AF080086EE057A37EE257A77EEC77A8BED1F7ACB
:10AF1800E7EE866A8BED1E7AF0EE667ACBED216A53
:10AF2800CBED206A02F05080DBF89C10BBF93EE0C4
:10AF3800DBF870304A1C07EE90EA7344012ACBF81C
:10AF48009C20CBF87030F8EEE77A01F06886DBEDEC
:10AF5800235ADBED256A07EE102A37EEE56AB8EECC
:10AF6800C75A012E86EE057A37EE257A77EEC77A2C
:10AF78008BED247AE7EE866A8BED237AF0EE667A1B
:10AF8800CBED266ACBED256A02F04780DBF8B010DE
:10AF9800BBF940E0DBF874304A1C07EE90EA7344D2
:10AFA800012ACBF8B020CBF87430F8EEE77A01F03C
:10AFB8005186DBED285ADBED2A6A07EE102A37EEB8
:10AFC800E56AB8EEC75A012E86EE057A37EE257A7D
:10AFD80077EEC77A8BED297AE6EE276A8BED287A29
:10AFE800F0EE667ACBED2B6ACBED2A6A02F03E8052
:10AFF800A8F80600BBF8B430664A013B1778ABF8EE
:10B00800B43002990023072F4B608B60CB607FF42C
:10B0180046A9F6F727F8DFF8B48194F828310493A5
:10B02800A0EB0A00A8F80000002B3FF43EA9013B62
:10B0380084F8283113B0BDEC0C8BBDE8F08F94ED8B
:10B04800567AB1F90000D4ED576AB1F902E0554AD1
:10B05800F4EEC76A80EAE0738EEAEE71A3EBE07360
:10B06800F1EE10FAA1EBEE71B8BFF0EE476A8B4231
:10B07800B8BF0B4607EE103A1378B8EEC77A27EE3A
:10B08800287A002B40F0FE81474B93ED006AB4EE1E
:10B09800CA6AF1EE10FA40F18487F7EE005A75EEAD
:10B0A800C65A3BEE477A65EEAA5A404BA7EE256A88
:10B0B80093ED007A26EE076AB5EEC06AF1EE10FA53
:10B0C80040F2F084C9EE865AB7EE007AB0EE476ACD
:10B0D800A6EEE56AF0EE466AF4EEC76AF1EE10FAFB
:10B0E80088BFF0EE476AF5EEC06AF1EE10FAB8BF15
:10B0F800F0EE6B6A2E4B93ED007A67EE877AA7EE37
:10B10800A68AFFF7B7B92B4B2B4C19682B4ADFF8E7
:10B11800BC8094F80031C9691288A8F80010A8F812
:10B128000220002B3EF43CAF06F0CEFB002384F84F
:10B138000031184B1B78072B7EF432AFF5F792FFDE
:10B148008246FEF72FBF1E4B1E4A2B4493ED007A12
:10B15800D2ED007A1C4B67EE277AF7EE006AF4EE20
:10B16800E67AF1EE10FA93ED007A88BFF0EE667A8F
:10B1780067EE877A27EE888AFFF72DBA882F002096
:10B1880060320020D0560020744A0020604700201A
:10B19800684700203C5000209C570020644D002048
:10B1A800CC4A0020D8570020E0570020D457002070
:10B1B800D05700205C3B00207C210020D0300020AC
:10B1C800D4220020C8570020C45700204050002037
:10B1D800D94BDFF8B8B31B789BF80020DD077FF563
:10B1E80024AE002A3FF427AED4ED573A94ED564AE0
:10B1F800D24BD4ED617A93ED005A94ED607AD4ED98
:10B20800545A94ED536ACE49CE4BF4EEC43AF3EE59
:10B21800046AF1EE10FA77EEA64A00F1578791ED2D
:10B22800026A26EE656AB0EE674AA6EE074AB4EEF1
:10B23800E44A34EE666AF1EE10FA48BFB0EE456AA9
:10B24800012A83ED006A3FF4F6AD91ED066A26EE19
:10B25800656AB0EE674AA6EE074AB4EEE44A34EEF1
:10B26800666AF1EE10FA48BFB0EE456A022A83ED2D
:10B27800016A3FF4E0AD91ED0A6A26EE656AB0EE28
:10B28800674AA6EE074AB4EEE44A34EE666AF1EE7F
:10B2980010FA48BFB0EE456A032A83ED026A3FF40C
:10B2A800CAAD91ED0E6A26EE656AB0EE674AA6EE63
:10B2B800074AB4EEE44A34EE666AF1EE10FA48BF83
:10B2C800B0EE456A042A83ED036A3FF4B4AD91ED0C
:10B2D800126A26EE656AB0EE674AA6EE074AB4EE31
:10B2E800E44A34EE666AF1EE10FA48BFB0EE456AF9
:10B2F800052A83ED046A3FF49EAD91ED166A26EEA9
:10B30800656AB0EE674AA6EE074AB4EEE44A74EE00
:10B31800666AF1EE10FA48BFF0EE456A062AC3EDF8
:10B32800056A3FF488ADD1ED1A6A66EEE56AB0EEBB
:10B33800674AA6EE874AB3EE046AB4EEE44A74EEAE
:10B34800466AF1EE10FA48BFF0EE456A072AC3EDE7
:10B35800066A3FF470ADD1ED1E6A66EEE55AE5EE79
:10B36800877AF4EEE74A77EEC67AF1EE10FAC8BFAC
:10B37800F0EE457AC3ED077A5DE5734BC7ED00BA89
:10B388001B689342BFF6B6A8704B1A88002384F84E
:10B398006431002A41F011846D4A6E4B11781868A7
:10B3A80081F00101F7F714F8FFF7ACB86A4EDFF83F
:10B3B800E08106F5F47506F51577F6EC017A9BED54
:10B3C800080ADBF81432F8EEE77A284627EE800AF6
:10B3D8009847A5F1E000DBF834319847A5F17000F3
:10B3E800DBF8A4319847D6F8F400DBF8B830984772
:10B3F8002435AF42A8EC010ADFD1FEF74BBF4E4916
:10B408000978C80703D45549098BA4F88811544909
:10B418005448098890ED037A07EE901AF8EEE77A17
:10B42800B4EEE77AF1EE10FA40F208864E4800884A
:10B4380007EE900AF8EEE77AB4EEE77AF1EE10FA42
:10B44800C0F2CC8549484A49D0ED006A91ED006ABE
:10B458004848C4ED636ABCEEC75A76EE665A15EEE4
:10B46800101AC4ED616AC4ED605A84ED646AA4F8E8
:10B4780088110121D0ED006A84F8941177EE677A7B
:10B48800FFF73AB93C4B93ED005AB5EEC05AF1EECE
:10B4980010FA40F30783394BD3ED004AF5EEC04A62
:10B4A800F1EE10FA40F3FE8234EEC77A66EEE95AFE
:10B4B80087EE246AC5EE856AB7EE007AB4EEC76AED
:10B4C800F1EE10FA88BFB0EE476AB5EEC06AF1EE49
:10B4D80010FA76EE876AB8BFB0EE6B6A66EE266A37
:10B4E800FAE5274A92ED007AF0EEE76AF4EEC76AC9
:10B4F800F1EE10FA7FF790A8224A92ED007AF0EE6A
:10B50800CD6AF4EEC76AF1EE10FA7FF785A81E4AF5
:10B5180099ED007AD2ED006AB0EEC77AB4EEE67A19
:10B52800F1EE10FA7FF578A801220399C4F86811A2
:10B5380084F86421FFF774B8D2350020842F0020E6
:10B54800A82F002060320020F457002060620020FD
:10B558006262002064620020104B0020304F0020FF
:10B5680040300020F4500020423000202C300020D1
:10B578002830002048300020D4570020DC57002015
:10B5880008580020045800200C5800201D500020A6
:10B59800684D00200299724BD1ED017A93ED007A43
:10B5A800F0EEE77AF4EEC77AF1EE10FA7EF5AAAF7C
:10B5B800D1ED027AF0EEE77AB4EEE77AF1EE10FA1E
:10B5C8007EF7A0AFD1ED037AF0EEE77AB4EEE77A32
:10B5D800F1EE10FA7EF796AF624B1B689A077FF57B
:10B5E800D3AE6149614BB3F90C20B1F900E0604872
:10B5F800AEEB020E00688EEAEE72A2EBEE728242A9
:10B60800BEF680AFB3F90E30B1F90220D21A82EA41
:10B61800E273A3EBE27398427EF774AFB4E6554B3E
:10B6280099ED007AD3ED006AB0EEC77AB4EEE67A07
:10B63800F1EE10FA7FF706A8FFF701B807EE103A07
:10B648004D4BDFF840811B78C4F81061B8EEC77A1B
:10B65800F7EE006A132B86EE879AB8F90400B4F85F
:10B6680014519BED080A01F03482444B444A93ED8F
:10B67800001A93ED053A93ED122A93ED176AD3ED6C
:10B68800091A93ED0E4AD3ED015AD3ED063A93ED1C
:10B698000A7A93ED0F5AD3ED132AD3ED186AD3ED36
:10B6A800044AD3ED030A67EE897A69EE288A29EEFF
:10B6B800088AA1EE273A02EB85060021A2EE286A45
:10B6C800C4F80411C4F80811A1EE884AE5EEA73AB7
:10B6D800A7EE085A93ED167AD3ED0D5A93ED021A98
:10B6E800D3ED0C1A86ED003AE2EEA86A64EEC34A7E
:10B6F80027EE467A93ED0B2AD3ED152A86ED204ADC
:10B70800E0EEC33A65EEC45A93ED143AC3ED053A38
:10B71800E1EE274AF0EE477AA1EEC45AE2EE085A63
:10B72800E2EEC66AE3EE287AC3ED064A83ED0E5AC6
:10B73800C3ED0F5A86ED406AC3ED176AC3ED187A58
:10B74800C4F80C11013505F01F05A4F81451A8F828
:10B758000400FEF782BCB0EE465AFFF706B800BFF9
:10B768000058002070360020CC36002028440020E5
:10B77800FC5700200C5800203C5000202843002093
:10B78800A440002040500020B94B1B78192B07D843
:10B798000121B84A01FA03F31A40002A41F07484DF
:10B7A800B54BB64EB64F01931B689D061CD5FB7A68
:10B7B800FF2B04D0B34A12789A4201F2EF80B7F90E
:10B7C8000880FB7DA6F80080FF2B04D0AD4A1278D4
:10B7D8009A4201F2DE80B7F91450758008201FF0F4
:10B7E800E9FE002840F03186B7F90600B6F900C036
:10B7F800B6F902E0B7F91210B7F91E20B6F90450ED
:10B80800B7F90430B6F906806045A8BF60467145AF
:10B81800A8BF7146AA42A8BF2A469C45A8BF0346AE
:10B828003380B7F91030B6F908009E45B8BF1946FD
:10B83800B7F92A307180B7F91C10B7F934E04345DD
:10B84800A8BF43468D42B4BF0D461546B7F936200A
:10B85800B580B7F92850B6F90A108242A8BF024647
:10B86800A845ACBF9846A846B7F94230B6F90C507F
:10B87800A6F806808B42A8BF0B467045ACBF1046A1
:10B888007046B7F94E203081B7F94000B6F90EE09E
:10B89800AA42A8BF2A468842C8BF0346B7F95A0039
:10B8A800B7F94C1073817045B7F95830764FA8BF77
:10B8B80070469E45A8BF0346A942D8BF1146B1812C
:10B8C800F381BB892BB3DFF8D081DFF8D0A1DFF893
:10B8D800B09108F11005B8F9023000EE103A504660
:10B8E800B8EEC00AF4F73EFE22F04CF9B9F904307C
:10B8F800B9F9062000B298420AF1240A09F10C09A4
:10B9080003DB82421346A8BF034628F8023FA84536
:10B91800E1D1574B1B78013B182B72D8DFE813F0A5
:10B928005F007100710019007100710071007808E2
:10B938007100710071007100710098087100710048
:10B948007100710071001900860871007100980873
:10B958005F004E4BB6F908101A6802B111609B6976
:10B96800B6F90A2003B11A60019B1B689A0601F117
:10B97800E98602220492D9027FF562AAFE7B112E83
:10B988003FF65EAA424B079333F91630DDF8108074
:10B9980000EE103A4046B8EEC00A751C1FF0F4F9E4
:10B9A80006F10E074346EDB29E1BFFB2DDF81C9070
:10B9B80000E0454605F10108A819122D5FFA88F83C
:10B9C800C0B23FF43DAA39F9153000EE103AB8EE8E
:10B9D800C00A1FF0D9F9B845EBD1FFF731BABB7BE4
:10B9E800002B42F079802B4B1B7813F0010342F0B7
:10B9F8007380264A1268002A02F04D8413600123DE
:10BA08000493019B1B68980603D4194A1278052AE7
:10BA1800B1D1049A13460233551CDBB21046EDB27D
:10BA28000493B6F9003000EE103AB8EEC00A1FF0E1
:10BA3800ABF9B6F9023000EE103A2846B8EEC00A63
:10BA48001FF0A2F9019B1B6895E722F09BF829F8E3
:10BA58001600FEF70DBC95ED007A0BEB4602B8EE2A
:10BA6800C78A928F29F8162028EE278AFEF7DEBBB0
:10BA7800D456002032413003744D0020503200204B
:10BA8800845800203437002080440020904400204F
:10BA9800D86E0020D23500204E320020CC54002031
:10BAA800000000005FED026AFFF724BB59023FF572
:10BAB80067A8FFF769B8F5F7D5FAA94B059A1B7877
:10BAC800DFF8A082801A012BA8F8020000F0758226
:10BAD800072B7EF4DFADF5F7C5FA0290FEF7DCBD63
:10BAE800F5F7C0FA029A9F4B801AD880FFF7C3B9BE
:10BAF800002F41F0618191ED006A9DED0A5A9A4B41
:10BB080025EE866AA5EE076AB0EE675AA6EE265AB3
:10BB1800BDEEC56A16EE107A16EE106AAF42A8BFDF
:10BB28002E46B842C8BF064606EE106AB8EEC66A88
:10BB3800012A83ED006A3FF479A991ED046A9DED2D
:10BB48000B5A25EE866AA5EE076AB0EE675AA6EE8E
:10BB5800265ABDEEC56A16EE107A16EE106AAF4286
:10BB6800A8BF2E46B842C8BF064606EE106AB8EE11
:10BB7800C66A022A83ED016A3FF458A991ED086A62
:10BB88009DED0C5A25EE866AA5EE076AB0EE675A57
:10BB9800A6EE265ABDEEC56A16EE107A16EE106AA3
:10BBA800AF42A8BF2E46B842C8BF064606EE106A86
:10BBB800B8EEC66A032A83ED026A3FF437A991ED0D
:10BBC8000C6A9DED0D5A25EE866AA5EE076AB0EE61
:10BBD800675AA6EE265ABDEEC56A16EE107A16EE1C
:10BBE800106AAF42A8BF2E46B842C8BF064606EE46
:10BBF800106AB8EEC66A042A83ED036A3FF416A9F0
:10BC080091ED106A9DED0E5A25EE866AA5EE076A3B
:10BC1800B0EE675AA6EE265ABDEEC56A16EE107A41
:10BC280016EE106AAF42A8BF2E46B842C8BF0646F5
:10BC380006EE106AB8EEC66A052A83ED046A3FF478
:10BC4800F5A891ED146A9DED0F5A25EE866AA5EECA
:10BC5800076AB0EE675AA6EE265ABDEEC56A16EE1A
:10BC6800107A16EE106AAF42A8BF2E46B842C8BF77
:10BC7800064606EE106AB8EEC66A062A83ED056A1D
:10BC88003FF4D4A891ED186A9DED105A25EE866A06
:10BC9800A5EE076AB0EE675AA6EE265ABDEEC56A4B
:10BCA80016EE107A16EE106AAF42A8BF2E46B842BA
:10BCB800C8BF064606EE106AB8EEC66A072A83EDC4
:10BCC800066A3FF4B3A891ED1C6A9DED115A65EE22
:10BCD800865AE7EE055AE6EEA57AFDEEE77A17EE04
:10BCE800901A8D42A8BF0D468842C8BF054607EE88
:10BCF800905AF8EEE77AC3ED077AFFF796B81B4A31
:10BD0800517900293EF4BDAD1949097800293EF45E
:10BD1800B8AD1278DFED174A07EE902A164AB8EE4A
:10BD2800677A128807EE901A06EE902AF8EEE77AFC
:10BD3800F8EE666A67EE277AB7EE007AC7EEA63A9B
:10BD4800F4EEE43AF1EE10FA88BFF0EE643AF4EE5D
:10BD5800C73AF1EE10FAB8BFF0EE473AFEF793BDD6
:10BD68003C5000204050002060320020E036002087
:10BD7800F2500020713DAA3FCC500020002E00F068
:10BD88005482002F41F0D286C049BEF1000F41F025
:10BD98000F8591ED006ADDED0A4ABD4B25EE866AF6
:10BDA800BDEEC55AA4EE876A15EE100AB0EE675AC2
:10BDB800A6EE265ABDEEC56A16EE107A16EE106A81
:10BDC800AF42A8BF2E46B842C8BF064606EE106A64
:10BDD800B8EEC66A012A83ED006A3FF427A891ED00
:10BDE800046A9DED0B5A25EE866AA5EE076AB0EE49
:10BDF800675AA6EE265ABDEEC56A16EE107A16EEFA
:10BE0800106AAF42A8BF2E468742B8BF064606EE64
:10BE1800106AB8EEC66A022A83ED016A3FF406A8E2
:10BE280091ED086A9DED0C5A25EE866AA5EE076A23
:10BE3800B0EE675AA6EE265ABDEEC56A16EE107A1F
:10BE480016EE106AAF42A8BF2E468742B8BF064614
:10BE580006EE106AB8EEC66A032A83ED026A3EF45B
:10BE6800E5AF91ED0C6A9DED0D5A25EE866AA5EEBB
:10BE7800076AB0EE675AA6EE265ABDEEC56A16EEF8
:10BE8800107A16EE106AAF42A8BF2E468742B8BF96
:10BE9800064606EE106AB8EEC66A042A83ED036AFF
:10BEA8003EF4C4AF91ED106A9DED0E5A25EE866AF8
:10BEB800A5EE076AB0EE675AA6EE265ABDEEC56A29
:10BEC80016EE107A16EE106AAF42A8BF2E468742C9
:10BED800B8BF064606EE106AB8EEC66A052A83EDB4
:10BEE800046A3EF4A3AF91ED146A9DED0F5A25EE56
:10BEF800866AA5EE076AB0EE675AA6EE265ABDEE28
:10BF0800C56A16EE107A16EE106AAF42A8BF2E4622
:10BF18008742B8BF064606EE106AB8EEC66A062A19
:10BF280083ED056A3EF482AF91ED186A9DED105AD3
:10BF380025EE866AA5EE076AB0EE675AA6EE265A7F
:10BF4800BDEEC56A16EE107A16EE106AAF42A8BFAB
:10BF58002E468742B8BF064606EE106AB8EEC66A95
:10BF6800072A83ED066A3EF461AF91ED1C6A9DEDE8
:10BF7800115A65EE865AE7EE055AE6EEA57AFDEE09
:10BF8800E77A17EE901A8D42A8BF0D468842D8BFAF
:10BF9800284607EE900AF8EEE77AC3ED077AFEF72F
:10BFA80044BF3C4B93ED006AFFF786B8F5F75AF8A3
:10BFB8000590FEF789B9DFF81081F5F753F8364A8E
:10BFC800D4F8783112680290C31A9A1AC4F8780122
:10BFD800A8F80430A8F80620FEF75EBBB4F888017C
:10BFE800884240F245852D482D49D0ED007A91EDE3
:10BFF800007A2C48C4ED637A77EE676AC4ED617AFB
:10C008000121C4ED606A84ED647AD0ED006ADFED49
:10C01800267A84F89411FEF76FBB244B1B88002BFB
:10C0280040F04585224A234B11781868F6F7D0F975
:10C03800D4F86821039B9A1AFEF733BA1E491F48A1
:10C04800D1ED006A1E4990ED006A0978C4ED636A73
:10C0580084ED646A002940F0B78476EEC65AF0EEA3
:10C06800466ABCEEC76A1748C4ED605A16EE101A45
:10C07800C4ED616AA4F88811FF21D0ED006A84F844
:10C08800941177EEC77AFEF737BB00BFA82F0020C0
:10C0980060320020D45700201C3400202C300020AF
:10C0A8002830002048300020000000006062002096
:10C0B8006262002064620020883200203030002054
:10C0C8006C4700204430002040500020D1ED015A38
:10C0D80065EEC65AB0EE674AA5EE874AB4EEE44A62
:10C0E80074EE665AF1EE10FA48BFF0EE455A012A8E
:10C0F800C3ED005A3EF49FAED1ED055A65EEC65A1F
:10C10800B0EE674AA5EE874AB4EEE44A74EE665A82
:10C11800F1EE10FA48BFF0EE455A022AC3ED015A73
:10C128003EF489AED1ED095A65EEC65AB0EE674ABB
:10C13800A5EE874AB4EEE44A74EE665AF1EE10FAB8
:10C1480048BFF0EE455A032AC3ED025A3EF473AED7
:10C15800D1ED0D5A65EEC65AB0EE674AA5EE874A8C
:10C16800B4EEE44A74EE665AF1EE10FA48BFF0EE07
:10C17800455A042AC3ED035A3EF45DAED1ED115A77
:10C1880065EEC65AB0EE674AA5EE874AB4EEE44AB1
:10C1980074EE665AF1EE10FA48BFF0EE455A052AD9
:10C1A800C3ED045A3EF447AED1ED155A65EEC65AB2
:10C1B800B0EE674AA5EE874AB4EEE44A74EE666AC2
:10C1C800F1EE10FA48BFF0EE456A062AC3ED056A9B
:10C1D8003EF431AED1ED196A66EEC66AB0EE674A32
:10C1E800A6EE874AF3EE045AB4EEE44A74EE656AA2
:10C1F800F1EE10FA48BFF0EE456A072AC3ED066A69
:10C208003EF419AED1ED1D6A26EEC66AE6EE077A4F
:10C21800F4EEE47A77EEE57AF1EE10FAB8BFF0EED4
:10C22800457AC3ED077AFEF706BEC949BEF1000F8D
:10C2380041F04A8191ED006ADDED0A4AC54B25EED1
:10C24800866ABDEEC55AA4EE876A15EE100AB0EEEE
:10C25800675AA6EE265ABDEEC56A16EE10EA16EE25
:10C26800106AAE45A8BF2E467045C8BF064606EE02
:10C27800106AB8EEC66A012A83ED006A3EF4D4ADAE
:10C2880091ED046A9DED0B5A25EE866AA5EE076AC4
:10C29800B0EE675AA6EE265ABDEEC56A16EE10EA4B
:10C2A80016EE106AAE45A8BF2E468645B8BF0646AC
:10C2B80006EE106AB8EEC66A022A83ED016A3EF4F9
:10C2C800B3AD91ED086A9DED0C5A25EE866AA5EE90
:10C2D800076AB0EE675AA6EE265ABDEEC56A16EE94
:10C2E80010EA16EE106AAE45A8BF2E468645B8BFBE
:10C2F800064606EE106AB8EEC66A032A83ED026A9D
:10C308003EF492AD91ED0C6A9DED0D5A25EE866ACC
:10C31800A5EE076AB0EE675AA6EE265ABDEEC56AC4
:10C3280016EE10EA16EE106AAE45A8BF2E468645F0
:10C33800B8BF064606EE106AB8EEC66A042A83ED50
:10C34800036A3EF471AD91ED106A9DED0E5A25EE2B
:10C35800866AA5EE076AB0EE675AA6EE265ABDEEC3
:10C36800C56A16EE10EA16EE106AAE45A8BF2E464C
:10C378008645B8BF064606EE106AB8EEC66A052AB4
:10C3880083ED046A3EF450AD91ED146A9DED0F5AA9
:10C3980025EE866AA5EE076AB0EE675AA6EE265A1B
:10C3A800BDEEC56A16EE10EA16EE106AAE45A8BFD5
:10C3B8002E468645B8BF064606EE106AB8EEC66A2F
:10C3C800062A83ED056A3EF42FAD91ED186A9DEDBE
:10C3D800105A25EE866AA5EE076AB0EE675AA6EEF1
:10C3E800265ABDEEC56A16EE10EA16EE106AAE457C
:10C3F800A8BF2E468645B8BF064606EE106AB8EEB8
:10C40800C66A072A83ED066A3EF40EAD91ED1C6AF2
:10C418009DED115A65EE865AE7EE055AE6EEA57AC5
:10C42800FDEEE77A17EE901A8D42A8BF0D468842B6
:10C43800D8BF284607EE900AF8EEE77AC3ED077AE8
:10C44800002F7EF4F8ACFEF7F0BC94F8BC31012B59
:10C4580001F0A184404B97F916005A8897F90AE031
:10C468001B883E4910FB03F31EFB02F281FB020C02
:10C4780081FB0301D217DB17C2EB2C12C3EB21138C
:10C4880042441D4432807580FFF7AEB9344FD4ED75
:10C49800017A94ED006A38887B6977EEA77AF0EE26
:10C4A800006AB0EE677AA6EE267A013804EBC0027D
:10C4B800D6EE267A083A1033F6EE003A27EE237ABB
:10C4C80067EEA37A84ED207AC4ED217A254C2746BD
:10C4D80004F1800192ED027A92ED036AD7ED036AC6
:10C4E800D7ED027A53ED014A13ED025A37EE674A47
:10C4F80076EEC65A77EE277AE4EE845A0138A2F12E
:10C508000802E5EE047A07F1080703F1080336EE9E
:10C51800267A01F10801E4EE877AE5EE475A67EEDC
:10C52800A37A25EEA37AC1ED007A81ED017AD1D103
:10C53800142E7DF446AEF4F795FD029BDFF82880B3
:10C54800C01AA8F80200D4F81851FDF73ABE00BF87
:10C55800A82F002060320020CC3600201F85EB5128
:10C568008C4000207C21002040500020DFF894946B
:10C5780099F80020900801F08986DFF88CE400F132
:10C58800010C4FEA4C1C0EEB0C070EF12003AEF128
:10C59800700113ED076A53ED056A13ED037A53ED45
:10C5A800017A53ED025A13ED084A53ED064A13ED8A
:10C5B800045A26EE066A66EEA66A27EE077A67EE42
:10C5C800A77AA4EE046A20339F42E4EEA46A01F13C
:10C5D8001001A5EE057AE5EEA57AF1EEC65AB1EEA0
:10C5E800E66AF1EEC76AB1EEE77A41ED085A01ED65
:10C5F800076A41ED066A01ED057ACAD1ACF1200C53
:10C60800E64404EB001012F0030318BF0EF1080E05
:10C618000FD05EED017A1EED027A67EEA77A013B34
:10C62800E7EE077A0EF1080EB1EEE77AA0EC017A90
:10C63800EFD1142E01F00C860135C4F81851FDF71E
:10C648002DBDE34FE348BA68B98920F0BFF9E24B42
:10C658001E78142E01F07885D4F818510135C4F8E5
:10C66800185114E7DA4FB7F800E0D7F804C04FEADA
:10C678005E084FEA880204EB8E055FEADE0E04EBE3
:10C68800020300F0A08010320EF1010ED34803EB34
:10C698000E1E2A4410330CF1100605F1100151ED5D
:10C6A800032A51ED043A10ED043A10ED032A51ED36
:10C6B800026A11ED016A50ED020A10ED010A12ED4D
:10C6C800044A12ED035A53ED044A53ED035A13ED8D
:10C6D800027A53ED017A12ED021A52ED011A73EE45
:10C6E800238A32EE228A40ED048A00ED038A70EE36
:10C6F800A68A30EE068A40ED028A00ED018A74EEC1
:10C70800848A35EE858A43ED048A03ED038A77EE41
:10C71800018A37EEA18A43ED028A03ED018A73EE9E
:10C72800633A75EE655A16ED035A32EE623A74EEC4
:10C73800644A25EE638A16ED044A23EE052A64EE60
:10C74800652AA3EE048A10339E4524EE843AA3EEAC
:10C75800842A00F1100006F11006A5EE853A01F1D1
:10C76800100102F11002E4EE852A01ED078A01EDBD
:10C77800082A02ED073A42ED082A56ED055A16ED49
:10C78800065A70EEE66A30EE466A31EE477A71EE86
:10C79800E77A26EE253A65EEE63A25EE674A67EE31
:10C7A800054AE6EE053AA6EE853AA7EE254AE7EEF3
:10C7B800A54A01ED063A41ED053A02ED064A42ED79
:10C7C800054A7FF46CAF1FFA88F8624641468148F3
:10C7D80013F058FE41467A68284613F053FE7E4B04
:10C7E8001B78142B7FF4AFAEA5E6D4F81CC1B4F8BF
:10C7F80014917B4BC9F120085FFA88F809EB4C17B4
:10C8080003EB87075FEA980301F08484013318017A
:10C818007449724A07EB000E07F1100313ED024A40
:10C8280013ED035A13ED016A13ED047A51ED024A30
:10C8380051ED035A51ED016A51ED047A64EE244A30
:10C8480065EE255A66EE266A67EE277A10339E450E
:10C8580042ED024A42ED035A42ED016A42ED047A82
:10C8680001F1100102F11002D8D15F49A0F11002C4
:10C87800174401EB020E224418F0030309D0B7EC69
:10C88800017AFEEC017A67EE277A013BE2EC017A45
:10C89800F5D1B9F1000F41F0C980142E7DF491ACA7
:10C8A800F4F7E0FB029BDFF86481D4F81851C01A52
:10C8B800A8F80200FDF785BCD4F81C714B4B4C4A14
:10C8C800DFED4C7AD2ED008A4B4AF9000B44F8EEC2
:10C8D800688A9B8809EE103A643BC82BA8BFC82316
:10C8E80068EEA78AF8EE497A782BB8BF782368EE05
:10C8F800A78A07EE903A3944B0EE680A02EB81083D
:10C90800B8EEE78A21F08AF9B8EEC99AF0EE409AB3
:10C91800B0EE680A21F0E4F838EE097A79EE487A40
:10C9280028EE098A67EE877AB7EE006A88EE277ADA
:10C93800142EF8EE007A77EE076A60EE277A89EE11
:10C94800A67A77EE065A36EE477AC6EE256A67EE7D
:10C95800A67A27EE267AC8ED006A88ED047AC8ED33
:10C96800026AC8ED017AC8ED037A01F06384234BAB
:10C97800194A013783FB073CACEBE77C0CEB4C0C0A
:10C988000135A7EB0C0C1678C4F81851C4F81CC173
:10C998002DE71B4A32F91350FEF71FBF184A32F928
:10C9A8001380FEF70EBFF4F75DFB0B4B02901E7869
:10C9B800142E05BFDFF85480D4F81851D4F8185154
:10C9C800A8F80050FDF752BB76EE665AFFF749BB50
:10C9D8008C4000207C2100203C5000208C2100202D
:10C9E800A44000203442002024420020A442002019
:10C9F800644D002027D4D236F84C002056555555A2
:10CA0800D86E002086400020FC21002040500020E5
:10CA1800D54BB6F906101A6802B111609B69B6F9D0
:10CA28000820002B7EF49FAFFEF79EBFDFF88083BF
:10CA3800002538F9023B00EE103AE8B2B8EEC00A19
:10CA480001351EF0A1F9042DF3D10495FEF7D9BFE5
:10CA5800DFF86083002538F9023F00EE103AE8B2AB
:10CA6800B8EEC00A01351EF08FF9062DF3D1ECE7B8
:10CA7800BE49BF48D1ED007ABE4990ED007A0978E9
:10CA8800C4ED637A84ED647A002901F0CB8277EEF5
:10CA9800676AB948C4ED617AC4ED606AFF21D0EDD8
:10CAA800006ADFEDB67A84F89411FDF725BEB44923
:10CAB8004B69002B3DF4F5ACB248B34B008893FBAF
:10CAC800F0F00B684FF0010E186081F811E0FDF7E7
:10CAD800E8BCAE4EAE4F96ED004A96ED057AD6ED1F
:10CAE800014A96ED066AD6ED046A96ED035AD6ED2C
:10CAF800025A67EE897A07EB8503A4EE277AA4EE3B
:10CB0800A76A66EEC76AA5EE476AE5EEA76A20EE51
:10CB1800070A86ED056AC6ED066A83ED007A29EEF6
:10CB2800088A21F02FF869EE288AD6ED0E5AD6ED3C
:10CB3800176A96ED091AD6ED121A96ED0F5A96ED68
:10CB4800187A96ED0A2AD6ED132A96ED0D6AD6EDD7
:10CB5800167A96ED0C3AD6ED0B3A96ED154AD6EDC7
:10CB6800144AE1EE085A002207EB8503E8EEA16AB1
:10CB780000B2C4F80421A2EE085AC4F80821C4F887
:10CB88000C21A8EEA27A26EE656A67EEE67AA3EE95
:10CB9800655AA3EE886AA6EEC47AE8EEA47A86ED12
:10CBA8000E5AC3ED205A86ED0F6AC3ED406A86ED32
:10CBB800177AC6ED187AFEF7C5BD71494A69002A89
:10CBC8003DF4A0AC0A6813604B74FDF79BBCBBF93D
:10CBD8003C30CBF8242007EE903A0122F8EEE77AB1
:10CBE800CBF86C30CBF888200023012ECBED1F7AD0
:10CBF800CBED1E7ACBF8803001F07682AE427EF41F
:10CC080093A9BBF93E30CBF8703007EE903A00227A
:10CC18000123F8EEE77ACBF82820CBF89C300023E4
:10CC2800012ECBED247ACBED237ACBF8943001F0AA
:10CC38005F82AE427EF4AAA9BBF94030CBF87430CB
:10CC480007EE903A00220123F8EEE77ACBF82C2081
:10CC5800CBF8B0300023012ECBED297ACBED287A22
:10CC6800CBF8A8307EF4C4A99FED448A032F39D0AD
:10CC7800B9F1000F09D007EE909AF8EEE77AF4EED2
:10CC8800C87AF1EE10FA01F10A83424ADBF87430EF
:10CC9800126894F82011A8F8060003EB550393FBDB
:10CCA800F5F50023CBF82C5093621363D36231B1AE
:10CCB800394B1B8823F40063002B7EF49BA9374B68
:10CCC8001B6813F4003341F0078235491A46C85CE3
:10CCD800012803F10C0300F042850132152AF6D130
:10CCE800FEF788B9B0EE480A20F04CFF00B2BFE763
:10CCF8002C4B187800F00107002F7EF49CA8FEF753
:10CD080094B82949DFED297A0968C4ED4C7A11F005
:10CD1800805840F03C8513F4800800F0DA824FF028
:10CD28000008B6EE007A67EE877AF4EEE75AF1EE7D
:10CD380010FA48BFF0EE675A40F12985C4ED665AEB
:10CD4800FDF722BF74EE677AB7EE007AF4EEC77A81
:10CD5800F1EE10FAC4ED4C7A41F36A8184EEA77AB9
:10CD68008DED0A7AFDF706BF904400208832002036
:10CD7800303000206C4700204430002000000000C4
:10CD8800686200208062002020A10700284300205C
:10CD9800A44000205C3B0020143700205C2E0020BB
:10CDA80058070308D2350020F43100200000008025
:10CDB8005632002052320020BCF1000F01F01680DC
:10CDC80091ED006A9DED0A5AAE4B25EE866AA5EEF6
:10CDD800076AB0EE675AA6EE265ABDEEC56A16EE89
:10CDE800107A16EE106AAF42A8BF2E46B842C8BFE6
:10CDF800064606EE106AB8EEC66A012A83ED006A96
:10CE08003EF419A891ED046A9DED0B5A25EE866A49
:10CE1800A5EE076AB0EE675AA6EE265ABDEEC56AB9
:10CE280016EE107A16EE106AAF42A8BF2E46B84228
:10CE3800C8BF064606EE106AB8EEC66A022A83ED37
:10CE4800016A3DF4F8AF91ED086A9DED0C5A25EEA4
:10CE5800866AA5EE076AB0EE675AA6EE265ABDEEB8
:10CE6800C56A16EE107A16EE106AAF42A8BF2E46B3
:10CE7800B842C8BF064606EE106AB8EEC66A032A6C
:10CE880083ED026A3DF4D7AF91ED0C6A9DED0D5A22
:10CE980025EE866AA5EE076AB0EE675AA6EE265A10
:10CEA800BDEEC56A16EE107A16EE106AAF42A8BF3C
:10CEB8002E46B842C8BF064606EE106AB8EEC66AE5
:10CEC800042A83ED036A3DF4B6AF91ED106A9DED37
:10CED8000E5A25EE866AA5EE076AB0EE675AA6EEE8
:10CEE800265ABDEEC56A16EE107A16EE106AAF42E3
:10CEF800A8BF2E46B842C8BF064606EE106AB8EE6E
:10CF0800C66A052A83ED046A3DF495AF91ED146A6B
:10CF18009DED0F5A25EE866AA5EE076AB0EE675AB0
:10CF2800A6EE265ABDEEC56A16EE107A16EE106AFF
:10CF3800AF42A8BF2E46B842C8BF064606EE106AE2
:10CF4800B8EEC66A062A83ED056A3DF474AF91ED22
:10CF5800186A9DED105A25EE866AA5EE076AB0EEAE
:10CF6800675AA6EE265ABDEEC56A16EE107A16EE78
:10CF7800106AAF42A8BF2E46B842C8BF064606EEA2
:10CF8800106AB8EEC66A072A83ED066A3DF453AF05
:10CF980091ED1C6A9DED115A65EE865AE7EE055A29
:10CFA800E5EEA67AFDEEE77A17EE902A9542A8BF3D
:10CFB80015469042D8BF284607EE900AF8EEE77A61
:10CFC800C3ED077AFDF737BF012A41F38D8007EEDD
:10CFD800101AB8EEC77AC7EE876AB1EEE68A032F51
:10CFE80015D0B9F1000F09D007EE909AF8EEE77A5C
:10CFF800F4EEC87AF1EE10FA01F15181DBF86C30E9
:10D0080003EB550393FBF5F3CBF82430F6E5B0EECC
:10D01800480A20F0B7FD00B2E3E7012A41F368802F
:10D0280007EE101AB8EEC77AC7EE876AB1EEE68A3D
:10D03800032F15D0B9F1000F09D007EE909AF8EE3A
:10D04800E77AF4EEC87AF1EE10FA01F12881DBF8FC
:10D05800703003EB550393FBF5F3CBF82830E8E584
:10D06800B0EE480A20F08EFD00B2E3E7012A7FF710
:10D07800FBAD07EE101AB8EEC77AC7EE876AB1EEB5
:10D08800E68AF3E560320020974B1B88DF0540F104
:10D09800D787964B964A93ED017AD3ED006AD3ED84
:10D0A800027A944B0793BDEEC77AB3F906E0924B28
:10D0B8000193FDEEE66A17EE103AFDEEE77A118B62
:10D0C800ADF82A3016EE902A17EE903AADF82820DF
:10D0D800ADF82C30894A8A48B2F90230B2F90020FA
:10D0E800884DD0ED007A9FED887A88484FF47A769B
:10D0F80003F5E16306FB03F302F5E16206FB02F2C6
:10D1080085FB03761E44DB1785FB0275C3EBE6231C
:10D1180077EEC77A079E0078378806901544D217AD
:10D128003046C2EBE522FDEEE77A35467688AD88D3
:10D138008446A3F5FA73761A0089ADF8403017EEE5
:10D14800903AA2F5FA72ADF83260BCF80E60ADF80C
:10D1580042206D1A401ABCF80A20ADF82E30BCF8EF
:10D168000C30ADF83450ADF83800751A0698684E92
:10D17800ADF83E50AEEB010E7F1A521A5B1A002131
:10D18800ADF836E0ADF83070ADF83A20ADF83C3087
:10D1980031607160B160F160002801F0CD805D4BB5
:10D1A800DFF87C815C4FCDF820B08A469946099417
:10D1B8003CE012AB03EB440030F9200CA9F8000066
:10D1C80098F902E001230D4403FA04F4534B57F88D
:10D1D80025501EFB00F083FB003EC017039B2C422A
:10D1E800C0EB6E100CBF01244FF0FF3498420EDBE9
:10D1F800059B02FB03F2494B83FB0253D217C2EB98
:10D208006313A3EB0C031BB28342A8BF034636F893
:10D21800112003FB042326F81130069B0AF1010AAA
:10D228009A4508F1070809F102097BDA98F806001F
:10D23800002837D198F8001098F9052005924D007C
:10D24800681807EB800098F90430C288808898F83D
:10D2580003E098F80140121A92B2304802FB03F337
:10D2680080FB03C0DB17C3EB60134FEA520CA3EB40
:10D278000C031BB20393BEF1000F9AD012AB03EB61
:10D28800440BB9F900003BF920BC584513DA864431
:10D29800704503DCF3455846A8BF704600B2A9F8AC
:10D2A80000008DE71630C0B21EF084F90028C1D105
:10D2B800A9F80000B1E783DDA0EB0E0EDE4503DB25
:10D2C8007045A8BF704683460FFA8BF0A9F8000096
:10D2D80076E7B6EE007AF4EEC75AF1EE10FA3FF7A9
:10D2E80020ADFDF751BC00BF26390020F4500020C6
:10D2F800304F0020D86E0020744D0020CC3600201E
:10D3080060320020C5B3A2910080BB445C56002067
:10D318005032002018230020845800201F85EB512C
:10D3280060560020DDF820B0099C97F90A00338880
:10D33800634A644910FB03F3F87A097882FB0352C5
:10D34800FF284FEAE373C3EB621200F0E6838142E1
:10D3580040F2E383079B33F9100097F9165073885E
:10D3680010443080564AF87D15FB03F382FB0352C4
:10D37800FF284FEAE373C3EB621200F0CB838142CC
:10D3880040F2C883079B33F9100097F92250B388FD
:10D39800104470804A4A97F8230015FB03F382FB78
:10D3A8000352FF284FEAE373C3EB621200F0AF8326
:10D3B800814240F2AC83079B33F9100097F92E5055
:10D3C800F3881044B0803E4A97F82F0015FB03F30A
:10D3D80082FB0352FF284FEAE373C3EB621200F0AB
:10D3E8009383814240F29083079B33F9100097F9A9
:10D3F8003A5033891044F080314A97F83B0015FBC6
:10D4080003F382FB0352FF284FEAE373C3EB621274
:10D4180000F07783814240F27483079B33F9100050
:10D4280097F94650738910443081254A97F8470088
:10D4380015FB03F382FB0352FF284FEAE373C3EBA8
:10D44800621200F05B83814240F25883079B33F9F4
:10D45800100097F95250B38910447081184A97F810
:10D46800530015FB03F382FB0352FF284FEAE373D3
:10D47800C3EB621200F03F83814240F23C83079B7A
:10D4880033F9100097F95E50F3891044B0810C4AC3
:10D4980097F85F0015FB03F382FB0352FF284FEA5E
:10D4A800E373C3EB621300F02383884280F0208388
:10D4B800079A32F910201344F381019BFEF774B9DF
:10D4C8001F85EB5134370020D1ED004A9DED0A4A03
:10D4D800B54B65EEA44AFDEEC53AE4EE074AB0EE58
:10D4E800674AA4EEA64A13EE900AB4EEC46AF1EEB7
:10D4F80010FAF0EE444A88BFF0EE454AFDEEE44AE1
:10D5080014EE90EA14EE906AAE45A8BF2E46704518
:10D51800C8BF064604EE906AF8EEE44A012AC3ED55
:10D52800004A3DF481ACD1ED044A9DED0B4A65EE0D
:10D53800A44AE4EE074AB0EE674AA4EEA64AB4EE5F
:10D54800C46AF1EE10FAF0EE444A88BFF0EE454A9C
:10D55800FDEEE44A14EE90EA14EE906AAE45A8BFD8
:10D568002E468645B8BF064604EE906AF8EEE44AB1
:10D57800022AC3ED014A3DF457ACD1ED084A9DEDAE
:10D588000C4A65EEA44AE4EE074AB0EE674AA4EEF8
:10D59800A64AB4EEC46AF1EE10FAF0EE444A88BF27
:10D5A800F0EE454AFDEEE44A14EE90EA14EE906A75
:10D5B800AE45A8BF2E468645B8BF064604EE906A1B
:10D5C800F8EEE44A032AC3ED024A3DF42DACD1ED4E
:10D5D8000C4A9DED0D4A65EEA44AE4EE074AB0EE0A
:10D5E800674AA4EEA64AB4EEC46AF1EE10FAF0EE69
:10D5F800444A88BFF0EE454AFDEEE44A14EE90EA4C
:10D6080014EE906AAE45A8BF2E468645B8BF0646BA
:10D6180004EE906AF8EEE44A042AC3ED034A3DF4A6
:10D6280003ACD1ED104A9DED0E4A65EEA44AE4EE36
:10D63800074AB0EE674AA4EEA64AB4EEC46AF1EE11
:10D6480010FAF0EE444A88BFF0EE454AFDEEE44A8F
:10D6580014EE90EA14EE906AAE45A8BF2E468645B1
:10D66800B8BF064604EE906AF8EEE44A052AC3ED10
:10D67800044A3DF4D9ABD1ED144A9DED0F4A65EE4D
:10D68800A44AE4EE074AB0EE674AA4EEA64AB4EE0E
:10D69800C46AF1EE10FAF0EE444A88BFF0EE454A4B
:10D6A800FDEEE44A14EE90EA14EE906AAE45A8BF87
:10D6B8002E468645B8BF064604EE906AF8EEE44A60
:10D6C800062AC3ED054A3DF4AFABD1ED184A9DEDEE
:10D6D800104A65EEA44AE4EE074AB0EE674AA4EEA3
:10D6E800A64AB4EEC46AF1EE10FAF0EE444A88BFD6
:10D6F800F0EE454AFDEEE44A14EE90EA14EE906A24
:10D70800AE45A8BF2E468645B8BF064604EE906AC9
:10D71800F8EEE44A072AC3ED064A3DF485ABD1ED9D
:10D728001C4A9DED114A65EEA45AE7EE045AE6EE4E
:10D73800A57AB4EEE76AF1EE10FAC8BFF0EE457AC2
:10D74800FEF76EBE0423032504930220FEF769B991
:10D758008223FCF724BDDFED157AFCF7ECBCD4F886
:10D76800245153003DB1981801EB80006D78407842
:10D77800A842BDF43FAC134401EB83010023C4F875
:10D788002411A4F8BE31C4F8C031FDF733BCB7EE9C
:10D79800007A77EE677AF4EEE75AF1EE10FA88BF6E
:10D7A800F0EE675AFFF7CABA603200200000024361
:10D7B800D1ED004A9DED0A4AD94B65EEA44AFDEE2B
:10D7C800C53AE4EE074AB0EE674AA4EEA64A13EE5D
:10D7D800900AB4EEC46AF1EE10FAF0EE444A88BF3B
:10D7E800F0EE454AFDEEE44A14EE907A14EE906AA3
:10D7F800AF42A8BF2E46B842C8BF064604EE906A9C
:10D80800F8EEE44A012AC3ED004A3DF40FABD1ED2E
:10D81800044A9DED0B4A65EEA44AE4EE074AB0EED1
:10D82800674AA4EEA64AB4EEC46AF1EE10FAF0EE26
:10D83800444A88BFF0EE454AFDEEE44A14EE907A79
:10D8480014EE906AAF42A8BF2E468742B8BF06467C
:10D8580004EE906AF8EEE44A022AC3ED014A3DF468
:10D86800E5AAD1ED084A9DED0C4A65EEA44AE4EE1E
:10D87800074AB0EE674AA4EEA64AB4EEC46AF1EECF
:10D8880010FAF0EE444A88BFF0EE454AFDEEE44A4D
:10D8980014EE907A14EE906AAF42A8BF2E468742E3
:10D8A800B8BF064604EE906AF8EEE44A032AC3EDD0
:10D8B800024A3DF4BBAAD1ED0C4A9DED0D4A65EE36
:10D8C800A44AE4EE074AB0EE674AA4EEA64AB4EECC
:10D8D800C46AF1EE10FAF0EE444A88BFF0EE454A09
:10D8E800FDEEE44A14EE907A14EE906AAF42A8BFB7
:10D8F8002E468742B8BF064604EE906AF8EEE44A20
:10D90800042AC3ED034A3DF491AAD1ED104A9DEDD6
:10D918000E4A65EEA44AE4EE074AB0EE674AA4EE62
:10D92800A64AB4EEC46AF1EE10FAF0EE444A88BF93
:10D93800F0EE454AFDEEE44A14EE907A14EE906A51
:10D94800AF42A8BF2E468742B8BF064604EE906A8B
:10D95800F8EEE44A052AC3ED044A3DF467AAD1ED7E
:10D96800144A9DED0F4A65EEA44AE4EE074AB0EE6C
:10D97800674AA4EEA64AB4EEC46AF1EE10FAF0EED5
:10D98800444A88BFF0EE454AFDEEE44A14EE907A28
:10D9980014EE906AAF42A8BF2E468742B8BF06462B
:10D9A80004EE906AF8EEE44A062AC3ED054A3DF40F
:10D9B8003DAAD1ED184A9DED104A65EEA44AE4EE61
:10D9C800074AB0EE674AA4EEA64AB4EEC46AF1EE7E
:10D9D80010FAF0EE444A88BFF0EE454AFDEEE44AFC
:10D9E80014EE907A14EE906AAF42A8BF2E46874292
:10D9F800B8BF064604EE906AF8EEE44A072AC3ED7B
:10DA0800064A3DF413AAD1ED1C4A9DED114A65EE74
:10DA1800A45AE7EE045AE6EEA57AB4EEE76AF1EE08
:10DA280010FAC8BFF0EE457AFEF7A9BA3D4B4FEAA7
:10DA380088075FEA990801EB070E03EBCC1C274423
:10DA480000F07D8408F101084FEA08180CEB080083
:10DA58000CF110030EF1100107F1100213ED024A48
:10DA680013ED035A13ED016A13ED047A51ED024ADE
:10DA780051ED035A51ED016A51ED047A64EE244ADE
:10DA880065EE255A66EE266A67EE277A10339842C5
:10DA980042ED024A42ED035A42ED016A42ED047A30
:10DAA80001F1100102F11002D8D1A8F11008C44404
:10DAB8000EEB0801474419F003093EF4EEAEBCEC46
:10DAC800017AF1EC017A67EE277AB9F10109E7ECFE
:10DAD800017AF4D1FEF7E1BE134BB6F90A201B68B0
:10DAE800002B00F0D8831A6001230493FDF789BF47
:10DAF800B7F95C20DFE4B7F95000C3E4B7F9440094
:10DB0800A7E4B7F938008BE4B7F92C006FE4B7F94C
:10DB1800200053E4B7F9140037E4B7F908001CE40F
:10DB280060320020A440002090440020BCF1000F87
:10DB380000F01683A9499DED0A4AD1ED004A65EE29
:10DB4800A44AE4EE074AB0EE674AA4EEA64AF0EE0D
:10DB5800444ABEF1000F06D0B4EE446AF1EE10FA62
:10DB6800C8BFF0EE454ABDEEC55A15EE106ABDEEC7
:10DB7800E45A04EE906A15EE103A9E4200F3D983F7
:10DB8800AB42A8BF2B4605EE103AB8EEC55A944BE7
:10DB9800012A83ED005A3DF44EA991ED045A9DEDFA
:10DBA8000B4A25EE855AA4EE075AB0EE674AA5EE51
:10DBB800264AB0EE445ABEF1000F00F0B083B4EE2E
:10DBC800C46AF1EE10FA40F3AA833046A842A8BF0F
:10DBD800284605EE100AB8EEC55A022A83ED015A06
:10DBE8003DF429A991ED085A9DED0C4A25EE855A78
:10DBF800A4EE075AB0EE674AA5EE264AB0EE445A9C
:10DC0800BEF1000F00F08183B4EEC46AF1EE10FAA1
:10DC180040F37B833046A842A8BF284605EE100A89
:10DC2800B8EEC55A032A83ED025A3DF404A991EDD2
:10DC38000C5A9DED0D4A25EE855AA4EE075AB0EE12
:10DC4800674AA5EE264AB0EE445ABEF1000F00F02E
:10DC58005283B4EEC46AF1EE10FA40F34C833046B6
:10DC6800A842A8BF284605EE100AB8EEC55A042AED
:10DC780083ED035A3DF4DFA891ED105A9DED0E4A4D
:10DC880025EE855AA4EE075AB0EE674AA5EE264A55
:10DC9800B0EE445ABEF1000F00F02383B4EEC46A1C
:10DCA800F1EE10FA40F31D833046A842A8BF28467B
:10DCB80005EE100AB8EEC55A052A83ED045A3DF45C
:10DCC800BAA891ED145A9DED0F4A25EE855AA4EE97
:10DCD800075AB0EE674AA5EE264AB0EE445ABEF19E
:10DCE800000F00F0F482B4EEC46AF1EE10FA40F3CB
:10DCF800EE823046A842A8BF284605EE100AB8EEC4
:10DD0800C55A062A83ED055A3DF495A891ED185A8F
:10DD18009DED104A25EE855AA4EE075AB0EE674AE3
:10DD2800A5EE264AB0EE445ABEF1000F00F0C582B7
:10DD3800B4EEC46AF1EE10FA40F3BF823046A8424E
:10DD4800A8BF284605EE100AB8EEC55A072A83ED83
:10DD5800065A3DF470A891ED1C5A9DED114A65EEE6
:10DD6800855AE4EE075AE5EEA67ABEF1000F00F0F8
:10DD78009C82F4EEC67AF1EE10FA40F196823246B1
:10DD8800AA42A8BF2A4604EE902AF8EEE44AC3ED58
:10DD9800074AFDF750B8134997F916E00B8897F929
:10DDA8000A20B1F9020010491EFB03F3524200FB9E
:10DDB80002F081FB03E2121181FB00E1DB17C017BF
:10DDC800C0EB2110991AD31A01440344A8EB0101AE
:10DDD8001D4431807580FDF707BD00BFA82F0020C6
:10DDE80060320020CC3600201F85EB5191ED006A8F
:10DDF800DDED0A4A25EE866AA4EE876AF0EE674AE8
:10DE0800E6EE264ABDEEE46A16EE103A984200F3B2
:10DE18009881AB42A8BF2B4606EE103AB8EEC66A08
:10DE2800B8F1000F00F03F83D54B012A83ED006A5B
:10DE38003DF401A891ED046ADDED0B4A25EE866AF2
:10DE4800A4EE876AF0EE674AE6EE264ABDEEE46A7B
:10DE580016EE106AB04200F37181AE42A8BF2E469A
:10DE680006EE106AB8EEC66AB8F1000F00F0098332
:10DE7800022A83ED016A3CF4DEAF91ED086ADDED1C
:10DE88000C4A25EE866AA4EE876AF0EE674AE6EE4B
:10DE9800264ABDEEE46A16EE106AB04200F34881E5
:10DEA800AE42A8BF2E4606EE106AB8EEC66AB8F1B2
:10DEB800000F00F01383032A83ED026A3CF4BBAF22
:10DEC80091ED0C6ADDED0D4A25EE866AA4EE876AAF
:10DED800F0EE674AE6EE264ABDEEE46A16EE106AF0
:10DEE800B04200F32281AE42A8BF2E4606EE106A69
:10DEF800B8EEC66AB8F1000F00F0E782042A83ED95
:10DF0800036A3CF498AF91ED106ADDED0E4A25EEF8
:10DF1800866AA4EE876AF0EE674AE6EE264ABDEE08
:10DF2800E46A16EE106AB04200F3FC80AE42A8BF65
:10DF38002E4606EE106AB8EEC66AB8F1000F00F079
:10DF48007C82052A83ED046A3CF475AF91ED146A6E
:10DF5800DDED0F4A25EE866AA4EE876AF0EE674A81
:10DF6800E6EE264ABDEEE46A16EE106AB04200F309
:10DF7800D680AE42A8BF2E4606EE106AB8EEC66A34
:10DF8800B8F1000F00F08682062A83ED056A3CF49A
:10DF980052AF91ED186ADDED104A25EE866AA4EEBF
:10DFA800876AF0EE674AE6EE264ABDEEE46A16EEA8
:10DFB800106AB04200F3BF80AE42A8BF2E4606EEFC
:10DFC800106AB8EEC66AB8F1000F00F07582072A29
:10DFD80083ED066A3CF42FAF91ED1C6ADDED114A22
:10DFE80065EE865AE7EE245AE5EEA67AFDEEE77A64
:10DFF80017EE902A904203DCAA42A8BF2A46104690
:10E0080007EE900AF8EEE77AB8F1000F7EF4D8AF81
:10E01800019A002A7EF4D4AFD145B8BFF0EE457A14
:10E02800FEF7CEBF77EEC76AF0EE477AFEF731BD4E
:10E038005449096811F080587EF473AEFEF76BBE40
:10E04800514B9FED526A93ED007A514BD3ED003A54
:10E058004D4BD3ED017A4E4B93ED014A4A4BD3ED2C
:10E06800026A4B4BD3ED024A4A4B37EE237A93EDC3
:10E07800005AD3ED015A484B019377EE847A37EE74
:10E08800057A76EEA46A77EEA57A27EE067A66EE2A
:10E09800866A67EE867A1946BDEEC77AFDEEE66AAD
:10E0A800FDEEE77A17EE102A0968CDED036A17EE40
:10E0B800903AADF82820CE04BDF90C20ADF82A30EE
:10E0C800ADF82C2000F1D480344A354B0792198BD7
:10E0D800B2F906E0FEF7FEBF324B1B78032B00F0C7
:10E0E80031810023FEF7F1BD9FED2F8AFEF777BF40
:10E0F8009FED2D8AFEF79CBF9FED2C0ADFF8C080AC
:10E1080025EE800A1FF03EFDD4F81851A8F8060045
:10E11800FCF757B82649274A8E46FEF7ADBB06EEF0
:10E12800100A2BE706EE100A05E706EE100ADFE6EE
:10E1380006EE100AB9E606EE100A42E706EE100AE5
:10E1480090E606EE100A69E6F2F78CFF1A4BDFF844
:10E1580070801E78029BC01AA8F80200FEF77CBAED
:10E168000AAB03EB8202FDEEC54A94464746724667
:10E178001249034814EE906AA046E64628E000BF1C
:10E1880060320020F4310020003200203333333F66
:10E198000C32002018320020744D0020D86E002068
:10E1A800304F00202A390020000000000000C8423B
:10E1B800244200207C2100203C500020A82F002071
:10E1C800405000209E45E0EC014A01F110012ED09C
:10E1D800D1ED004AB3EC014A65EEA44AE7EE044AE1
:10E1E800B0EE674AA6EEA44AF0EE444A32B1B4EE65
:10E1F800446AF1EE10FAC8BFF0EE454AFDEEE44A73
:10E2080014EE90CA664504EE906A04DCAC45A8BFDB
:10E21800AC4604EE90CAF8EEE44A002FD2D1019C35
:10E22800002CCFD1D145B8BFF0EE454ACAE74446E5
:10E23800FCF701BEF2F716FF029BDFF80083D4F863
:10E248001C71D4F81851C01AA8F80200FEF78FBB49
:10E25800F2F708FFA64BDFF8E4821E78029B99F8D4
:10E268000020D4F81851C01AA8F80400FEF7E4B941
:10E27800A04B07931946A04BB1F906E0198B8E45C0
:10E28800BCBF5242ADF82C20FEF724BF9B4800F1DA
:10E29800800EFEF7B8B901230493FDF7B2BBA8F8C6
:10E2A8000600ABF8B450FCF7ACBEFDEEE77A17EE0B
:10E2B800902AB242FFF669AD62E5BDEEC55A15EE89
:10E2C800100AB042BFF63BAD05EE106A3CE5BDEE64
:10E2D800C55A15EE100AB042BFF60CAD05EE106A2D
:10E2E8000DE5BDEEC55A15EE100AB042BFF6DDAC1D
:10E2F80005EE106ADEE4BDEEC55A15EE100AB0420E
:10E30800BFF6AEAC05EE106AAFE4BDEEC55A15EE29
:10E31800100AB042BFF67FAC05EE106A80E4BDEE8D
:10E32800C55A15EE100AB042BFF650AC05EE106A99
:10E3380051E405EE106A28E4714FFEF7F6BF714606
:10E34800FFF7B9BB1AF046F9FCF754BE94F87431DC
:10E35800002B7CF497A9FCF782B9DFED6A7AF4EE1A
:10E36800E7DAF1EE10FA62DCDFED677AF4EEE7DA6D
:10E37800F1EE10FA5BD4654BD3ED007AB1EE677A13
:10E38800B4EEC7DAF1EE10FA54D4B4EEE7DAF1EEEF
:10E3980010FA88BFB0EE67DA5D4BC7ED00BA1B68AC
:10E3A8009342BCF6A7A8FDF717B95A4A5A4B10680A
:10E3B8001B689847594B9BED007AD3ED007A584B70
:10E3C800D7ED006A83ED020A564B67EE277A2B4495
:10E3D80027EE8C7AD3ED007A534B67EE277AF0EE6E
:10E3E800665AEDEE275A93ED006AB1EE467AF4EEDE
:10E3F800C75AF1EE10FA08D4F4EEC65AF1EE10FA44
:10E408008CBFB0EE467AB0EE657A484B1B78012B8C
:10E4180002D0192B7CF4ADA8DFED457AB4EEE7DA2B
:10E42800F1EE10FACCBF01230023FCF7ADB89FED45
:10E4380041DAB1E7B0EE47DAAEE7019E002E7FF48D
:10E4480080ADD145B8BFB0EE456A7AE5132B05D14A
:10E45800B0EE480A1FF096FBA9F80000B0EE480A93
:10E46800DBF8143234489847214B1B78132BB0EE55
:10E47800408A7BF4EBAE1FF085FBA9F80200FBF79E
:10E48800E5BE019E002E7FF4F3ACD145B8BFB0EED7
:10E49800456AEDE4019E002E7FF476ADD145B8BF04
:10E4A800B0EE456A70E5019B002B7FF4BDACD14509
:10E4B800B8BFB0EE456AB7E4019E002E7FF487AD81
:10E4C800D145B8BFB0EE456A81E5019E002E7FF4C4
:10E4D80015ADD145B8BFB0EE456A0FE5019E002ED7
:10E4E8007FF4E9ACD145B8BFB0EE456AE3E400BFBC
:10E4F8003C500020D86E0020304F00207C210020A6
:10E508008458002000C0F84400C0F8C41058002007
:10E51800F4570020845700209857002094000020CA
:10E5280000320020AC57002014580020D456002098
:10E538000000964200000000F84C002040500020E7
:10E548002DE9F04F724B734A1C7893B000F59C414B
:10E558002031814607911160002C00F00D856E4A2C
:10E568001268904240F22E826C4A6D491768DFF8B3
:10E57800E8B10492013C1C706A4C039107F480577F
:10E58800002F40F02C82039B5B7D002B40F0C08461
:10E59800049B1B681D0400F11A87634B9945A378F7
:10E5A80000F29D83002B40F09D83604B0593049BF4
:10E5B8001F6817F4805940F05584039BBBF9066027
:10E5C8005B8B9E42B4BF00260126594B1B6813F093
:10E5D800805300F00E82059A127812F0010200F0C2
:10E5E8000F8203985349408C91ED037A07EE900A05
:10E5F800F8EEE77AB4EEE77AF1EE10FA80F2E18706
:10E60800002E40F004824C4D95F8A010002940F0EF
:10E61800FE814A494A480D6895F82D50002101604D
:10E62800416081604749002D40F0F2810D70002A59
:10E6380040F0F381444B1A78002A50D10399BBF972
:10E6480000E04F8B898BBBF90200BE45CCBF80250B
:10E65800002545F040038E45A8BF2B469B0843F094
:10E668008005B842C8BF2B4643F040058842A8BF82
:10E678001D46BBF904E0BBF90600AD0845F0800370
:10E68800BE45C8BF1D4645F040038E45A8BF2B4672
:10E698009B0843F0800E284DB842C8BF734643F02C
:10E6A800400E95F8A2708842B8BF73469F4201F0A9
:10E6B8002181A5F8A42085F8A620244985F8A23050
:10E6C8000F78002F01F06D805F2B01F0F8806F2B21
:10E6D80000F0CF87059B1B78DB0740F19187049BEF
:10E6E8001B4A1B68069203F00403002B40F0FB84CE
:10E6F8000DF14008174D0023C8F8043005F1500902
:10E70800109340F6330A192740F2833629E000BFF8
:10E718003C440020E03F002038440020744D002095
:10E72800304F0020F0360020404B4C00D2350020FE
:10E73800F4310020F4500020442300204836002003
:10E748000C320020F0220020C03C0020481C002091
:10E758007036002038340020D86E002004354D452E
:10E7680020D0AA78EB789A4217FB0261F6D26A7831
:10E77800043217FB03633BF912205245A8BF5246E7
:10E78800B2F5617FB8BF4FF461728A42E6DD9A4202
:10E79800E4DC29782429E1D840460435F4F7CCFD97
:10E7A8004D45DED1B34B98E803001F78B24B83E8A0
:10E7B8000300002F00F022840121AF48F4F7CCFDBC
:10E7C800002840F0A681E378002B40F0A281AB4CF2
:10E7D80023881DB225F00105AEB2B342268000F0B1
:10E7E8008986A74D02270E204FF014094FF0FF0825
:10E7F8002F7085F8019085F8028019F007FF3946D7
:10E808009D482688F4F7A8FD002841F0258026F0C9
:10E8180002039BB2B34223800AD0994B1421FF22F2
:10E8280002250E201D7059709A7019F0EFFE268887
:10E83800944BDFF89CA21978DAF804000393B50723
:10E8480008BF81F00201C1F34001F3F7C1FD2421A3
:10E858008948F4F781FD30B9059A1378590744BF00
:10E8680023F004031370069B1B6813F00A0F24D0CF
:10E8780005218148F4F770FD002800F06F8625888F
:10E888006B0740F169877C480621F4F765FD00288D
:10E8980000F051866F0640F17C8707217648F4F72F
:10E8A8005BFD50B1784B794AB3F90430784982FB63
:10E8B8000302DB17C3EBA2030B800C216E48F4F7AD
:10E8C8004BFD2288002800F0408142F480739A4270
:10E8D800238009D06A4B02251421FF220E201D70C7
:10E8E80059709A7019F092FE6A4B1B78082B00F049
:10E8F80038810E2B00F03581049B1B685E0544D5DA
:10E90800654B1B79002B00F0E98014215A48F4F775
:10E9180023FD002840F0E7800DF0EEF9012019F002
:10E92800BDFD90B3DFF8AC8100254FF0CC0902E0C3
:10E93800DDB2022D29D809FB05F76B1C58F80760D2
:10E94800002EF5D1C378554A90F9020052F82330C9
:10E958000196032200920121324619F027FA034654
:10E9680005EB450000EB0010049353B1314608EB6A
:10E978008000CC2221F011FA049B48F807300135B9
:10E98800EDB212F0DDF80028D3D1059B1B78DD0726
:10E9980040F1FA804249434A01230B701370039BEC
:10E9A800DAF80000197801F00101F3F711FD069B70
:10E9B8001D686A0700F15881EB0600F1728113B0F7
:10E9C800BDE8F08F384B394A1F68049307F4805725
:10E9D8000392DFF804B1364C002F3FF4D4AD002188
:10E9E8002548F4F7B9FC00287FF4CDAD0FF0EAFB19
:10E9F800C9E578023FF5EFAD059A127802F00102F9
:10EA08002C4D002185F8A010002E3FF402AE2A49B3
:10EA180001200870002A3FF40DAEF9067FF50AAE12
:10EA2800264A1278D2063FF505AEB9F1000F7FF4F9
:10EA380001AE002B7FF4FEAD7D023FF5FBAD204B10
:10EA48001B78002B01F042831E4B9B78002E41F06F
:10EA58004D833BB11C4A1D4B12681B689B1A002B47
:10EA6800C1F2E9831020134D19F0D0FD012385F878
:10EA7800A130DFE537360020F431002026390020A8
:10EA88006C30002050620020CC3600206766666635
:10EA9800202D002034340020E4500020C41903083D
:10EAA800D3350020502D0020744D0020304F002019
:10EAB800F036002044230020F0220020FC31002002
:10EAC800481C0020F070002088620020F83D0020DB
:10EAD80054620020286B0020D86E0020059B1B780C
:10EAE800D8077FF519AF3C201AF0A4FE00283FF4A0
:10EAF8004CAF02F0D1FE3C201AF048FE00283FF44B
:10EB080044AF02F0C9FE3C201AF040FE0028F0D1C4
:10EB18003BE7069B1B689A077FF559AEAC4C2688E5
:10EB2800F3073FF574AE46F001039E4223803FF49D
:10EB38006EAEA84B1421FF2202250E201D705970BD
:10EB48009A7019F063FD268861E622F480739BB2FF
:10EB58009A4223807FF4BEAE9F4B1B78082B7FF42C
:10EB6800C8AE228822F040039BB29A4223803FF429
:10EB7800C3AE984B02251421FF220E201D70597038
:10EB88009A7019F043FDB7E6944B93F80090B9F1E9
:10EB9800000F5FD1DFF89082914F18F8030C3E7890
:10EBA8004146A8F103051CF0DAFC002800F0B88300
:10EBB800002E40F00A8405F1080168791CF0CFFCAA
:10EBC800002841F095818749A87A1CF0C8FC0028E4
:10EBD80000F0B983022E41F08F818349E87B1CF055
:10EBE800BEFC002841F08C818049287D1CF0B7FCD0
:10EBF800002800F0B983042E41F086817C49687EA4
:10EC08001CF0ADFC002841F083817A49A87F1CF0F4
:10EC1800A6FC002800F0B983062E41F04C81764905
:10EC280095F823001CF09BFC002840F015877349D9
:10EC380095F828001CF093FC002800F0B983082EF2
:10EC480040F0F4866E4995F82D001CF088FC0028E9
:10EC580040F0B9836B4B01221A701CF004FF069B2D
:10EC68001D686A077FF5A8AE03201CF0A3FC0028E6
:10EC780000F05886238813F008067FF49DAE08201C
:10EC880019F0D4FD6048614B006818606049614A1A
:10EC9800069D614BBBF806002D68088016601E6053
:10ECA8008AE616201CF086FC002800F01D862388C2
:10ECB80013F400747FF483AE4FF4007019F0B6FDBE
:10ECC8005148534D5149534A534BBBF806600068AD
:10ECD8002E80086014601C6013B0BDE8F08F0BB97B
:10ECE8000123A3704D4B05931B201F7894F82160D6
:10ECF8001CF060FC012E07F00109824600F0DB855C
:10ED080007F00203069394F82030DFF82081444D81
:10ED1800052B00F29A80DFE813F08B004F00060005
:10ED2800D800F900BD00012E04BF052384F8203067
:10ED3800B9F1000F00F00D81039B3A4FB3F9181099
:10ED4800B8F80030002261F30F0263F31F4200237A
:10ED580061F30F0361F31F43CBF80420396862693C
:10ED6800CBF80030914200F21384012E41F0DC818F
:10ED7800032294F820300692CAE71CF047FC0128C9
:10ED880007D1284FB8F802303A68642101FB032301
:10ED98002361BAF1000F04D098F80630002B40F038
:10EDA8008C80012E51D01F4F22693B689A42C0F0D7
:10EDB800F485012384F82030012E6BD098F80730B1
:10EDC800012B00F0CF8006F001FA94F820309FE77D
:10EDD800263900206C30002034340020D335002040
:10EDE800980000205C2F0020612F0020662F002053
:10EDF8006B2F0020702F0020752F00207A2F002005
:10EE08007F2F0020502D00203C2D0020382D002081
:10EE18002C2D0020302D0020282D0020D235002058
:10EE28001437002088620020522F00205030002024
:10EE3800B9F1000FA1D14FF48060BAF1000F00F0D2
:10EE4800778319F0F3FC00232361069B002B3FF422
:10EE5800AEAB069819F0DAFB049B1F6817F48059CB
:10EE68003FF4ABAB1D21B248F4F776FA00287FF4E3
:10EE7800A4ABB04A039BD2881B8BBBF90660991AD6
:10EE88008E4240F3948513449E42B4BF0026012667
:10EE9800FFF79BBBA84F3A68B8F80230642101FB22
:10EEA80003234FF480600022236184F82020E2705D
:10EEB80019F0A4FC94F820302AE706F087F9032219
:10EEC8004FF47A7384F82020E3619B4F2B8843F03A
:10EED80002032B800FF076F93A68E36913440422A1
:10EEE800A36184F82020012E40F051853B68A26977
:10EEF8009A42AAD2914B187818B91CF05BFB0028EB
:10EF0800A3D12B8823F002032B80C4E78A4FEAE7BA
:10EF1800039A013BD27D3BF91330002A40F033833A
:10EF2800A3F57A73B3F57A7FA8BF4FF47A7323EA0F
:10EF3800E37307EE903A9FED827AF8EEE77A67EE90
:10EF4800877A804AFCEEE77A17EE903A1380FFF74B
:10EF580024BB794F3B6847F230520323E26184F8BF
:10EF68002030B3E706F032F9032240F6B83384F8CC
:10EF78002020E361704FA9E7734F3B78002B00F026
:10EF88004F87724BDFF8D881DFF8D8B1DFF8D8A106
:10EF9800039345465E46049099460EE019F804101E
:10EFA8009847032C28DC88B93B782AF8020F0134EB
:10EFB8009C4205F1040580F2DD80072CE1B2304661
:10EFC800DBF80430EADD984700B2EDE738F8242092
:10EFD8006B88801A4FF47A719B1A01FB00F040F697
:10EFE800CA0290FBF3F00844904240F2EE23A8BF17
:10EFF80010469842B8BF184600B2D5E7DFF86CA1B2
:10F00800DFF86C81524D0AF15A064FF0010951465A
:10F018001AF8010C1CF0A3FAF8B19AF804009AF84F
:10F0280002309AF803E000EB400105EB8101013B57
:10F03800D1F8B42003EB4303434493420DD095F831
:10F04800E02081F8B0E009FA00F022EA0000C1F8F7
:10F05800B430C1F8B87085F8E0000AF1060AB24584
:10F06800D5D13C49344A3C4B3C4D09681B78D2F811
:10F07800009008910793A5F1B00A00266B685BB36E
:10F088001F784FB3AA68A9EB0202002A0ADB9AF894
:10F09800E0200121B14022EA010209F5FA718AF85B
:10F0A800E020A960079ABAB12A7859780432D2B216
:10F0B800002940F08C8203993BF91220098B01F159
:10F0C800C800824240F335849AF8E0109A7841FAF1
:10F0D80006F3D80740F1A5840136042E05F10C0586
:10F0E800CCD1FFF769BB1A4D95F8AA3053B1059BEF
:10F0F8001B78DE0706D5039BBBF906205B8B9A427B
:10F1080000F3658411210A48F4F726F9002800F075
:10F11800468295F8AE302BB995F8A83013B932234A
:10F12800A5F8AC30012385F8AE30FFF7E1BA00BF8F
:10F13800F43100203430002088620020481C002070
:10F14800AAF1823F243900204C540020304F00207F
:10F1580044230020CC700020ED380020F423002048
:10F16800645400203437002042230020692E0020F8
:10F17800CC000308DDF81090C44A04921146C44A32
:10F188000968A2FB092A42F201020A404FEA9A1AC8
:10F19800059200F00082BF4DBF48C04CC04A95F8A8
:10F1A80000E0007884F800E01070BEF1000F04D091
:10F1B800BB4A92F800E08EF0010EBA4D0F2085F898
:10F1C8002400002B00F0FA82B74B039E0C931B78A7
:10F1D800B6F826C00B931C463B78B78C039EB34AFF
:10F1E800368B0E962646A2FB0442520802EB4202D8
:10F1F800B21AD2B2CDF824C001F48051089295F821
:10F208002580DFF8C0B2DFF8E8C20A900AF59672E6
:10F2180076460F9105F1280400200692CDF8349027
:10F22800AE46002E00F03A823EF910201FFA82F90D
:10F23800B9454FEA400103D3099DA94540F27282BE
:10F248005CF82020924580F032823BF90120059D30
:10F25800002D40F04682013098422BF8012004F13D
:10F268000604DEDB0A98924ADDF834908EF8258091
:10F278000F280CBF012100218EF82400117000F026
:10F28800A4828C4C8C4E8D4F35883868A168626892
:10F29800E06045F00405401A90427F4F3580804D6C
:10F2A8004FF0010188BF00223970297088BF84F8A7
:10F2B8002120002B00F09B82049A03991768804E46
:10F2C800B1F824C0B1F818E07E4817F480573546E5
:10F2D80040F0D38239460EE06A7802EB820202EBF4
:10F2E800820202F2EE2292B20131994220F8022BF8
:10F2F80005F102050ED016F81120002A00F016823A
:10F30800022AE9D00131028820F8022B994205F13E
:10F318000205F0D10C9A137801331370FFF730B956
:10F3280008F1050168791CF01AF900283FF44BAC84
:10F33800012E40F0DD8505F10D01A87A1CF00FF9CA
:10F34800002840F0D9856049E87B1CF008F90028BE
:10F358003FF44AAC032E40F0D3855C49287D1CF06D
:10F36800FEF8002840F0D0855949687E1CF0F7F86F
:10F3780000283FF44AAC052E40F0CA855549A87FBD
:10F388001CF0EDF8002840F09685534995F82300C5
:10F398001CF0E5F800283FF44AAC072E40F05C83E7
:10F3A8004E4995F828001CF0DAF8002840F03E8312
:10F3B8004B4995F82D001CF0D2F800283FF44AACD0
:10F3C800092E3FF447AC4FF009094B4631E3354D60
:10F3D800D5F88830A9EB0303002BFFF6DEA8414AD5
:10F3E80095F88C30517C079AC5F8882001333E4A3D
:10F3F800039E32F81120B17D03F00F0385F88C309D
:10F408002B4492B292FBF1F283F8902095F8901079
:10F4180095F8912095F8923095F89C000A4495F853
:10F428009310134495F89420194495F895300A449C
:10F4380095F89610134495F89720194495F8983044
:10F448000A4495F89910134495F89A20194495F8A8
:10F458009B300A44134495F89D1095F89F20184452
:10F4680095F89E3001440B441A4442F30B12642A67
:10F47800F17DA8BF642213B209B1C2F1640307EE9B
:10F48800903A9FED1A7AF8EEE77A58E5744D002025
:10F49800D34D6210BC3F002084140020ED380020BA
:10F4A8008514002044230020F9530020ABAAAAAAFF
:10F4B80032370020F0360020143700208862002000
:10F4C80098540020D86E0020612F0020662F00205D
:10F4D8006B2F0020702F0020752F00207A2F00201E
:10F4E8007F2F0020046200202062002014AE2341F8
:10F4F800FC5300200221C648F3F72EFF00283FF4F2
:10F5080086A92580B7073FF593A946F00203B342C1
:10F5180023803FF48DA9BF4B02201421FF221870CD
:10F528000E2059709A7019F071F82688FFF780B983
:10F5380019F064F987E425F040039BB2AB422380BD
:10F548003FF4ABA9B34B02251421FF220E201D70F6
:10F5580059709A7019F05AF8FFF79FB9238823F069
:10F568000405ADB2AB4225803FF48DA9A94B022515
:10F578001421FF220E201D7059709A7019F046F858
:10F588002588FFF780B9C3F53B6308331BB2C7E48E
:10F5980003230693DFE4A04A92F800E005E695F815
:10F5A800A830002B3FF4A4A8059B1B7813F0010397
:10F5B8007FF49EA8012285F8A83085F8A920FFF7D6
:10F5C80097B8964D012185F8A010FFF720BA0129B8
:10F5D80000F0E0839AF8E0200123B340013613439A
:10F5E800042E8AF8E03005F10C057FF447ADFFF7EB
:10F5F800E3B8059B8A4A1B781060D80700F1F581AB
:10F6080095F8A61000297FF46AA8B5F9A430322B22
:10F618007FF765A895F8A2200120572A85F8A6004B
:10F6280000F02E84049B1B6813F0040302D05A2AAE
:10F6380000F039855D2A00F0B1845B2A00F0D3849C
:10F648005E2A00F0DD84562A00F01285972A00F021
:10F658001E85A72A40F06A847249049B0A781B68B1
:10F6680042F004020A70704A069203F00403FFF79E
:10F678003CB8B2F5FA7FFFF632A895F8A620002A22
:10F688007FF42DA8059B1B78012185F8A610D907C2
:10F6980000F142840EF0D8F8FFF721B8002F3FD0D0
:10F6A8005CF8202092454FEA4001FFF4CEAD5F4A56
:10F6B8005E4D525C05EB0109002A00F09D80022A8C
:10F6C80047D199F8012002EB820202EB820202F292
:10F6D800EE2292B2032833DD059D12B2002D3FF4CD
:10F6E800BAAD089D24F81520B8F1000F03D10B9D81
:10F6F800022D7FF6B0AD2288B4F80290B4F80480E9
:10F708004A4490444A4A0FFA88F882FB0852494D05
:10F71800A2EBE87225F8018012B24FF001089AE5D1
:10F728003A464100069D4CF8205090E5CAB2022A9C
:10F7380004D9032A7FF4E6AD6246D5E57246D3E5DF
:10F74800012505FA00F90A9D25EA090512B20A956C
:10F758007DE53BF80120BDE745F004039D42238089
:10F768000AD02C4B02251421FF220E201D7059703F
:10F778009A7018F04BFF25882F4B304AB3F90430A4
:10F788002F4982FB0302DB17C3EBA2030B80FFF7B1
:10F798007AB845F04003AB4223807FF4D3AEFFF73D
:10F7A8007CB839461A48F3F7D7FD00283FF421AF53
:10F7B80085F8A7700EF048F8FEF78CBF2149224A59
:10F7C8000C91DFF890B0012111701B2110480593AE
:10F7D800F3F7C2FD059B00287FF453AD1B4C1C4F6B
:10F7E800E2683B68A3609B1AC82B00F23B83049B2A
:10F7F8001F6807F480578DE5C2B2022A40F2C8821A
:10F80800032AA6D10E9A0F9D002D08BF3A4661E73C
:10F81800F43100206C300020ED3800204423002013
:10F82800FC3D0020FC310020703600209854002058
:10F8380056555555B4230020CC36002067666666B9
:10F848000C2D0020F953002032370020F03600201C
:10F8580088620020D86E002026F001039BB2B342D4
:10F8680023803FF44FAE0E202F7085F8019085F865
:10F87800028018F0CBFE268844E600210FE06A7863
:10F8880002EB820202EB820202F2EE2292B2013114
:10F89800994220F8022B05F102053FF43BAD16F81A
:10F8A80011201AB1022AEAD00288F0E7CAB2032A64
:10F8B800FAD87246EBE700230693FFF724BAB2F5AD
:10F8C800FA7FFEF60CAF95F8A630002B7EF407AF52
:10F8D800059B1B7801210B4085F8A61000F0A48237
:10F8E8000EF070FCFEF7FBBE4FF4007018F086FFB8
:10F8F800FFF765B8BE4ABF491068B5F9A420C769C3
:10F9080081FB07018911FF17781A00F5FF407F3046
:10F9180082423EF7D2AEC91B0A4412B2A5F8A4200F
:10F92800FEF7CBBE082018F069FF069B1D68FFF79D
:10F9380043B8C8398A423DDA9AF8E0109A7841FA11
:10F9480006F3D9073FF5C8AB52420120099218F0D7
:10F958003DFF7B1E099A162B00F2C280DFE813F0E8
:10F96800B001C6019701EF01DC01030282016D01BC
:10F97800560131011A01C000EF010501030282019D
:10F988006D01EF00D900C300AE00960080003A6810
:10F99800E3691344A361FFF758BA05F017FC032283
:10F9A80040F6B83384F82020E361FFF78FBA0126C8
:10F9B800FEF70BBE9AF8E0300122B24023EA0203B8
:10F9C80009F5FA728AF8E030AA60FFF785BB0021D2
:10F9D8008948F3F7C1FC00287FF494AB322385F8FB
:10F9E800AA00A5F8AC30FFF78DBB844B1B78002B21
:10F9F8003EF475AEE378002B7EF471AE95F8A7302F
:10FA08000133DBB2032B85F8A7307EF668AE7C4B5A
:10FA18005B7813B9002E7EF462AE0EF0D3FBFEF7CE
:10FA280059BE002A0CBF012002208FE74FF00809B9
:10FA38004B4603EB83031D4487F80090A978687848
:10FA48000BF094F8059B6F4A1B7801211170D907B8
:10FA58007FF503A9FEF7A3BF4FF007094B46E8E778
:10FA6800DAF8E400DFF8A08190F8361098F8023050
:10FA780011446429A8BF642121EAE17180F8361095
:10FA8800002B40F08B8316F081F9A3E5DAF8E40047
:10FA9800DFF8748190F8371098F802301144FE2985
:10FAA800A8BFFE2121EAE17180F83710002BEAD0C7
:10FAB80016201BF0DDFDDAF8E400E4E70898DFF82B
:10FAC800488141781144B1F5967FA8BF4FF49671EB
:10FAD80021EAE171417098F80230002B40F0588318
:10FAE800DAF8E400CFE7DAF8E400DFF81C8181787F
:10FAF8001144C829A8BFC82121EAE171817098F88A
:10FB08000230002BBFD014201BF0B2FDDAF8E4005D
:10FB1800B9E7DAF8E400DFF8F08041781144C82941
:10FB2800A8BFC82121EAE171417098F80230002B82
:10FB3800A9D013201BF09CFDDAF8E400A3E7DAF85B
:10FB4800E400DFF8C48001781144C829A8BFC8219F
:10FB580021EAE171017098F80230002B93D012204D
:10FB68001BF086FDDAF8E4008DE7DFF89C80089842
:10FB780098F80230417911446429A8BF642121EA28
:10FB8800E1714171002BABD00E201BF071FDDAF84A
:10FB9800E40078E7DAF8E400DFF86C80017A98F896
:10FBA80002301144C829A8BFC82121EAE1710172B5
:10FBB800002B3FF468AF0B201BF05AFDDAF8E40085
:10FBC80061E7DAF8E400DFF84080C17998F802309C
:10FBD8001144C829A8BFC82121EAE171C171002BCD
:10FBE8003FF451AF0A201BF043FDDAF8E4004AE77E
:10FBF8005C3B0020D34D6210F4310020ED3800202A
:10FC0800F0700020502D0020943C0020DAF8E40029
:10FC1800DFF87885817998F802301144C829A8BF9F
:10FC2800C82121EAE1718171002B3FF42CAF092032
:10FC38001BF01EFDDAF8E40025E7DAF8E400DFF847
:10FC48004C85417998F802301144C829A8BFC821C9
:10FC580021EAE1714171002B40F05382112F7FF4AA
:10FC680046AF10E7DAF8E400DFF82085017998F864
:10FC780002301144C829A8BFC82121EAE1710171E5
:10FC8800002B40F0D082102F7FF447AFFBE6089995
:10FC9800DFF8F8840F791744642FA8BF642727EA90
:10FCA800E7770F711BF0FEFC98F80230002B3FF449
:10FCB80017AF032039461BF0DBFCDAF8E400E2E674
:10FCC8000898DFF8C88401781144FA29A8BFFA21F6
:10FCD80021EAE171017098F80230002B3FF400AF7F
:10FCE80001201BF0C5FCDAF8E400CCE60898DFF840
:10FCF8009C84817811446429A8BF642121EAE171B8
:10FD0800817098F80230002B3FF4EAAE02201BF015
:10FD1800AFFCDAF8E400B6E60898DFF87084C17939
:10FD280098F80230114481F30801C171002B3FF4A7
:10FD3800D7AE05201BF09CFCDAF8E400A3E6089B8C
:10FD4800DFF84884997998F8020011446429A8BF1B
:10FD5800642121EAE1719971002840F0DA810D2FC0
:10FD68007FF405AFBCE6DAF8E400DFF82084C17858
:10FD780098F802301144C829A8BFC82121EAE171C6
:10FD8800C170002B40F05F820F2F7FF4DCAE7AE663
:10FD98000E9A9FE43BF912209978B2F5617F4FF4EF
:10FDA800966393FBF1F332DB40F633019142A8BF2F
:10FDB80011460C2FA1F5617191FBF3F100F0F98068
:10FDC800182F7FF407ACC9B2C8290B46A8BFC823AF
:10FDD800DAF8E400C27DDFB297423FF4FBAB9A1A2F
:10FDE800DFF8A883C77548BF0732D71098F80230E4
:10FDF8000137FFB23BB9002F3FF4ECAB384618F09F
:10FE0800E5FCFFF7E7BB18201BF032FCF3E70C2FEB
:10FE180000F0E680182F7FF4DDAB00210B46D7E712
:10FE2800C34A0392FFF7A8B9C249096811F400311F
:10FE380040F0EA800B46C048C65C0F2E03F10C0365
:10FE48003DD001311529F7D1049BBC491B680691A7
:10FE5800FA3AA5F8A420002203F0040385F8A620A6
:10FE6800FEF743BCB64A049B1F68138823F00403BB
:10FE78001380012307F4805784F82130FFF74ABA2A
:10FE8800AE4AB04B069210461A68AF494FF47A73DF
:10FE9800B3FBF2F3C3EB431203EB82030268DB000C
:10FEA8005707A1F8B43000F1A280049B1B6803F047
:10FEB8000403FEF71ABC4FF006094B46B9E5A34EFA
:10FEC800D6F800E04B00BEF1000F07D05F1800EB3A
:10FED80087079EF801E07F787745B5D20B449C4FA1
:10FEE8009C4900EB8300002330603B800B60ABE74C
:10FEF8004FF001094B469CE54FF002094B4698E547
:10FF08004FF003094B4694E54FF004094B4690E542
:10FF18004FF005094B468CE5049B8F491B680A6026
:10FF2800864A069203F00403FEF7DFBB0021BB2AD2
:10FF3800109100F09880B72A00F09180BE2A00F056
:10FF48009580BD2A67D0792A00F05A817A2A00F074
:10FF580050819E2A00F047819D2A00F03D81AE2AFB
:10FF680000F03381AD2A00F02981EF2A00F02081CA
:10FF7800FD2A00F01781FB2A00F04F81FE2A00F0CD
:10FF88004681F72A00F067817B2A7EF4A8AB4FF4FC
:10FF9800FA6102201BF0E6F8FEF7A1BB6F4B0022C6
:10FFA80001206F4D6F492A700B6018F00FFCFEF7A7
:10FFB80096BBCFB26A4B09915B78BB423FF40AAB60
:10FFC800DFF8C88138461BF0A7F998F8023009997C
:10FFD8001BB1C9B20C201BF04BFB0137FFB20AE77B
:10FFE80000273946E6E7604B01220220D9E7049B47
:08FFF8005E4A1B680A2111801A
:020000040801F1
:1000000003F00403FEF775BB5B4B02220320CCE731
:100010005A490978032900F0868019460FE74FF600
:10002000FE73574A474896890690D0893344014465
:100030009381D18110F06AF8F2F7D8FC10F04EF8F5
:10004000F5F776FE012018F0C5FB049BB5F8A42057
:100050001B68FA3A0021A5F8A42003F0040385F8F0
:10006000A610FEF746BB0B464FF6FE71D9E70B46CE
:100070000221D6E70223D4E710F048F8F2F7B6FCE5
:1000800010F02CF8F5F754FE012018F0A3FB95F8BA
:10009000A220FFF7DFBA049B3A4A1B684FF4C871ED
:1000A0001180284A069203F00403FEF722BB95F85C
:1000B000A820002A40F0DE8095F8AA3083F00103E2
:1000C00085F8AA30002B40F0D0800C2018F0A2FA5E
:1000D000FEF709BB002E3EF4C9AC2B4D95F8A130BC
:1000E000002B3EF4ABAA18F079FA002385F8A13072
:1000F000FEF7A4BA002BF0D02449254A09684FF432
:100100007A7000FB03131360E7E7112009921BF0DC
:10011000B3FADAF8E400099AA4E50D2009921BF07D
:10012000ABFA099A1FE618F059FAB5F9A4208FE640
:1001300003230693FEF791BE304F00205C2E002073
:10014000580703087036002014370020644D002043
:10015000E04A0020A02200203A2300203C23002077
:10016000FC3D0020783B00203C3600204836002033
:10017000C63B0020EA700020143C00202A390020F1
:1001800028440020EC7000204423002088620020D6
:10019000F83D0020943C002015201BF06DFADAF8A1
:1001A000E40074E417201BF067FA9DE400210120AD
:1001B0001AF0DCFFFEF797BA002108461AF0D6FFC6
:1001C000FEF791BAFF2100201DF01EFB95F8A2203A
:1001D000CFE6012100201DF017FB95F8A220C5E60F
:1001E0000021FF201DF010FB95F8A220BBE60120A6
:1001F0001DF00AFB95F8A220B2E6224A137A43F0DA
:1002000001031372FEF76FBA1E4A137A23F001033B
:100210001372FEF768BA002103201AF0A7FFFEF759
:1002200062BA002102201AF0A1FFFEF75CBA10208A
:1002300009921BF021FADAF8E400099A27E5124D39
:100240000DF0C4FF002385F8A130FEF7F7B90F20A9
:1002500009921BF011FADAF8E400099A98E50021F6
:1002600004201AF083FFFEF73EBA0B2018F0D2F9F3
:10027000FEF739BA054A85F8A81085F8A900069254
:10028000FEF737BA183700204423002070360020CC
:10029000024B1A889B780280837070471401030810
:1002A000084B196861B130B45D68074C642202FBE9
:1002B00005F2B2FBF1F2228030BC002018605860D9
:1002C000704700BF2C240020D0300020704700BFB2
:1002D0006F4B1B78002B3AD02DE9F0416D4B6E4DE2
:1002E0009B79AC68A860013B82B0041B032B00F231
:1002F0009C80DFE803F04A0231291BF08BF90028CB
:1003000000F09B80654B66491B78B5F84220D1ED23
:10031000037AEA64DB0700F1AA8002FB04F007EE2F
:10032000900ADFED606A604BB8EEE77AD5ED127A9D
:100330005A60E7EE267A1A60BDEEE77AC5ED127ACA
:1003400085ED117A83ED027A02B0BDE8F081564A5C
:100350001360536093607047544B1B681801F3D5CA
:10036000FF2012F095FE03780A2B88BF00214E4B28
:100370009CBFB0F90420B0F90610296588BF0A4671
:100380006A655A601A609960DEE7494A494BD2793A
:10039000DFF8308133F81220B8F902304648B8F956
:1003A000001092B207EE902A40F6E44707FB02F6EF
:1003B000C3EB1633B8EE670A4FF47A7606FB03F305
:1003C00093FBF1F3AB61F0F7D1F8D5F818E0D5ED78
:1003D000047ADFED346AB8F90220334BB8F900C073
:1003E000C3F804E00EFB04F007EE100AB8EEC77A7B
:1003F000BCEEC06AE7EE267A8DED016ABDF8041006
:10040000C5ED047ABDEEE77A07FB01F7C2EB1737BB
:1004100006FB07F683ED027A96FBFCF685ED037A80
:100420006E611E6002B0BDE8F0811F4B00221A60B1
:100430005A609A6002B0BDE8F0811C4B1B68DE0672
:100440007FF560AF154BB5F842201B78EA64D907F9
:100450007FF563AFB5F94010184B00FB01F083FB4B
:100460000013C017C0EBA3100244EA6455E7FDEE89
:10047000E77A134E17EE900AA0F57A7101FB01F3AB
:1004800086FB0306D817C0EB26100844E2E700BF3E
:10049000F2500020E03600202C240020D23500202D
:1004A000F45000202FE33E31C0500020744D002056
:1004B000046200202062002048240020D34D6210F6
:1004C0001F85EB51AC2D0020F0B53E4B5B79012B25
:1004D00083B03DD0022B0FD03B4B00221A805A80B4
:1004E0003A4B1B78022B05D1374A394B5188128879
:1004F00019805A8003B0F0BD364B1B681B01EFD545
:10050000FF2012F0C5FD03780A2B56D8B0F902205F
:100510003149D31781FB0212C3EBA2039BB207EE52
:10052000903AB8EE670A2D4C04F15C00A4F85A30FA
:10053000F0F71CF8FCEEC07A234AB4F85A30CDED3F
:10054000017A5380BDF80430A4F858301380C7E70F
:10055000234A244B9278214D33F81240A4B207EE7F
:10056000904A05F18400B8EE670AEFF7FFFF1E4AD4
:100570001549107896785378FCEEC07A00EB40105D
:10058000CDED017ABDF8042044F6FB77C3EB0333CD
:1005900000FB027200FB0474B2FBF3F2B4FBF3F352
:1005A000B2FBF6F2B3FBF6F392B29BB2A5F8802051
:1005B000A5F882300A804B8092E79FED0C0A002359
:1005C000B1E700BFE0360020CC5000203C500020B6
:1005D00040500020744D0020676666662C24002081
:1005E0000462002020620020633B00200000000025
:1005F000F8B52C4D2C4C2D496E792D4B2D4A2E4F94
:100600000420087084F8A80000216420012EA4F8BA
:10061000AA10A4F8AC103970197059605870118084
:10062000518021D0022E10D0A979244A002301291B
:10063000136084F8AE305360936023D0022912D146
:100640001F4A636453609360F8BD282204F1580088
:100650001FF0A7FB4CF250319FED1A0A04F15C0029
:10066000F2F720FEE0E7F8BD282204F180001FF039
:1006700098FB4CF250319FED130A04F18400F2F71D
:1006800011FED1E7104AE36053609360D3609FEDA1
:100690000F0A02F110004CF25031BDE8F840F2F7B9
:1006A00001BE00BFE03600202C2400202A390020A3
:1006B000182D0020CC500020F2500020C050002007
:1006C00070240020CDCCCC3D38240020CDCCCC3EB5
:1006D0002DE9F0432F4DD5F8B03083B01BB195F81C
:1006E000B430022B02D003B0BDE8F0834FF02008F5
:1006F0004046294C05F1B809012655271AF05EFF3E
:10070000A0B199F800300BB9217891B908F101082E
:100710005FFA88F8B8F1230F04F1010409F1010927
:10072000E1D040461AF04AFF0028EAD189F80000DB
:10073000ECE7D5F8B00050B30DF1080EAA220EF880
:10074000052D8DF802108DF800708DF801608DF880
:100750000430694655225340082213F0800F02F1FD
:10076000FF324FEA430318BF83F0310312F0FF0258
:10077000DBB2F2D1714502D011F8012FEBE7AA22CA
:1007800069468DF803308DF8042018F09FFF89F832
:100790000060BBE72C240020180103081F4B1878C9
:1007A000002839D01E4A1389FBB11E4A9FED1E6AEC
:1007B000D2ED026A07EE903AF8EEE66AF8EE677A52
:1007C00007EE103A77EEE66AB8EEC77A66EE866A0A
:1007D000C6EE877AFDEEE77A17EE900A6428A8BF86
:1007E000642020EAE070C0B2704710B40F4B547818
:1007F0001B88117804FB1032091B642300FB01F0F5
:1008000003FB02F3B3FBF0F06428A8BF64205DF89B
:10081000044B20EAE070C0B2704700BFF2500020E5
:10082000E0360020C05000200000C842CC5000201C
:100830002DE9F04F794D81B0F0F718FCD5F8C040A4
:100840000022C5F8BC20002C00F0A580237D052BDC
:10085000074617D9216A23690B44C31A9342B8BFCC
:1008600005F1C0010ADBD5E0137D052B0AD9136A17
:1008700012691344FB1A002B80F2CC8051F8042F2C
:10088000002AF1D14FF0010B0023B9461E46C5F8EE
:10089000BC3098469A46274623E07A6A39693B7D00
:1008A000A9EB0204B4FBF1F40134A4B213FB04F38A
:1008B000013301369BB2B6B23C83FB82984506D227
:1008C000BBF1000F01D1012C5FD99846BA46D5F88B
:1008D000BC30013305EB8302C5F8BC30D2F8C070E0
:1008E00047B3BB68C3B1FC8A002CD6D1396A4846ED
:1008F000A9EB01019847D0B195F82031002B52D1D6
:100900003B7DC7F82490013601334FF00102B6B2A7
:100910003A83FB820124D1E73B6A3A69A9EB0304DD
:10092000B4FBF2F4A4B23C8334BBFB8AC6E73C833D
:10093000FB8AC3E72B686A683949013316443C4691
:1009400085E848004F46C1F800A0BAF1000F27D053
:10095000DAF8203095F82021AAF81640FB1ACAF8D8
:100960001C30CAF82090002A35D1DAF80C304846FD
:1009700001B0BDE8F04F18473B7D13FB04F3013392
:1009800001369BB2B6B2FB8298E73A7D062A04BFD5
:100990009846BA469BE72B68214A01332B601460C6
:1009A00001B0BDE8F08FF0F761FB1E4B1E4A1F4CF3
:1009B00011681A68A0EB090002EB000E2268C3F868
:1009C00000E09042A1EB5111014438BF1046164A95
:1009D0002060116094E7F0F749FBDAF80C30044628
:1009E0009847F0F743FBDAF82C20DAF82830DAF8E9
:1009F0003010001B9042A3EB53130344014438BF53
:100A00001046CAF82830CAF83010CAF82C0001B0D5
:100A1000BDE8F08F4FF0000B36E700BF2C2400201C
:100A20005C3B0020C0300020C4300020C8300020D3
:100A3000F0B43423184F194A03FB00F3D2F82461B1
:100A4000FC58FD18002E6B684B600C600DDDD2F871
:100A5000C0309D421DD0C032002303E052F8044F45
:100A6000A54216D00133B342F8D10022342303FB50
:100A700000700A720369CB60037D4B72836AC56A9A
:100A8000046BC2690A615B094D618C61CB61F0BC8A
:100A900070470122EAE700BF3C0100202C2400201F
:100AA0002DE9F041244ED6F82451162D27DC002DD7
:100AB0003DDDD6F8C030984221D005F1804106F1E5
:100AC000C007013907EB81013B4603E053F8042FCF
:100AD000904214D08B42F9D1D6F8C0409CB1237D0E
:100AE000017D8B420ED3154A002405E052F8043FE5
:100AF0004BB11B7D8B4206D30134A542F6DA0020B0
:100B0000BDE8F08100248046601C80002A1B011F84
:100B100006EB840439443844920001351FF027F96C
:100B2000C4F8C080C6F824510120BDE8F081E6D1A8
:100B300006F1C007D0E700BF2C240020EC240020E1
:100B4000182830D0162807D8184B342202FB003062
:100B500019B1C3680BB1A3E7704770B5144DD5F850
:100B60002441002C0FDDD5F8C03098420CD005F19F
:100B7000C0063346002203E053F8041F884206D023
:100B80000132A242F8D170BD002205F1C0069000EA
:100B9000011DA21A920031443044013C1FF0E7F8D5
:100BA000C5F8244170BD034B1868D1E73C01002013
:100BB0002C2400205C3B002010B54FF4804082B014
:100BC00017F070FC00B30022032390F90200009399
:100BD00001924FF4E1334FF4804117F0EBF80C4BE6
:100BE000C3F8B00070B1012402221620214683F818
:100BF000B84083F8B94083F8BA4083F8B420FFF7CF
:100C00009FFF204602B010BD014BD3F8B000E9E7CA
:100C10002C240020F0B50D4685B006460068F0F79C
:100C2000A5FB95E81800E41A0023039324238DF80C
:100C300008304D238DF80930B5F90A30FF2C2246D3
:100C4000A8BFFF2201333DD02B7B002B0CBF3E23DE
:100C50003C238DF80A30FE2C2B898DF80B208DF863
:100C60000C3031DD23128DF80D408DF80E30072742
:100C70003A4602A93068F0F77FFB02ABDA190DF1B2
:100C80000B0100238A4221D1002C8DF807300CDDA6
:100C9000224629683068F0F76FFB2B689DF8072023
:100CA0001919994216D18DF8072001220DF107017B
:100CB0003068F0F761FB3068F0F752FB04F109008F
:100CC00005B0F0BD2123C4E70527D1E711F8010BDA
:100CD0004340D7E713F8010B4240E2E72DE9F34721
:100CE000012017F0DFFB174EDFF85CA00024CC27B3
:100CF00008B1022C02D902B0BDE8F08707FB04F866
:100D000056F8085015B10134E4B2F1E7C37890F910
:100D100002005AF8233001950322009201212A464D
:100D200017F048F8814648B104FB0760CC222946F9
:100D30001FF037F8013446F80890E4B20FF004FFD2
:100D4000D6E700BF286B0020C41903082DE9F04F37
:100D50002DED088BBC4CBD4BC4F83C3887B000234C
:100D6000C4F84038F2F7ACFBF0F7FEFEF1F708FEEE
:100D700008B9F4F78FFAF4F7DBFF0522B449B54858
:100D80001FF05AF808B1F4F785FA94F84438B24DD8
:100D900043F0010384F84438B04B9A78B04B1A7092
:100DA000B04B1B682B6011F097FC01210220F1F77A
:100DB00047FBF1F727FD2B6819070BD5AA4B1A7AC9
:100DC0000A2A07D80123934040F20342134201D07C
:100DD00011F00CFB6420A54EF5F78CFAF4F74AFBF2
:100DE000A34ADFF8BCE20023B146995D03F10F008E
:100DF00003F11307304437440EEB010A10F8018F5A
:100E0000B8F1000F05D09AF80CC0C44508BF82F8AD
:100E100058C090F80480B8F1000F05D01EF801C04A
:100E2000C44508BF82F859C08742E7D1B2F85800DC
:100E300040B104EB810109EB03005065C1F848287B
:100E400002F517722033602BCFD12868C0F38010D1
:100E500010F0D8FF2B68DA0740F1BF8310F062FF73
:100E6000B4F86068834B94F85C081E80002E40F054
:100E7000BA83F0F753FE804A8049106094F85D28E9
:100E8000003218BF01220A7058B194F85E38C6715A
:100E9000002B4FF02402827114BF11210121F1F7C0
:100EA000D3F80020F1F7A2FA754B764E03F1300C1F
:100EB0004FF0000853F8057C77B313F9092CA118FB
:100EC00006EB021091F862E891F8659891F868A82D
:100ED000991E11F801BFF34591F802B008BF80F8E0
:100EE00004E0CB4591F804B008BF80F80590D345E5
:100EF00008BF80F806A08B42EBD11101721810795F
:100F000050B1507940B1907930B177505979D17161
:100F10009979117282F80C8010339C45CAD110F077
:100F2000EBFDDFF88091DFF8808159F8063C0293F1
:100F3000002B3AD019F90A6C142303FB06871A46D2
:100F4000002138461EF02DFFA219A9F1030A92F8DC
:100F50006B3892F86DB803931AF8011F039B9942FE
:100F600003D11846F0F7DAFDB8609AF80310594536
:100F700003D15846F0F7D2FDF860D145ECD11423E7
:100F800003FB06F108EB0102906870B1D06860B114
:100F90002644A9F10A0048F8010096F86F18029B50
:100FA000117496F8711853605174374B09F1100998
:100FB0009945BAD1354F17F039FF97F80890B9F134
:100FC000000F2DD04846F0F7A9FD314E80467060E5
:100FD00018B12F2383710023C3713F78002F40F095
:100FE0000683484618F00EF80746C8B1B8F1000F5E
:100FF00004D0027A02214046F0F70AFADFF8AC800A
:10100000244A00230193009339468023404619F077
:101010000BFFB268802333611360012308F8083C9A
:101020001D491E4A4B79581E4342434113708B7928
:101030005E1E7342734113712B681F0400F1078316
:1010400013F000733AD033E02C240020E913000899
:10105000D228030841360020744D00203C36002081
:101060003C500020B43C0020304F00201C010308FD
:10107000542500206062002064620020626200202B
:1010800085010308784D0020D6010308B0700020C8
:101090009C70002000A24A04E03600201862002064
:1010A0000C4F0020B601030828620020A470002025
:1010B000D74BDB7AA3F108014B424B41937017F0F9
:1010C00035FDD4F874383BB9D4F8782822B9D4F86F
:1010D0007C28002A00F09F801BB208EE103ADFED5A
:1010E000CDAADFEDCD8ACD4AB8EEC88A002128EE20
:1010F0002A8A117038EE280AFDEEC07A17EE903A6F
:101100002033402B00F2A582F1F7C8FFF0EE409AA1
:10111000FDEEC87A17EE903A2033402B00F29C8205
:10112000B0EE480AF1F7BAFFB0EE40AAB4F9783849
:1011300009EE103AB8EEC99A29EE2A9A39EE280A31
:10114000FDEEC07A17EE903A2033402B00F28782F2
:10115000F1F7A4FFB0EE40BAFDEEC97A17EE903A6F
:101160002033402B00F27E82B0EE490AF1F796FF61
:10117000B0EE409AB4F97C3808EE103AB8EEC88A5E
:1011800028EE2A8A38EE280AFDEEC07A17EE903A49
:101190002033402B00F26982F1F780FFF0EE408AA5
:1011A000FDEEC87A17EE903A2033402B00F26082B1
:1011B000B0EE480AF1F772FF69EE806A68EE8A7A4B
:1011C000F0EE665AE7EE895A954B28EEA96A20EEB2
:1011D0000A7AC3ED035AF0EE465AE7EE495AE6EEB4
:1011E000897AA6EE497A68EE8B8A2BEE400A2AEEBF
:1011F0004BAA69EE8B9AC3ED008A83ED010A83ED59
:10120000029AC3ED045A83ED05AA83ED067AC3ED75
:10121000077AC3ED089A07F03DFB40B9022101208F
:10122000F4F73EFF7F4A138843F00103138094F8DC
:1012300044387D4F012143F00203084684F84438C6
:10124000F1F7FEF800210846F1F7FAF80021022034
:10125000F1F7F6F80A260120F0F7CCF80020F0F7B5
:10126000C9F81920F5F746F83B68DB0302D40120E2
:10127000F1F7BCF81920F5F73DF80020F1F7B6F8C2
:10128000013EE8D131463046F1F7DAF83146012027
:10129000F1F7D6F8F3F736FF644B654F186814F092
:1012A0000DFC644B18880EF005FE634B3A781A70FB
:1012B00003F060FE2A68614B12F4805F9E8A18BFBB
:1012C0005F4A9B7818BF9688042BB84604D14FF428
:1012D0008050F1F74DFB002603F06EFC594B304671
:1012E00019780FF09DFD94F8443843F0040384F816
:1012F000443814F009FA14F0C1F9534B1B680BB1D0
:101300000FF068FC14F04EF903F03CFF16F0CEFB32
:101310004FF4197200214D48DFF85C914C4E1EF0DD
:1013200040FDFFF7DBFC4B4B00271F809F7012F046
:101330005DFE494B37604FF0FF3AC3F800A04846C6
:10134000464BC4F8803808F003FF454A84F88E788D
:10135000012384F88C38537884F88DA80D3384F8F1
:10136000883813781E3384F889383368042B04D006
:101370005A1C32603B4A42F823902B689F0340F18D
:101380008E8094F89C38384FDFF8F0A0C7F800A0A2
:10139000013B84F89438C82094F89D3884F8953837
:1013A000F4F7A8FF3868DFF8D89015F0EBFC89F85F
:1013B0000000C820F4F79EFF3B68C4F8A4380AF187
:1013C00010072A4BC4F8A038384608F041FE012324
:1013D00084F8AC38002384F8AE38FF2384F8AD38A5
:1013E000082384F8A838152384F8A938204B1F60F7
:1013F00099F800303BB13368042B04D05A1C32609A
:10140000184A42F823701B4C10220021204639E074
:10141000304F002035FA8E3CDB0FC93F941400207A
:1014200094430020143700205C2E00204836002012
:101430003434002028440020D4560020484700209F
:10144000343000201D500020D0560020286B002092
:10145000C43C0020F03600200C060020CC0103081C
:101460001C360020C83C002038360020F801030854
:101470002837002018370020AC2C0020BC2C00207E
:10148000313700201EF08DFC002009F0A7F9EFF79E
:10149000EDFD064609F0BCF9774B3344E360774C29
:1014A000002323702B68DE0308D509F0FFF8012321
:1014B0002370734B93F8F10015F0F8FA2B68580578
:1014C00001D50AF0E7FD2B68190101D511F0B4FD33
:1014D0001BF026FA98F80030052B03D1694B4FF426
:1014E000C8721A80684B694C1A684FF47A73B3FB60
:1014F000F2F3C3EB431203EB8203654ADB00A2F86D
:10150000B430644BC8224FF400601A8016F0CAFF52
:1015100098B1614B90F9020093F83230002B14BF60
:101520001823002301930323009300224FF49653C2
:101530004FF4006116F03EFC2060236813B1574B56
:10154000574A1A604FF4005016F0ACFF554C98B152
:10155000514B90F9020093F83230002B14BF08234E
:10156000002301930323009300224FF416534FF4FA
:10157000005116F01FFC2060236813B1474B4A4A04
:101580001A604A4A137843F008031370FFF730F8E3
:10159000474B1A68920306D5464A07215172117AC1
:1015A00041F001011172444A12681A6019F000FCFE
:1015B000424A138843F08003138017F053F9FFF772
:1015C000FBFA3F4A92F8443863F07F0382F84438CC
:1015D00007B0BDEC088BBDE8F08F9B047FF540ACF5
:1015E00010F04AFB3CE4314619F0B4FD5CE4012FF5
:1015F0007FF416AD404617F03DFA7068F0F7E6FE4E
:101600004FF4E073336137703623002604A88DF859
:1016100010308DF811708DF812608DF8137007F08E
:101620006BFF372305A88DF814308DF815708DF8F1
:1016300016608DF8177007F05FFF224AD36943F0F8
:101640003003D361204B1E85A3F82864E8E401230E
:1016500034E5DFED1E9A5BE59FED1CAA66E59FED84
:101660001BBA79E59FED199A84E5DFED188A97E5B5
:101670009FED160AA0E500BF404B4C00FC3800204F
:10168000F0370020EC700020644D0020206E002018
:10169000E04A0020EA7000204F2F00204037002051
:1016A0009C000020DC350020B8000020FC31002028
:1016B000744D002018370020B43C0020143700205F
:1016C0002C24002000100240001000400000000008
:1016D00008B50E4B1978012913D00DD3022902D178
:1016E0000020EFF787FEEFF7C1FC094B00F5F4206F
:1016F00000F59070186008BD00210846F0F7A0FEC4
:10170000F1E70020F0F79CFEEDE700BFF37000204A
:10171000F47000202DE9F04F83B0484C484F019001
:10172000019803685B699847002840F08380DFF8E0
:1017300018914448D9F80430DFF810E1C3F30803E6
:101740004FF00A0A4FF0100C4FF47A75002B3BD182
:10175000EFF31183002B37D10168A26800BF036843
:101760009942F9D1DEF8006005FB06F39B1AB3FB42
:10177000F6F305FB013101260091D9F80430C3F3DB
:101780000803002B3BD1EFF31183002B37D1036803
:10179000A16800BF02689342F9D1DEF800B005FBF2
:1017A0000BF2521AB2FBFBF205FB0323009A9B1AC1
:1017B000B3F57A7FE1D3BAF1010AB1D0D9F8043098
:1017C000C3F30803002BC3D0EFF311828CF312880C
:1017D000A6682368D90302D501233B60A668036885
:1017E0003968D2B282F31188DEF80020194405FB73
:1017F00002F39B1BB3FBF2F305FB0131BBE7EFF3F5
:1018000011888CF31288A1682368DB0344BF3E6013
:10181000A16803683A685FFA88F888F31188DEF8EF
:1018200000801A4405FB08F35B1AB3FBF8F305FBD1
:101830000233BBE703B0BDE8F08F00BF10E000E06B
:10184000846200208862002000ED00E08C620020AD
:10185000124B1A6890420CD09A68904215D01A69BF
:10186000904214D09A69904213D01A6A904212D0D2
:101870007047002110B403EBC1040022A28043F89A
:101880003120C2625DF8044B70470121F2E702216A
:10189000F0E70321EEE70421ECE700BFE44E00206F
:1018A000F8B50A4E05460024A359AB4204EB0607DF
:1018B00007D12846FFF7CCFFCC22002138461EF086
:1018C00070FACC34B4F5197FEED1F8BD286B002046
:1018D0002DE9F04FDFF884B32DED028B9BF800303B
:1018E0008BB0072B099000F0468700230793CE4C5E
:1018F000236805935D0500F1EE84CC4B1B680693CD
:10190000180700F11084CA4BCA4DB3F800A0CA4CA6
:10191000CA4BCB491E68B1F906907289914580F295
:10192000A581C84B4FF07E521A60DFF8348394F9DA
:101930000820B1F900E0B8F81870207994F805C0D3
:10194000AEEB0703002A14BF01224FF0FF32002B39
:10195000B8BF5B42B3F5FA7FA8BF4FF4FA73984261
:1019600080F25E811B1A07EE903AF8EEE77A77452F
:10197000C5ED007A03DDF1EE677AC5ED007AB1F9C5
:1019800002E0AEEB0703002BB8BF5B42B3F5FA7F72
:10199000A8BF4FF4FA73984280F27B811B1A07EEBE
:1019A000903AF8EEE77A7745C5ED017A03DDF1EE7E
:1019B000677AC5ED017AB1F90410CB1B002BB8BFD3
:1019C0005B42B3F5FA7FA8BF4FF4FA736345CCBF0F
:1019D000A3EB0C0C4FF0000C02FB0CFC07EE90CAC2
:1019E000F8EEE77AB942059BC5ED027ABCBFF1EE8D
:1019F000677AC5ED027A13F48053049300F0EE8009
:101A0000B9F5FA6F4A46A8BF4FF4FA62B2F57A7F89
:101A1000237BB8BF4FF47A72A2F57A72002B40F0A4
:101A2000F5808949DFF83CE281FB0230D317C3EB34
:101A30006013581C6FF0630C3EF910003EF913E080
:101A40000CFB0323A0EB0E0003FB00F381FB03213F
:101A5000DB17C3EB61139E440FFA8EFE07EE90EA8C
:101A6000049BB8EEE78A85ED038A002B40F0B18332
:101A70001AF04003089340F0C982069B13F0140F3C
:101A800003D01AF4027F40F03284704B1B7823B1EC
:101A9000B8F81A304B4580F2878294F83E701FB137
:101AA0001AF0030F40F03B8594F84420002A40F0E0
:101AB000BC8398F81E70002F00F0EE80022F00F01B
:101AC0002785032F00F00885614B598898F81F304F
:101AD0000233DBB2002A00F00E85002900F00B85EE
:101AE0005C480768B1FBF7F10FB2A4F87470ABB3B0
:101AF00007EE907AF8EEE77AF7EE006A86EEA77ABC
:101B0000012BD5ED007AD4ED226A77EEE67A67EE06
:101B1000877AC4ED1E7A21D0D5ED017AD4ED236AFF
:101B200077EEE67A022B67EE877AC4ED1F7A15D03E
:101B3000D5ED027AD4ED246A77EEE67A032B67EED0
:101B4000877AC4ED207A09D0D5ED037AD4ED256AE1
:101B500077EEE67A67EE877AC4ED217A9BF800107B
:101B6000092901F08880002F40F39B8093B394ED06
:101B7000227AD4ED1E7A77EE877A012BC4ED227A91
:101B8000C5ED007A21D094ED237AD4ED1F7A77EE5B
:101B9000877A022BC4ED237AC5ED017A15D094ED36
:101BA000247AD4ED207A77EE877A032BC4ED247A59
:101BB000C5ED027A09D0D4ED257A94ED217A77EE3D
:101BC000877AC4ED257AC5ED037A013B022BB8BFB5
:101BD0000223DBB2002A18BF022363E0B8F81A2000
:101BE0009145C0F2F081B9F5FA6FD4BFC2EB090399
:101BF000C2F5FA634FF47A7101FB03F1207BC2F561
